:020000040800F2
:10000000005000209951010839520108813B010834
:100010003952010839520108395201080000000024
:10002000000000000000000000000000395201083C
:10003000395201080000000039520108ABED0008F8
:100040003952010839520108395201083952010860
:100050003952010839520108419E00083D9E0008AE
:100060003952010839520108395201083952010840
:1000700039520108395201086DAD000839520108A2
:10008000CDD200083952010839520108395201080D
:10009000395201083952010839520108399E0008C5
:1000A00039520108C5D1000839520108D5D10008DC
:1000B000B5D10008A5D1000895D100085963000802
:1000C0005D63000851630008556300083952010858
:1000D0003952010865AD00085DAD000855AD000856
:1000E000B9ED00083952010839520108000000003A
:1000F0000000000000000000000000000000000000
:0C01000000000000000000005FF808F1A3
:100110002DE9F04F754B764EA5B033600023736028
:1001200010F024FC18B910F043FC08F0D1F908F0E5
:1001300075FA704A704C1378704D43F001031370D8
:1001400000230C930D930E934FF4E0130F93236849
:10015000A87B43F480332360A36943F01003A361B9
:10016000236803F400330D930C9B01330C930D9B18
:100170001BB90C9BB3F5A06FF2D123685E4913F451
:10018000003301D0022315E00A6842F001020A6040
:100190000C93236803F002030D930C9B01330C9323
:1001A0000D9B1BB90C9BB3F5A06FF2D123689B0785
:1001B00039D501230E93524B52491A6842F010026E
:1001C0001A601A6822F003021A601A6842F00202EA
:1001D0001A606368636063686360636843F48063A4
:1001E0006360494B1A68043B22F070425A60474AE8
:1001F0001160616821F47C116160596841F000412F
:100200005960D96821F40041D9609B681F0449BF37
:100210003F4B4FF4E01313604FF480130F930E9B8A
:10022000012B01D117E0FEE7022B18D168B10F9B1B
:10023000B3F5801F02D14FF4A01305E00F9BB3F577
:10024000E01F02D14FF400130F930F9963680B4323
:1002500043F4803302E0636843F46013636023680F
:1002600043F0807323602168234B8901FBD55968D3
:1002700021F003015960596841F002015960636837
:100280001D4903F00C03082BF9D14B68DFF88C8073
:1002900003F00C03042B03D0082B03D0194B12E0FE
:1002A000136810E04B684868C3F38343C70303F146
:1002B000020301D4174905E0496811F4003F1168B1
:1002C00018BF49084B43C8F8003063681249C3F3AC
:1002D00003130B44197ED8F80030CB40C8F8003027
:1002E0001368084A93421BD101221DE0B77C000825
:1002F00068080020F0330020001002402C1000207D
:100300000020024000127A00041001404400002046
:10031000001BB70000093D0010A20108600000208A
:100320008A4A934202D10222894B1A70DFF878A2DE
:10033000884BDFF878C2CAF80C30A3690DF1900B36
:1003400043F00103A361636A834FB360636A60464D
:1003500043F080736362A3694FF0000943F01C030C
:10036000A3614FF6FF732BF82C3D5946CDF814C00E
:100370008DF866900DF0B5F8384659460DF0B1F895
:10038000594676480DF0ADF8754A5846536843F023
:10039000007353600FF01CFA724A199B4946B3FB75
:1003A000F2F3714A714813600C2217F050FAD8F832
:1003B00000304FF47A72B3FBF2F36D4A013B5360A5
:1003C000F0238AF823300723C2F808901360AB6843
:1003D000DFF8DC91DFF8DC81C9F8003098E80F0025
:1003E0008BE80F00A3694FF0100A43F00803A361E4
:1003F000A369199843F00803A36108233B611AA974
:10040000C7F810A00DF06DF81B981CA90DF069F845
:10041000D9F80020100713D5564B93F89221012AE2
:100420000ED8554993F89321896811F0805300F054
:10043000F28505E04F4B002283F8932108F0C2FAC1
:1004400064200EF0A8FCA0224C48002117F0FFF910
:10045000E369002243F00703E361A36943F4006307
:1004600043F00C03A361444B4FF0000803F10C016F
:1004700002F8018001320E2AF5D1FF229A76DA764F
:100480001A775A773E4B3F4A41461A603E483C2213
:10049000D9F8004017F0DBF94146C4F38017052373
:1004A0003A4ADFF8E4E0885C0C224A4302F80E0086
:1004B00047B91E3801289FBFFF2003F1FF3302F820
:1004C0000E00DBB201310529EAD1314A95F805A0C9
:1004D0001370304B304983F800A0304B264A33620A
:1004E000C0330B602E4BA10603EBCA035B7848BFF9
:1004F00001235362002340F2DC512A4A22F81310F0
:100500000133082BF7D112A800211C2217F09FF904
:1005100014F4007CDFF8A09004F400684ED0A3042B
:100520000AD4B8F1000F0AD095F8862109F10C031E
:10053000012A08BF4B4604E0CDF8189002E009F10B
:100540000C030693CDF860B03AE000BF001BB70083
:100550001B3400200005FA05000C0140001001408A
:100560000000014040420F00182A0020A41F002074
:1005700010E000E02C10002068080020602A002015
:10058000E02B002020120020E42B002071C901087C
:10059000E10F0020740300207C2B0020401000207D
:1005A000E8C601084A0F002000ED00E00008014005
:1005B000242F002038A2010810A20108CDF818C08D
:1005C000BAF10E0F04D00AF0EF0ABAF1080F02D107
:1005D00001238DF85A300120CDF81CC00EF098FA96
:1005E000DDF81CC018B14088003018BF0120C4F3EA
:1005F00040038DF84E30C4F3403300F001008DF815
:100600004830C4F3C0338DF84D008DF850708DF82C
:100610004B30B8F1000F07D095F8868108F1FF370D
:10062000D7F1000848EB0708C4F300438DF85130B8
:100630001CF1000318BF01238DF85230736AB5F81E
:100640004801003318BF01238DF85330C4F3005321
:100650008DF85430B5F84A31ADF85E00ADF8583039
:10066000E004B5F8563148BFBA48ADF85630C4F387
:10067000804348BFB0F850018DF84F30B5F8543181
:1006800048BFADF85E00B3F5FA7FADF85C3084BFCB
:100690000023ADF85E3095F8D631AF4886F82830A3
:1006A000002386F8293043709DF85A3004F0010188
:1006B000002BC4F3C0028DF84C808DF849108DF8E2
:1006C0004A200CBF0023022301B902B1013309EB18
:1006D0008309D9F838309A1E1A33099300230892F7
:1006E0000793089B33F8024F08934FF6FF739C4221
:1006F00000F08E819DF84D20E3B2240AE5B21AB1D4
:100700009A1E012A40F27F819DF8502032B1934910
:100710001A018958924A914200F075819DF8510062
:1007200030B18E491A0189588D4A914200F06B818F
:100730009DF84E2052B18949059E01EB03114A688C
:10074000B24203D10A89102A00F05D819DF84B2046
:1007500052B18249059E01EB03114A68B24203D1AE
:100760000A89022A00F04F819DF84C2052B17B4942
:100770007C4E01EB03114A68B24203D10A89022A76
:1007800000F04181189E7EB1744F326807EB031769
:100790007968914208D13A89B188914200F0338159
:1007A000F188914200F02F81022C02D19DF848205F
:1007B00003E0012C04D19DF84920002A00F0238198
:1007C0009DF85320654C1E015AB19DF85A2042B93C
:1007D000A3F10802012A04D8A25963498A4208BF3A
:1007E00004259DF85420344452B19DF85A203AB95A
:1007F00010B10C3B012B01E0043B032B40F2EB80DA
:10080000012D48D1594FDFF854A1FF2387F87030EC
:1008100087F871300AEB06035A7B586803F1080920
:100820001B894FF00008ADF8643019A9022387F83E
:100830007480C7F880408DF867308DF8662087F89F
:100840002C80C7F83080C7F83480C7F83880C7F8E4
:100850006C8087F8728087F873800CF042FE5AF83B
:10086000060099F80210424609F037F92046414641
:100870002A460AF0CBF93E4BC7F88C80C7F8843083
:100880003C4B2046C7F8883007F1840107F1880205
:100890000AF004FAB7E0022D4CD19DF81C204FF06D
:1008A0001C0C0CFB02FC314B002703EB0C080A93D9
:1008B0009DF81C304FF0010988F87530274B88F8F7
:1008C00076709A19517B506802F1080A12898DF8E6
:1008D000661088F87E7019A988F87490C8F880406E
:1008E000CDF82CC0ADF864208DF867500CF0F9FD00
:1008F0001A4B9AF8021098593A4609F0EEF8204639
:1009000039464A460AF082F91B490A9BDDF82CC099
:10091000C8F8841019496344C8F8881003F18401A9
:10092000C8F88C7020460A1D0AF0B8F9079B4B44A2
:10093000079368E0032D4CD19DF84F300B4D104EBE
:1009400003B395F82A70204608214FF6FF72002362
:1009500033E000BF2C1000209108002094C401084F
:1009600000040040000C0140002C014068080020F9
:100970004995000829960008159B00081F95000856
:100980002C2A0020BDF85C2095F82A70B2F5FA7F79
:10099000BDF85E300BD986492046B1FBF2F2082142
:1009A00092B209F0EFF8834B46F827000AE082493B
:1009B0002046B1FBF2F2012192B209F0E3F87F4B3D
:1009C00046F82700C36095F82A30013385F82A30AD
:1009D00019E0042D17D1BDF85620774B784D93FBC5
:1009E000F2F22046BDF85830012192B295F8296004
:1009F00009F0C8F895F8293005EB86060133C6F8EA
:100A0000540185F82930089B099A93427FF469AE16
:100A10006B4D6C4B95F82920002485F874216A4AA7
:100A20001C7016789846A6F11702022A19D82B6A6C
:100A30000021185903EB040913F05EFB10B16B6A37
:100A40005BBB25E0614F99E80F00274487E80F0062
:100A500098F8003010340133C02C88F80030E6D10B
:100A6000EDE75B4B13F836E003EBC603D3F804C0A5
:100A700088F800E0BCF1000FE1D07445DFDA534F95
:100A800023011F4463440FCB013487E80F00F4E7D0
:100A9000504F3B68DA0424D41DE04F4B4F4A13F803
:100AA000360003EBC6035C681070002CF0D0002306
:100AB0008342EDDAC3EBC3016218D2F800C0DFF85D
:100AC00044E1013341F80EC001EB0E079188B98073
:100AD0009279BA71ECE706F0EF03082B404B25D171
:100AE00026E098F80030012BF5D93E4C04EB0313B7
:100AF00003F1100810344445EDD054F8100C4FF0B9
:100B00007C5113F065F94FF07C5144F8100C54F807
:100B1000140C13F05DF94FF07C5144F8140C54F8A8
:100B20000C0C13F055F944F80C0CE3E70E2E08D129
:100B30001A78182E42F010021A7008D10EF0D0FB6D
:100B400005E01A78192E22F010021A70F5E70EF05F
:100B5000ABFB3B68244C5B035EBF244B01221A7045
:100B6000234B24481A78994642F004021A70224A0C
:100B700011789046022934BF142310238DF8663073
:100B80004FF002038DF86730A3694FF4805243F0B1
:100B90000403ADF8642038BF0026A36128BF0126F6
:100BA00019A90CF09EFC154B76B3154A2DE000BF39
:100BB00000127A004996000840420F00399600085A
:100BC000680800205C2A002074030020B002002086
:100BD000E8C60108242F0020F8AF0108082B0020E8
:100BE00028180020B802002000100240E007002072
:100BF000F0330020000801401B340020FC330020AB
:100C000029E80008092B0020714A00201A600EF024
:100C1000E1F8704B704E93E80300A3698BE8030082
:100C200043F00803A36119981AA90CF05AFCE36970
:100C3000304643F48043E3612369594643F48043DB
:100C4000236118238DF866304FF42043ADF86430EB
:100C500003238DF867300CF044FC04224FF48043EA
:100C6000304659468DF8662005924FF4805AADF80B
:100C700064300CF036FC1023304659468DF866304F
:100C8000ADF864A00CF02DFC2369322043F48043BE
:100C90002361236923F480432361504B198801F4B5
:100CA000415141F4457141F003011980998B21F4C0
:100CB00000610904090C998307211982198889B2F6
:100CC00041F0400119809F23C6F810A08DF84430F0
:100CD00000238DF845308DF846308DF847300EF002
:100CE0005AF8059AC6F814A0584611A911F0EAFB63
:100CF000C6F810A09DF866309DF865201B0243EAF7
:100D000002439DF867201343354A934215D03220A1
:100D10000EF041F8C6F814A0F52011F009FCFF20F0
:100D200011F006FC7028C6F810A006D198F8003023
:100D3000022B02BF2B4B03221A7098F80030032BB2
:100D40000CBF1F20022006F0BCFE98F80030032BD9
:100D500003D001200CF016FE07E002200DF0D8FEB3
:100D60000028F6D04388002BF3D03E684FF0100BDC
:100D700006F40043059306F4006307931A4B002121
:100D800018465A46089398F8008016F060FD4FF612
:100D9000FF72089BADF8442002224FF0000A16EAC9
:100DA00002018DF846208DF847A01E4620D024A9C8
:100DB00021F84CBD0D480EF0B7FE04233370072216
:100DC000012386F801A0B370F2709A4611E000BFCB
:100DD0003DE8000858A20108000C0140003800401E
:100DE000152020001B340020692C00200008014041
:100DF0008A46B8F1010F12D9202224A921F84C2DDE
:100E00009F480EF091FE052201233272B3720AF15F
:100E10000102072386F809A0F3725FFA82FA059BA4
:100E20008BB124A9022221F84C2D95480EF07CFEAE
:100E300001220AEB0201072386F805A03271B27184
:100E4000F3715FFA81FA079B93B1022224A921F87A
:100E50004C2D8C480EF068FE092201233273B373C7
:100E60000AF10102072386F80DA0F3735FFA82FAF4
:100E70006268854842F4404262606269DFF8088235
:100E800042F001026261A26942F40072A2610EF0B6
:100E900027FC7E4A002419927D4ABAF1010F1A926A
:100EA00094BF224680221E924FF480721F924FF40C
:100EB0008062209220224046219219A94FF40052CC
:100EC00022921B94CDF870A01D9423940EF0EAFB9F
:100ED000D8F800206F4942F00102C8F800204A68A3
:100EE000BAF1010F22F4702294BF0020012022F4F5
:100EF000807242EA00224A608868674A0AF1FF333A
:100F0000024042F4602242F002028A60CA6ADBB206
:100F100022F4700242EA0353CB6201233219917822
:100F2000002963D0305D591C0928C9B2D278DFF896
:100F300064C112D9A0F10A0EDCF80CA00EEB4E0E23
:100F40004FF0070808FA0EF82AEA080802FA0EF22B
:100F500048EA0202CCF80C200FE0DCF8108000EB2D
:100F6000400A4FF0070E0EFA0AFE28EA0E0E02FAA9
:100F70000AF24EEA0202CCF81020062BDFF814E148
:100F800010D8013BDEF8342003EB83034FF01F0C35
:100F90000CFA03FC22EA0C0200FA03F31343CEF826
:100FA000343022E00C2B10D8073BDEF8302003EB66
:100FB00083034FF01F0C0CFA03FC22EA0C0200FA28
:100FC00003F31343CEF830300FE0A3F10D02DEF847
:100FD0002C8002EB82021F23934028EA030C00FAC4
:100FE00002F34CEA0303CEF82C300B460434102CE9
:100FF00094D1284B9A6842F480729A609A6842F0C1
:1010000001029A609A6842F008029A609968214A3F
:101010000C0743D5FAE7013A092A3FF611AAD8F896
:101020002C0006935946C7F814A0CBF80000059889
:101030000CF057FA059B3C201A46082313610DF06B
:10104000AAFE069BC7F810A01F4695F893319F4251
:10105000BFF6F0A9059BDFF82CA04FF00808CAF8EE
:1010600010807820C3F814800DF08AFE059BCAF822
:1010700014807820C3F810800DF082FE0137E4E779
:1010800000080140000C0140080002404C240140CF
:101090007A2C002000240140FDF7F1FF936843F013
:1010A00004039360C14B9E6816F00406FAD1C04C4D
:1010B0009A68B4F85C0142F4A0029A60002840F0FB
:1010C0001386B4F95E31002B40F00E86B4F960311E
:1010D000002B40F009863B6898031FD5C8200DF00F
:1010E0005AFEAE200CF0B9FB08B10CF0BBFB85F842
:1010F0007501C8200DF04FFEAE4B0021C5F87831C8
:10110000AD4D0C22284616F0A2FB0223EB7010F026
:1011100052FA0DF019FEA94B0344AB60A84D94F8A8
:101120006CC12B68B4F86401B3F956E094F863110C
:1011300094F86B21CDF800E0B4F80CE06346CDF8EC
:1011400004E094F80FE0CDF808E008F065FF10B96E
:1011500001200DF09BFE99F80030102243F00203AD
:1011600089F80030974B4FF00A085A6108221A613B
:10117000DFF850921920D9F80C3008F1FF3883F0CD
:101180001003C9F80C30D9F80C3083F00803C9F803
:101190000C300DF000FE01200DF01CFE19200DF0AA
:1011A000FAFD00200DF016FE18F0FF08E0D108232C
:1011B000C9F810304FF0100A834BC9F810A01A6814
:1011C000984612F0080F09D0804BC9F814A01B688C
:1011D00098477F4B0122C9F810A01A707D4BDFF8A9
:1011E0001C921B68187B12F09FFD7B4912F0F0FDEA
:1011F00007F04AF88246B9F8000012F095FD514612
:1012000012F0E6FD16F030FD744B1880B9F80000BE
:1012100012F08AFD0146724812F08EFE714912F0FA
:101220008BFE714B6C491860704B186912F0D0FD41
:101230006F4912F0CDFD6F4BFF2118606E4B1B22E2
:10124000184616F004FBDFF8B8E10022734602707E
:10125000D8F80020012112F0020F8EF800101FBFF5
:10126000417003218EF80010022118BF81705107D0
:1012700041BF9EF8001001F1010E83F800E04FF02D
:10128000030E48BF00F801E012F00A0F0ED01A78E2
:1012900004218154511CC9B24FF0050E00F801E041
:1012A000D11C02321970D2B20621815439688F06DE
:1012B00041BF1A78571C1F70072748BF87540A067A
:1012C00008D51A7809278754971C01321F70D2B2AB
:1012D0000A2787546779082F01D00E2F08D11A7872
:1012E00002F1010E83F800E04FF00B0E00F802E06F
:1012F0001A7811F4803F4FF00C0C00F802C002F194
:10130000010E1CBFDFF8F8C002325FFA8EFE83F8D0
:1013100000E01FBF8CF80020374A4FF00E0C02F897
:101320000EC04A0748BF1A784FF0120C41BF02F1B5
:10133000010E83F800E04FF0100E00F802E01A787A
:1013400011F4806F02F1010E5FFA8EFE83F800E067
:1013500000F802C00ED094F820C2BCF1000F09D0F2
:10136000DFF89CC002328CF80020234A4FF0130CA7
:1013700002F80EC01A7811F4007F4FF0140C00F838
:1013800002C002F1010E1CBFDFF874C002325FFA26
:101390008EFE83F800E01FBF8CF80020164A4FF045
:1013A000150C02F80EC0182F40D12BE0002401408C
:1013B0002C100020B611002014290020404B4C00B6
:1013C0005C0F0020000C014024180020DC1F0020CE
:1013D000682C0020D001002035FA8E3CE00100206E
:1013E0000AE81C4100401C4624010020341F002054
:1013F000BD378635CC010020290F002028000020B1
:10140000280F00201A784FF0160E00F802E002F1C3
:10141000010E5FFA8EFE4FF0170C00F80EC002F1BD
:10142000030E0232D2B283F800E087540A0341BFB0
:101430001A78571C1F70192748BF8754CF0541BF22
:101440001A78511C19701A2348BF8354002198221E
:101450009E4816F0FCF908F012FD9D4A9D4BB4F829
:1014600052111A609C4BB4F8980119809B490023D3
:101470000B808B709A490A6081B29A4A22F8131045
:101480000133122BF9D1984F3B68D9045CBFB4F8F3
:101490009E1111801B0740F1C58094F89231062BF4
:1014A00000F2BA80DFE803F004070E3954747400C8
:1014B00045F2F05201E042F6F8228C4B1A8008F017
:1014C00067FDA8E042F6F822884B1A8012F02CFC47
:1014D000874912F07DFC874912F070FB12F064FE20
:1014E0000023854A42F823000133122BF9D1834AA5
:1014F000834940201160834A13700DF043FB00289C
:1015000000F08A8001234FF0070A90F90000402183
:101510008DE808047C4A7D4B78E042F6F822734B54
:1015200040201A807A4A754B1A60764B10221A7046
:101530000DF028FB00286FD001234FF0000990F92F
:10154000000040218DE80802724A4FF4E1335DE06B
:1015500042F6F822654B40201A806F4A674B1A60AA
:10156000684B08221A700DF00DFB002854D001239F
:101570004FF0000C90F9000040218DE80810674AF8
:101580004FF4E13306F0CAFA654BC3F87C013FE043
:1015900042F6F821554A062B11805A494FF00C02A9
:1015A000DFF8B4C1DFF8B4E15E4C5F480A700FD0D9
:1015B000002323708CF800308EF800301B2303705A
:1015C0005A4B4FF4E1341A70594B05221A700CE053
:1015D000002121708CF800108EF80010212101707C
:1015E0005249544C0A70524A1370534A434B40209C
:1015F0001A600DF0C7FA78B101234FF0000E90F990
:1016000000008DE8084023464C4A402106F086FA47
:10161000003018BF012028B9082006F027FF484AEB
:10162000364B1A603B68374A13F4804F1FBF0821BE
:1016300011704448314918BF086042F20101194055
:1016400099B144F6206029490880980441BF0821D7
:1016500011703D48294948BF0860D90741BF0C2196
:1016600011703A48254948BF086011781C06A1F15D
:101670000401517040F1AE802948DFF8E4A04FF03A
:101680000009334CC0F880A14946152200F5C2700C
:10169000DFF8D0B084F80190C4F80490C4F8089042
:1016A00016F0D5F8AAF105034846CBF800300BF048
:1016B000B2FA284B02201B68E3600DF063FA0028A1
:1016C00052D1802006F0D2FE7DE000BF841E0020B3
:1016D000B6110020000E0020040E00209C330020D4
:1016E00090330020602F0020242F002020020020B3
:1016F000CDCCCC3F0000B044A03200202C00002014
:1017000059330108201F0020FD340108A086010084
:10171000453301085134010831330108053401080B
:1017200068080020B82B0020DB2B00208B33002022
:10173000DC2B002090D0030055F5000869F5000867
:10174000B533010889330108A53301089533010831
:1017500040010020482F00208C330020B92B0020AE
:10176000201200206001002090F805E06378C7494E
:101770000C2202FB03125278724504D00133DBB213
:10178000042BF4D900236370DBF8003062781B78F7
:1017900090F90000002B4FF00C0303FB021314BF61
:1017A0004FF0030E4FF0010E00225B78CDF800E001
:1017B0000192022106F0B2F9B54B1860002880D0E2
:1017C00001200BF028FA2868B24B00F5C5721A60A8
:1017D0000BF0C8FA3B68980553D5AF4AAF4C069B4F
:1017E000102523609369AE4843F001039361069B83
:1017F00010A91B888DF84250ADF8403002238DF8B7
:1018000043300BF06EFE2368A5485B8810A9ADF845
:10181000403004238DF842300BF063FE2368012032
:10182000197A0BF049FE23689E4A5B684FF0000965
:10183000536119A88DF86950012519938DF86890A6
:101840008DF86A500EF032F9236811A85B7A8DF892
:1018500046908DF8443003238DF845308DF847507D
:1018600010F012FE904B914A1B683C3B1360D8F875
:1018700000304FF0FF3243F01003C8F800308C4BBB
:101880001A608C4B8C4A8D4C13608D4A80331360E8
:101890003B680025D903257040F1AF8040F22A391A
:1018A000DFF854A2DFF8F0B10EF066FC4FF001084B
:1018B0004A465046294684F8008015F0C8FFDBF8F8
:1018C0001830804843F00403CBF818304023ADF8BB
:1018D000403018238DF8433010A903238DF842308F
:1018E0000EF022F9DBF81C30774A43F00203CBF804
:1018F0001C30764B764C1B68ABF6947BB3FBF2F353
:101900002288013B22F45C721204120C22809BB2EA
:101910001D22A2852385A4F81480238C23F00103C3
:101920001B041B0C2384238CA188228B23F002032D
:1019300022F0730212041B04120C1B0C89B242F039
:10194000600243EA0803A1802283A5862384238BB7
:1019500023F008031B041B0C43F008032383B4F893
:1019600044306FEA43436FEA53439BB2A4F84430D8
:10197000DBF8A83F43EA0803CBF8A83F58460DF030
:10198000AFFE544BCDF868A0199380231E934FF4FB
:1019900080734FF0100A1F9358464FF4005319A953
:1019A00022931D95209521952395CDF86CA0CDF817
:1019B00070900DF077FEA38911A89BB243F40073D9
:1019C000A381DBF8003043F00203CBF800308DF840
:1019D00044A08DF845808DF846508DF8478010F072
:1019E00053FD3D4B1A683D4B43F826200136202E0F
:1019F000F7D10BF083FC0BF081FC3B685A0540F1FA
:101A00008F80374C374BD4F8C46404201E600DF02F
:101A1000B9F80421C4F8C8040DF08EF8324B84F8EC
:101A2000CC0408201E600DF0ADF8304B0821186082
:101A30000DF082F82E4D84F8CD04002128462C228A
:101A400015F005FF8E236B704FF07C09E0234FF0FB
:101A50007D08EB7085F8009085F82B80254D2C22B1
:101A60000021284615F0F3FE8A236B701020A02376
:101A7000EB7085F8009085F82B80C4F8D0640DF0E9
:101A800081F81021C4F8D40438E000BF189E010882
:101A900010290020580E0020001002403C010020B8
:101AA000000C014000040140482F002038010020B4
:101AB0007C0F00205C120020F0180020E1070020BD
:101AC000542900200008014000366E01600000200B
:101AD000000400403404004060A20108E207002036
:101AE000680800201818002070180020BC1800207A
:101AF0004018002075180020010A00200DF01CF885
:101B000084F8D8042020C4F8DC640DF03BF82021D0
:101B1000C4F8E0040DF010F884F8E40411F010F9B2
:101B2000814B824C1B78022B65D1814A002513889A
:101B3000322023F040031B041B0C138013884FF446
:101B4000805623F038031B041B0C138013889BB2B0
:101B500043F0400313809F238DF844308DF84550A7
:101B60008DF846508DF847500DF015F98DF86550F9
:101B7000704D04226E6119A811A910F0A3FC2E610A
:101B80009DF866309DF865201B0243EA02429DF8ED
:101B900067301343684A934219D00AD8A2F51A4213
:101BA000033A93420CD002F51A420232934209D012
:101BB0001CE0624A934205D00132934207D015E0FF
:101BC000202300E0802323804FF4807302E04FF451
:101BD000807323806380A38822881B02A360534301
:101BE000E360574B012283F8E52404E000232380BF
:101BF0006380A360E360E4681CB3E40A26464FF008
:101C00000008A0450BDA08EB04056D100DF164091E
:101C1000E802494610220BF0D1FD0F2806DC0BF03C
:101C200053FA474BF602C3F8E8640AE0002359F878
:101C30002320013254D10133042BF8D12E462C46F7
:101C4000DFE73B683F4A13F4002318BF01231370FA
:101C50000DF07AF83C4B18603C4B5A791946052A2E
:101C600002BF3B4B4FF4C8721A803A4B4FF47A7262
:101C70001A80394BC8221A80384A137843F0080377
:101C80001370374A137823F00203137040F60203EF
:101C90003A6813406BB13348334B1860334B032021
:101CA0001870334B012018703248002303803248EB
:101CB0000380930341BF314B04221A71DA7844BF89
:101CC00042F00102DA708B6801223B602C4B1A70E3
:101CD0002C4A137863F07F03137025B0BDE8F08FB2
:101CE00005F101082546AAE7274B00221A7000B229
:101CF00012F01AF8254912F06BF81990B4F95E0148
:101D000012F012F8214912F063F81A90B4F9600148
:101D100012F00AF81D4912F05BF81D491B9019A832
:101D200006F0BCFAFFF7D7B91B34002018000020DA
:101D300000380040000C014018BA20001740EF00A6
:101D4000680800206C300020000200202C100020C9
:101D5000100E00201234002010340020281800201B
:101D600019340020A8110020101800207418002039
:101D700054000020F80E0020FA0E00201429002044
:101D8000E0070020F03300204800002035FA8E3CA8
:101D9000282C0020954A2DE9F04F1568944C05F544
:101DA0009C43944E20332360336889B013F4804FF2
:101DB000059205D111F06CFC10B923790133237120
:101DC0008D4A13784BB18D4909688D4240F2E58008
:101DD00003F1FF3882F80080DFE09846884B5FFA15
:101DE00088F51F78DFF83892AF4231D9D9F8003042
:101DF000072D98BF595D834B88BF29461B688048D3
:101E00009847032D1ED8D9F8002005F10E0302EBE8
:101E100083039988DA88A8B14FF47A73401A58433B
:101E2000531A90FBF3F040F6C90300F57A7098421C
:101E300005DC40F2EE239842B8BF184601E040F6B8
:101E4000CA0080B204EB4505E88008F10108C5E747
:101E500094F804800325B8FBF5F50F2384F82A30A5
:101E600094F82B3005EB4505019394F82C30C5EB25
:101E700008050393D9F80030DFF8ACA10293EBB268
:101E800004930025BD4255DA5F4B4FEA450933F80C
:101E900015B0019B53B911F0FBFB28B1039B002B3C
:101EA00008BF4FF0000B01E0DDF804B0029B988AF8
:101EB000584502D8D88A58450ED2E8B211F092FBA4
:101EC000032D8346DFBF94F82AE00120A8402EEAC4
:101ED0000000D8BF84F82A0011F0DAFB18B14B4893
:101EE00029F800B022E0049B94F876002AF813B099
:101EF00030B9B8F1020F15D93D4B012083F87600B7
:101F0000BAF80000BAF802300344BAF804000344F7
:101F10003F489BB229F800301BB2032093FBF0F33B
:101F20009BB200E05B46394829F8003001350AF1E0
:101F3000060AA7E794F82A203648A2F10F014A4280
:101F40004A4184F89020344B6AB1344A12685201F5
:101F500009D40268D9689A60521AC82A1DD9012288
:101F600083F8212019E002689868DA605B68121A29
:101F70009A4288BF284B4FF0000184F82B1088BF8D
:101F800083F821100025BD4207DAE8B211F02AFBE0
:101F90001E4B23F815000135F5E73368DD0405D540
:101FA0001E4B1B68D80701D411F07AF9059B1F68F6
:101FB0001B4B1A68907A002838D01449137B0138DB
:101FC00031F810001BB1C0F53B60083080B200B2A0
:101FD000A0F57A70B0F57A7FA8BF4FF47A7020EA46
:101FE000E07011F0A1FE0F4955E000BF0034002061
:101FF000540D0020242F002098330020943300201B
:10200000201F00202C0000205A0D0020602F0020EF
:10201000CC0D0020482F00209C330020240F0020EE
:102020009033002000007A44820D002033681904A8
:102030003AD5D4F89430934DFB1A002B34DB07F5D6
:102040009C432033C5F894308F4BD27A59798F4B0B
:1020500033F8113095F898109BB293FBF2F30131ED
:1020600001F00F0285F898202A4482F8993003463F
:10207000874A825C0130134410289BB2F8D11BB20E
:1020800093FBF0F000B26428A8BF642020EAE0705F
:1020900011F04AFE7F4911F04FFF7F4911F098FE81
:1020A00012F082F87D4B188033687D4D13F4807FE9
:1020B00000F00F817B4BDFF8F0919F4205D999F832
:1020C000022012B9012289F8022099F80220002A80
:1020D00000F0FF80744A95F8008092F82170C8F3F0
:1020E00080087A1E57425741704A002F9246116865
:1020F00018BF4FF0000BC1F38063019308BF4FF08E
:10210000030B99F82020052A00F2DD80DFE802F0B9
:10211000034E537988A5B8F1000F3AD0D4F8AC003B
:10212000B4F8B0100CF0CDFD012809D16049614A26
:1021300009681268C988642000FB0122C9F81020D0
:10214000019B6BB15A4A126812794AB111F0FAFC3C
:10215000032289F820204FF47A72C9F81C20D0E7B6
:10216000002F40F0B080534AD9F8101010684E4A42
:1021700088420AD9029211F0E5FC029A032182F802
:10218000201040F6B831D161BBE7012182F8201060
:10219000B7E7019B4FF4806013B106F057F901E0F7
:1021A00006F043F90022C9F810208CE0002F49D135
:1021B00011F0C8FCA5E727B1052289F820200120ED
:1021C00000E03846B8F1000F0CD0D4F8AC204FF046
:1021D000020BD189384A11805180918034490968B5
:1021E0004988D180334A1168D9F81420914202D825
:1021F000B8F1000F64D147F23052C9F81C20032215
:1022000021E02A7842F002022A7011F049F8294AA6
:10221000D9F81C1012680A44C9F81820042212E0E8
:10222000244A9FB11168D9F8182091424BD9234A0A
:1022300012781AB9DAF80020D30744D42A7822F0A9
:1022400002022A70052289F820205AE71268D9F87C
:102250001C100A44C9F8182035E01549154A0968C8
:102260001268C988642000FB01224FF48060C9F81D
:102270001020002289F8202089F8032006F0D5F8E4
:102280003FE700BF540D0020692C00207A2C00206D
:10229000ED0D00200000C84200C07F44800F0020E8
:1022A00019340020404B4C009C330020240F0020A8
:1022B000EC330020482F0020602F00201400002065
:1022C00000287FF41EAFBBF1000F02D058460CF07F
:1022D0009FFD924F07F5C570B7F852110CF0F1FC55
:1022E0000197834668B911F01FFC8D4B0022C3F89B
:1022F00000B0C3F804B0C3F808B08A4B1A605A6043
:102300009A602B785F0736D53368D80633D5864B6D
:102310001B78D9062FD4854B1B789BB1019B93F872
:10232000E231BBF1000F15D17BB1814B1A68D4F8B3
:10233000B4309B1A002B08DA10F0B2FF7D4B83F803
:10234000B8B018E0BBF1000F0DD110200CF060FD0B
:1023500001230EE03BB1764A4FF47A71126801FB1B
:102360000323C4F8B43094F8B83023B10CF038FD2E
:10237000002384F8B830019B93F8E0A193F8E111B1
:10238000B3F89AE1B3F89CC1002318466A4F80085D
:1023900037F9132001337245C4BF60F07F00C0B22B
:1023A0006245B8BF40F04000042BB946EED194F826
:1023B000B930604A834205D192F8BA30F92B04D87B
:1023C000013300E0002382F8BA30584B84F8B9009A
:1023D0001A785A4F9846E2B93B68DA0708D5BBF13C
:1023E000000F16D12B78DB0713D510F0A9FD10E0F4
:1023F0002B7858070DD54F4B93F82B304BB1504BE2
:10240000DB7833B911B110F04BFF02E0BBF1000FE4
:10241000F9D094F8BA30474A142BDFF840B140F0B5
:10242000AF8098F800301AF1000A18BF4FF0010A87
:102430006BB392F8B9305F2B11D12B7803F0040302
:1024400003F0FF0113B110F02BFF08E00B20039104
:1024500002920CF0DDFC029A039982F8BA10BAF1EC
:10246000000F14D094F8B9307D2B10D12B7803F0E5
:10247000040303F0FF0213B110F012FF07E00B207A
:1024800002920CF0C5FC2B4B029A83F8BA202B78F1
:1024900003F0040303F0FF01002B71D194F8B9306D
:1024A000244A572B15D1274B4FF47A721A80336880
:1024B000190601D50AF0A6FC234B1B685A0742BF38
:1024C000224A0A21118013F0080359D1204A1380AF
:1024D00056E03068400716D55A2B14D11D4B18789A
:1024E00020B119701C4B01221A7049E092F8BB30E0
:1024F00083F0010382F8BB300BB10C2000E00D200B
:102500000CF086FC3CE05D2B00F01F855B2B00F09F
:102510001E855E2B24D1032000F01ABD2C10002054
:102520007C29002004270020281800201400002007
:10253000482F0020540D0020602F0020240F002081
:102540009C33002012340020241800201034002076
:102550001C100020372D0020382D00205C0F00209B
:10256000562B01D106F02EFA98F80030002B00F01F
:10257000058594F8B9306F2B40F0FA8410F0E0FC38
:102580003368580732D594F8BB30A3B12B7859077C
:1025900011D5019BB9F90620B3F89A319A420ADDA8
:1025A0003B6813F0010301BFAC4A32211180AC4AF1
:1025B00008BF82F8BB303B68DA030AD5A94B1A780A
:1025C0002AB9A94A127812B9A44A322111800122EB
:1025D0000BE0A54A13784BB12B7803F0040303F00A
:1025E000FF011BB9A14B117001221A70DBF800909A
:1025F00000233B6009F17B0809F1CB0A98F8002021
:1026000098F8013018F8010C9A420BD241460CF0B0
:1026100023FB38B118F8022C012303FA02F23B68BD
:1026200013433B6008F10408D045E7D1904B1B7879
:1026300053B1904B904F1A68984612F0020FDFF892
:10264000509240F03A8332E309F1CA0709F58978DC
:102650003A787B7817F8010C9A4225D239460CF06B
:10266000FBFA08B397F804E00C21BB7801FB0E419C
:10267000824A013B03EB43031344D1F8C42097F88B
:1026800003909A4276480FD0C1F8C430002390F8E6
:10269000F020C1F8C830012303FA0EF322EA030345
:1026A00081F8C09080F8F03006374745D0D1744BA0
:1026B000DFF8E0A1D3F80080724B4FF0000B1B68ED
:1026C000029394F82B300393DAF80030002B00F0DB
:1026D000E58293F80090B9F1000F00F0DF82DAF89C
:1026E000042002998A1A002A0CDB01F5FA72CAF852
:1026F000042094F8F010012202FA0BF221EA0202FF
:1027000084F8F020039A002A00F0C8821AF8042CFA
:1027100059780432D2B2002940F081825A4931F905
:1027200012105A4AB2F8982102F1C800814201DD24
:102730009F7814E0C83A914202DA99784F420EE04D
:1027400094F8F020012303FA0BF322EA030384F840
:10275000F030029B03F5FA73CAF804309EE294F855
:10276000F03043FA0BF3DB0700F19882002FCCBF67
:10277000022001200CF072FB09F1FF32384B132AC2
:1027800000F28482DFE812F01400230032004400DB
:1027900061008800ED005201B701EC011B028202CA
:1027A000440055008800ED005201BF00240189015A
:1027B00098F8001040460F44FA2FA8BFFA2727EADE
:1027C000E77788F800700CF02DFA01201EE098F8E9
:1027D000011040460F44642FA8BF642727EAE7771B
:1027E00088F801700CF01EFA02200FE098F8031030
:1027F00040460F44642FA8BF642727EAE77788F88C
:102800000370D3F8F4100CF0C5F903203946D3E176
:1028100098F805100D2039446429A8BF642121EAE5
:10282000E17188F805100CF07BFAB9F10D0F00F09A
:102830002D8298F804100E2039446429A8BF642121
:1028400021EAE17188F80410B6E198F80610052035
:10285000394481F3080188F80610ADE1102D0020FD
:10286000540D0020362D0020372D0020382D00205B
:102870001E340020240F002024180020D4A20108B8
:10288000840F0020482F0020602F00202C100020F3
:10289000EC180020180E0020D3F8F8301A78022A1D
:1028A00022D13846049311F03FFAA94911F044FBB4
:1028B000049B596A059311F083F90021049011F0EB
:1028C00025FC059B48B9049AA249104611F03CFC2E
:1028D000049A059B10B19F4A00E000225A620F2023
:1028E00011460CF009FA0AE099780F203944C829FA
:1028F000A8BFC82121EAE17199700CF011FAB9F171
:102900000F0F00F0C381944BD3F8F89099F8003082
:10291000022B1AD1384611F007FA8D4911F00CFB41
:10292000D9F8201011F04CF90021074611F0EEFB08
:1029300030B93846874911F007FC10B1854F00E0E7
:102940000027C9F82070122059E199F801101220CF
:102950003944C829A8BFC82121EAE17189F80110CA
:102960002AE1D3F8F8301A78022A22D138460493A3
:1029700011F0DAF9774911F0DFFA049B196B05932E
:1029800011F01EF90021049011F0C0FB059B48B91D
:10299000049A7049104611F0D7FB049A059B10B1B8
:1029A0006C4A00E000221A63102011460CF0A4F9D2
:1029B0000AE0197B10203944C829A8BFC82121EAA0
:1029C000E17119730CF0ACF9B9F1100F00F05E81F0
:1029D000614BD3F8F89099F80030022B1AD13846A1
:1029E00011F0A2F95B4911F0A7FAD9F82C1011F0F7
:1029F000E7F80021074611F089FB30B93846554900
:102A000011F0A2FB10B1534F00E00027C9F82C7061
:102A10001320F4E099F80B1013203944C829A8BFFB
:102A2000C82121EAE17189F80B10C5E0D3F8F8302C
:102A30001A78022A22D13846049311F075F94749D1
:102A400011F07AFA049BD96B059311F0B9F80021C3
:102A5000049011F05BFB059B48B9049A3D49104670
:102A600011F072FB049A059B10B13A4A00E0002273
:102A7000DA63112011460CF03FF90AE0997D11202C
:102A80003944C829A8BFC82121EAE17199750CF021
:102A900047F9B9F1110F00F0F9802F4BD3F8F890F6
:102AA00099F80030022B1AD1384611F03DF92B4924
:102AB00011F042FAD9F8381011F082F800210746D7
:102AC00011F024FB30B93846224911F03DFB10B11A
:102AD000204F00E00027C9F8387014208FE099F8E3
:102AE000151014203944C829A8BFC82121EAE17172
:102AF00089F8151060E0D3F8F89099F80030022BAF
:102B00001AD1384611F010F9114911F015FAD9F817
:102B1000281011F055F80021074611F0F7FA30B9E6
:102B200038460C4911F010FB10B10A4F00E00027A5
:102B3000C9F82870092062E099F803100920394487
:102B4000C829A8BFC82121EAE17189F8031033E040
:102B5000000020410000C842540D002000007A44CB
:102B6000D3F8F89099F80030022B1AD1384611F0BA
:102B7000DBF8B44911F0E0F9D9F8341011F020F87D
:102B80000021074611F0C2FA30B93846AD4911F0BC
:102B9000DBFA10B1AB4F00E00027C9F834700A200F
:102BA0002DE099F80D100A203944C829A8BFC82182
:102BB00021EAE17189F80D100CF0B2F866E0D3F863
:102BC000F89099F80030022B1DD1384611F0ACF87E
:102BD0009D4911F0B1F9D9F8401010F0F1FF002132
:102BE000074611F093FA30B93846964911F0ACFA1D
:102BF00010B1944F00E00027C9F840700B2039460F
:102C00000CF07AF842E099F817100B203944C829E3
:102C1000A8BFC82121EAE17189F81710CCE7012982
:102C200034D19878894B33F91230B3F5617F05DBE5
:102C300040F633029342A8BF134601E04FF461739C
:102C4000B9F10C0F22D14FF4966292FBF0F0A3F58C
:102C5000617393FBF0F37E4ADFB21378BB4215D069
:102C6000042F34BF3B4602231370019A09FB032350
:102C7000784A03F2BA7313600DF055FE48463946A0
:102C80000CF04EF8781CC0B20CF0E8F894F8F02084
:102C9000012303FA0BF3134384F8F0300BF1010B1B
:102CA000BBF1040F0AF10C0A7FF40EADC1E43368E6
:102CB000D80510D5684BDB786BB13B6899070AD50E
:102CC000B9F8003013F0010A0AD110F02DFF0120ED
:102CD00005F0BCFB04E0012005F0A7FB012300E0A8
:102CE0000023D8F8002052070DD563B1012005F06C
:102CF0009CFBB9F800309B0708D410F015FF0220A8
:102D000005F0A4FB02E0022005F08FFBB9F80030CB
:102D1000524A13F0030F4FF0100114BF51611161BB
:102D20003A6812F00A0F27D0D8F80020D00609D54B
:102D300059070AD4042005F089FB494B1B88A4F8E5
:102D4000FC3002E0042005F070FBD8F800309A0651
:102D500007D5B9F800305B0606D4402005F076FBB5
:102D600002E0402005F061FBD8F80030580642BF71
:102D70003B4B1B88A4F8FE303B68990609D4D8F871
:102D800000301A0540F1B0804FF4807005F05EFB12
:102D9000AEE0344B1B789B076ED5334B1B78042B6E
:102DA0006AD9D8F8003013F4007A0FD0B9F800309F
:102DB000DF063AD4102005F049FB202005F035FB52
:102DC0002A48011D09F088FF02232AE0B9F80070A3
:102DD00007F01007BFB22FB1102005F026FB012726
:102DE00084F800A1D8F80030580512D5D4F8043181
:102DF0001F495A89B1F90030002BB8BF5B4293429A
:102E000007DAB1F90230002BB8BF5B429342C0F23F
:102E10000881B9F80030990608D5202005F005FB97
:102E2000002384F80031012700E0002794F80831DE
:102E30009BBB0E200BF0ECFF0E4B012283F8082108
:102E40002BE000BF0000C84200007A44602F002041
:102E5000DC2E0020840F00209C330020000C014059
:102E60001C100020281800202E1800208C0F002095
:102E700024100020540D0020B9F8003003F0300376
:102E8000002B3FF47CAF102005F0CFFA202005F096
:102E9000CCFA002384F8003102E0002F3FF46FAF3A
:102EA000002214466B4B002023F814006A4B191DB6
:102EB00003F10A0721F814000021D151174478606A
:102EC000B96023F8140003F132075A33D151D150BD
:102ED000174413447860B960586099601432002C2C
:102EE0007FF44DAF0124DDE74FF4807005F09DFACB
:102EF0005A4B5A791C46082A01D00E2A02D140208A
:102F000005F093FA33685A0540F1A18094F8203215
:102F10001BB92B7813F0040F03E0D8F8003013F43A
:102F2000002F0BD04E4B00221A703C200CF088FB77
:102F3000002800F08C800EF0DBFFF6E70FF000FFBA
:102F400009B0BDE8F04F06F09ABF012000E0022072
:102F50005FFA80F8019A08F1FF3382F8B83705F07C
:102F6000B7FA05F05BFB40460BF078FFFFF708BBB4
:102F7000BAF1000F02D07E2B3FF400AB94F8B930C9
:102F8000972B06D1374B4FF4C872A3F8BC20FFF73C
:102F9000F7BAA72B06D1344A137843F00403137011
:102FA000FFF7EEBA0022BB2B079201D1022303E008
:102FB000B72B04D14FF6FE73ADF81E3009E0BE2BDF
:102FC00001D1022303E0BD2B1AD14FF6FE73ADF8F9
:102FD0001C30DBF80030BDF81C10B3F858200A4450
:102FE000A3F85820BDF81E10B3F85A200A44A3F8DD
:102FF0005A2005F0E7FC002384F8BA30FFF7C0BA86
:10300000792B04D1194AD37823F0010306E07A2BF7
:103010007FF4B6AA154AD37843F00103D370FFF7C3
:10302000AFBAB9F800309B063FF500AF202005F09D
:103030000DFA0F4B0F481A685B68011D4360026070
:1030400009F04AFE074B012783F80071EEE609B04C
:10305000BDE8F08F143400205E0E00202C100020FC
:10306000DD2B0020540D00202818002014290020FA
:1030700030180020940F0020BA4B2DE9F04FB3F91F
:103080000610B94B89B01F6801937A8991420EDB13
:10309000B1F5FA6FFC79BFBF8B1A6343A2F5FA64EE
:1030A00093FBF4F4ACBFC4F16404643400E0642422
:1030B000AE4BAF4A1868B2F898A1054692F9622162
:1030C000049092B205920293002240F2E630A54BA2
:1030D0004FEA420B33F912300393CAEB030303F2B6
:1030E000F316864203D8002BB8BF5B4201E04FF4D1
:1030F000FA73022A049E4FF064002FD096F811E173
:10310000BEF1000F04D07345CCBFCEEB0303002308
:1031100093FBF0FCDFF8A0E26FF063093EF81C803F
:1031200009FB0C390CF1010C3EF91CE00FFA88FC8C
:10313000CCEB0E0E0EFB09FE9EFBF0FE8D4EC64440
:1031400026F80BE0BE18367973438B4E93FBF6F3EB
:1031500064339BB2634393FBF0F02DE096F812E1E9
:10316000BEF1000F04D07345CCBFCEEB03030023A8
:1031700093FBF0F0DFF82C826FF0630C0CFB00394E
:1031800038F910E0013038F91000002BCEEB0000C8
:1031900000FB09F999FBFCF90598CEEB090909FB3D
:1031A00000F97448B8BF5B42A0F80490B879434373
:1031B000714893FBF0F064306B784FF0640E43433A
:1031C00093FBFEF36D4E022AB354EB7A6C4E00FB78
:1031D00003F393FBFEF3B3546B7D664E00FB03F0E9
:1031E00090FBFEF0674B9854674B0FD183F802E0D9
:1031F000039B53450EDB5E4CB4F89A21914215DBDC
:10320000B1F5FA6FA8BF4FF4FA6110E09C54039B2C
:10321000534504DA36F80B305B4226F80B300132A6
:10322000032A05F101057FF450AFE4E71146891A3E
:103230004FF47A735943C2F5FA62B1FBF2F1642795
:1032400091FBF7F2DFF874E16FF063033EF81200D0
:1032500003FB021101323EF9122003B2D21A51438C
:1032600091FBF7F30344F380484B424D1B885A0609
:103270003BD5474A474B10881B88181A00B210F0FC
:1032800053FD454910F0A4FD074604F0FDFF8046BC
:10329000384604F086FF0746B5F9020010F044FDF9
:1032A0008146B5F9000010F03FFD4146824610F01E
:1032B0008FFD39468346484610F08AFD0146584640
:1032C00010F07CFC10F04AFF41462880484610F080
:1032D0007FFD39468046504610F07AFD0146404653
:1032E00010F06EFC10F03AFF68802C4F3B689B0793
:1032F00040F19F8045F20721294B2A4D1A686B69DE
:10330000D31A8B4240F395806A610CF025FE264B60
:10331000DFF8AC901A789846032AB9F8003051D1FA
:103320000A2B59D90023282088F800300BF033FDF0
:103330000CF012FE1D4B18880CF0F8FD1C4B1A689F
:10334000D37890FBF3F0013008281A4BA8BF08206F
:103350001870537980B243432B83137958436883A1
:103360003AE000BF602F0020840F00205C0F002097
:103370002C100020241000200CFEFFFF102700203E
:10338000EE0E0020242700205C290020EC180020ED
:10339000520E00201C10002035FA8E3C242F0020F5
:1033A00000340020E00E002074180020822C002041
:1033B00010180020540000200A2A0020F2290020C2
:1033C000141800200A2B07D803239C4A88F80030E1
:1033D000002313702B836B8398F80030984A012BDD
:1033E0000CD002D3022B1BD023E02A8BB9F800307B
:1033F0009A421EDD012388F800300FE0B9F8001072
:103400006B8B8B4202DD022313700FE08D4B1B8B05
:103410000133994202DD002313700AE0082006E020
:103420006B8BB9F8002001339A42E3DC07200BF0E4
:10343000EFFC3D682F0577D5834B824F1A68FB69F7
:10344000C3EB020845F2072398456DDD7F4BB6F9C3
:1034500006B0D3F800904FF47A7099F80A30FA6108
:10346000012B98FBF0F8B4F85211ABF57A7B784E4B
:1034700003D042D3022B20D041E0764B396A5A7BED
:10348000754B4FF0080E33F8122091FBFEF392B209
:10349000C91A8B183B6293FBFEF3BA8440F6E442F0
:1034A0009BB25343B9F80820C2EB13335843B9F920
:1034B000063090FBF3F0306021E0684BB9F808A0CB
:1034C0001B78C6F800A0580719D565480BF0F9FB22
:1034D00020B915F0100F18BF4FF0000B0BFB0BF3CA
:1034E000322293FBF2F3B9F906205B445A434FF4BE
:1034F0007A7392FBF3F3534400E0002333603368A4
:10350000D7E90A0103FB08F84FF47A7398FBF3F844
:1035100010EB080041EBE8710023C7E90A01514AAA
:1035200010F062FE504B1860504E3368D90427D516
:103530002A0622D54E4B1B789B071ED54D4B18787B
:1035400004281AD900224C4B0521D718951C4FF09E
:103550000A0E122AD154E9B287F801E004D0B0EB88
:10356000510F2A46EFD800E014215A18322002F8F1
:10357000010CFF225A540F2000E00A200BF048FCF7
:103580003E4D2A68002A51D03D4B3E4F186839689D
:10359000984681424AD83C4BDFF8F8901978526837
:1035A000E1B94FF0010A83F800A0B9F80030D35C0C
:1035B00023B350460BF00EFC344B83F800A010F000
:1035C00073F8B9F80030CBB92B681B78053B53452D
:1035D00014D80BF0B9FB2E4B18600FE04FF0000A27
:1035E00083F800A0B9F80030D35C3BB150460BF033
:1035F000F1FB264B83F800A010F056F82B68B9F8C1
:1036000000205B6823499B5CFE2B02D100230B80CA
:103610000CE0FF2B02D10BF0E3FB07E0D8F8000031
:103620000A2505FB030301323B600A800B4D2B7812
:103630005F0733D5184B08225A616DE05400002013
:1036400074180020E00E0020003400201018002024
:103650001C180020692C00207A2C0020193400202E
:10366000B6110020407E050020180020240F002005
:10367000281800202E180020FC2E0020282A0020C8
:10368000482F0020202A00201C2A0020C0330020C0
:1036900020320020242A0020000C01403268D0078C
:1036A0005CBF43F001032B70984B1B7819075EBF7A
:1036B0002B7823F001032B70D30248BF2B78944A58
:1036C00044BF23F001032B70924B1B6813F0040FCF
:1036D00002D09149098851B99049098809B19F07D9
:1036E00005D48F4B1B88003318BF012333B102234D
:1036F00013702B7823F001032B7004E02978CE0798
:1037000058BF022313700BF01FFB864B1B68C01AB7
:10371000002801DB0FF0C8FF0FF012FB824B1E7870
:103720000393002E00F0AA80804F3B68002B00F02E
:10373000358738680BF012FC002800F02F877B4B90
:103740007B4C18680BF007FC092801D03F2852D1A8
:103750004FF000094D462668DFF8F88136B175480C
:10376000D8F80010324614F0BFF810B9C14605B9B8
:103770004546714B08F110089845EFD3EDB1D5F8E7
:1037800000C0D9F8008023681CF803E018F8030093
:10379000704512D15A1C674958B92D2B09D8DFF84A
:1037A00090E1CEF800204FF0200E01F803E088549D
:1037B00003E001F803E02260E5E723680BB14D4523
:1037C00010D05E480EF08AFC4D4507D855F8100B16
:1037D0000EF084FC09200EF079FCF5E758480EF055
:1037E0007DFC002623689E42A3D2524B985D0EF0CA
:1037F0006DFC0136F6E72368002B40F0B486042800
:1038000040F0F0864B480AF059FB00F0C7BED8F8EC
:103810000000DFF83CA10BF0A1FB28B3DAF80000B0
:103820000BF099FBD9F80030834693F848209ABBF7
:10383000242840F09180012283F84820D9F80030F4
:10384000DFF808A193F848B0BBF1060FDFD193F879
:10385000490000F053FF002800F0A7800EF096FB0F
:103860003B68002283F84820364B93F83530002B14
:1038700040F067864C36982E00F09086324BF21856
:1038800092F84A100129F5D1304FF3583A60304A86
:10389000B94613609046BAE7012A04D14D2814BFF7
:1038A00000220222C8E7022A04D13C2814BF0022C9
:1038B0000322C1E7032A0AD140284FF000029FBF2C
:1038C0001A71DA715871987198BF0422B4E7042A0A
:1038D00008D19A7983F8490080EA020B83F806B090
:1038E0000522A9E7052AA9D159791A79914299792E
:1038F00006D941409971511C1971134418729DE702
:1039000081420CBF0622002296E700BF2818002043
:10391000C03300202418002010340020100E002096
:1039200012340020C43300201E340020F82E002062
:10393000502900202029002038AF010874C5010853
:1039400079C50108E00E0020841E0020CC1800205C
:10395000D018002058AD01082B78DA4A59073FF5F6
:103960006DAF2328DAF8003012D10492039A0121B6
:103970001170D549D5480B60D5490B630EF0AEFBED
:10398000D4480EF0ABFB049A137843F00203137093
:10399000D14B1B681B785B4501BFD04AD04B1A60E6
:1039A000D04A04BFD04BDA6048E7DAF8002092F83A
:1039B00049304C2B00F0A18400F29180352B00F0AF
:1039C0007C8239D82B2B00F0708420D8252B00F076
:1039D000478404D8232B00F0378200F0FFBD272B4B
:1039E00000F04584292B40F0F9850EF0ABFAA4F8DD
:1039F00082010EF0A7FAA4F884010EF099FA84F877
:103A000086010EF09FFAA4F8880100F095BD2F2BD7
:103A100000F0F48404D82D2B00F04B8400F0DEBDC0
:103A2000312B00F00085332B40F0D8850EF080FA62
:103A300084F8940100F080BD412B00F0998418D8DF
:103A4000392B00F0218404D8372B00F09E8400F03D
:103A5000C5BD3C2B00F0CD803E2B40F0BF850EF065
:103A600067FA84F8E2010EF063FA84F8E10100F0ED
:103A700063BD442B00F00B8526D8432B40F0AE8568
:103A80000EF056FA0023A36060710EF065FAA36889
:103A90001843A0600EF04CFA84F892010EF052FA2E
:103AA000A4F85C010EF04EFAA4F85E010EF04AFA9A
:103AB000A4F860010EF046FAA4F882010EF042FA72
:103AC000A4F8840100F038BD482B00F05E834A2B37
:103AD00040F084850EF036FAA08100F02DBDD12B88
:103AE00000F07D8320D8CC2B00F00E820FD8C82B9D
:103AF00062D004D84E2B00F00D8400F06FBDC92BAE
:103B000000F04683CA2B00F0838000F067BDCE2B07
:103B100000F02E83C0F02383CF2B00F04982D02BFE
:103B200000F0128300F05ABDD82B00F023810BD88F
:103B3000D32B3BD027D3D42B00F07E82D62B40F062
:103B40004D854FF000086CE2F22B00F0D58212D8C0
:103B5000EF2B40F04385DFF8A081D8F800900EF0FD
:103B6000F1F9A9F85A00D8F800800EF0EBF9A8F89E
:103B7000580000F0E1BCF32B00F0A884FA2B00F011
:103B8000008300F02BBD2B7803F0040303F0FF0843
:103B9000002B40F0D1840EF0CBF9022884F8B8074E
:103BA00040F2D882514B83F8B887D3E20EF0CAF9BD
:103BB0004F4B188000F0C0BC92F805804FEA5808BF
:103BC000B8F1120F03D906F0EBFE00F0B5BC4FF0D0
:103BD0000009C14507D20EF0B5F9464B23F819008C
:103BE00009F10109F5E73A4B012283F8342000F08E
:103BF000A3BCDFF80481D8F800900EF099F989F899
:103C00000000D8F8003018780BF06CFC00F094BC81
:103C1000394B1A6898461278022A40F08E804FF08D
:103C20000008DFF8D49008F1080BD9F800A00EF0D6
:103C30007FF910F075F8314910F07EF94AF82B0041
:103C4000D9F800A00EF074F908F10A030AEB830A10
:103C500010F066F82A4910F06FF9CAF80400D9F894
:103C600000A00EF065F910F05BF8264910F064F939
:103C700008F10E0B08F10108B8F1030F4AF82B0008
:103C8000CFD1B8F1070FD9F800A03DD10EF050F90F
:103C900010F046F8194910F04FF9CAF84400D9F865
:103CA00000A00EF045F910F03BF8144910F044F96B
:103CB000CAF84800D9F800A00EF03AF98AF84C008A
:103CC00035E000BF19340020F82E0020A9C50108F6
:103CD000E00E002079C50108E02B0020EFBEADDE2C
:103CE000F04F00200400FA0500ED00E02C10002049
:103CF000500E0020602F00205C0F002000002041AB
:103D00000000C84200007A440EF012F9C2448AF85A
:103D10000100D9F800A00EF00BF9C2448AF80B009C
:103D2000D9F800A00EF004F9C2448AF8150008F191
:103D30000108B8F10A0FA4D1FEE34FF00009D8F84A
:103D400000A00EF0F5F8CA448AF80100D8F800A0E7
:103D50000EF0EEF8CA448AF80B00D8F800A00EF076
:103D6000E7F8CA4409F10109B9F10A0F8AF8150008
:103D7000E5D1E1E38046DFF8749308F1080BD9F848
:103D800000A00EF0DFF80FF0CBFFD24910F0D4F80E
:103D90004AF82B00D9F800A00EF0D4F808F10A0375
:103DA0000AEB830A0FF0BCFFCA4910F0C5F8CAF845
:103DB0000400D9F800A00EF0C5F80FF0B1FFC54916
:103DC00010F0BAF808F10E0B08F10108B8F1030F72
:103DD0004AF82B00CFD1B8F1070FD9F800A01AD1BB
:103DE0000EF0B0F80FF09CFFBA4910F0A5F8CAF831
:103DF0004400D9F800A00EF0A5F80FF091FFB549E6
:103E000010F09AF8CAF84800D9F800A00EF09AF815
:103E10008AF84C0012E00EF095F8C2448AF80100CE
:103E2000D9F800A00EF08EF8C2448AF80B00D9F839
:103E300000A00EF087F8C2448AF8150008F10108C6
:103E4000B8F10A0FC7D177E30EF072F81328824653
:103E50003FF6B9AEDFF89492D9F800800EF068F81A
:103E600000239D490C2202FB0312117A814220D1CA
:103E7000137808EB8A0888F879300EF059F888F83A
:103E80007A000EF055F888F87B000EF051F8934A4E
:103E9000934B88F87C001A60D9F80000914B002100
:103EA000186079300AF0FCFE8F4B80F0010018702A
:103EB00042E301331C2BD4D185E60EF039F80B28F0
:103EC00080463FF680AE894BD3F800900EF030F874
:103ED00003283FF678AE0BFB089B8BF8CE000EF064
:103EE00027F88BF8C9000EF023F88BF8CA000EF003
:103EF0001FF88BF8CB000EF01BF88BF8CC000EF0FF
:103F000017F88BF8CD0017E35379092B7FF65BAEDA
:103F1000019BD3F800800EF00BF8019B88F800009D
:103F2000D3F800800EF004F888F801000EF000F8D5
:103F3000019B64281B68A8BF642018710DF0F8FF6E
:103F4000019B64281B68A8BF642058710DF0F0FF26
:103F5000019BFF281B68A8BFFF2098710DF0E8FFA8
:103F6000019B6428D3F8008028BF642088F80700EC
:103F70000DF0DEFF019B88F80200D3F800800DF001
:103F8000D7FF019B88F80300D3F800800DF0DAFF1B
:103F9000DAF80030A8F80A005B790A2B40F2CC82EC
:103FA000534BD3F800800DF0C3FF88F80800C3E23C
:103FB0000DF0C8FF6FF4AF6283189BB2C62B98BF99
:103FC000A4F898010DF0BEFFA4F844010DF0BAFF6B
:103FD000A4F846010DF0B6FFA4F848010DF0B2FFB9
:103FE000A4F8DA010DF0A4FF84F8EF010DF0A0FFB2
:103FF0000DF09EFF84F8F0010DF09AFF84F8870120
:104000000DF096FF84F894010DF092FF374BD3F832
:1040100000800DF097FF00EB80004000A8F85600EC
:1040200032E10DF08FFF334B23F8180008F101083F
:10403000B8F1080FF5D17FE253790F2B7FF4C3ADB0
:104040000DF076FF072880463FF6BDAD029BD3F802
:1040500000900DF077FF0E2303FB08F8029BC1448C
:10406000A9F81901D3F800900DF06CFFC144029B30
:10407000A9F81B01D3F800900DF064FFC144029B26
:10408000A9F81D01D3F800900DF052FFC144029B26
:1040900089F81F01D3F800900DF04AFFC144029B3C
:1040A00089F82001D3F800900DF042FFC144029B33
:1040B00089F82101D3F800900DF03AFFC144029B2A
:1040C00089F82201D3F800900DF046FFC844C8F8E3
:1040D000230131E200007A4440A30108701100205E
:1040E000480E00204C0E0020140000205C0F002021
:1040F000840F0020DE2E00200DF01AFF0F288046CE
:104100003FF661AD0DF014FFC8EBC808A04488F875
:10411000D4000DF00DFF88F8D5000DF009FF88F8E8
:10412000D6000DF005FF88F8D7000DF001FF88F8E4
:10413000D8000DF0FDFE88F8D9000DF0F9FE88F8E2
:10414000DA000BF0CDF8F7E12B785B0700F1F48192
:104150000CF02EFC04F0BCF904F060FAECE12B78D2
:10416000580700F1E981CC4B4FF4C8721A80E3E1A3
:104170002B78590700F1E081C84A137843F0040313
:104180002BE02B785A07E5D528E208F0DBFFD3E1D6
:104190000DF0CEFEC14B1A7810B142F0020201E0E0
:1041A00022F002021A700DF0C3FEBD4BDFF814833B
:1041B00018700DF0D1FEC8F800000DF0CDFEC8F863
:1041C00004000DF0BFFEB74B18800DF0BBFEB64BE0
:1041D000B64A1880137843F002031370ACE10DF077
:1041E000A7FE83460DF0B8FE82460DF0B5FE81466F
:1041F0000DF0B2FE80460DF0A5FE0DF0A3FE0DF011
:1042000097FEBBF1000F14D1A94B1020C3F800A0FA
:10421000C3F8049004F009F9A04A137843F00103AD
:104220001370B8F1000F00F08781A24BC3F8008033
:1042300082E1BBF1100F40F07F819F4BC3F800A0DB
:10424000C3F80490B8F1000F02D09A4BC3F8008075
:1042500099489A4B0222011D1A7008F03DFD6BE14E
:10426000A0600DF079FEA3681843A06064E10DF032
:1042700069FEA4F85C010DF065FEA4F85E010DF086
:1042800061FEA4F8600157E10DF052FE84F87C0154
:104290000DF04EFE84F880010DF04AFE84F87F0197
:1042A0000DF046FE84F8810146E10DF041FE60719B
:1042B00042E10DF03DFE84F892010DF043FEA4F8BA
:1042C0009C010DF03FFEA4F898010DF03BFEA4F810
:1042D0009A010DF02DFE3B6884F893015B79DFF8BD
:1042E000E881082B40F228810DF02CFEA8F89E01F1
:1042F0000DF028FEA8F8A0011EE10DF019FE84F8CB
:10430000D8010DF015FE84F8D9010DF01BFEA4F8BC
:10431000DA0111E192F805800323B8FBF3F8B8F154
:10432000120F3FF650ACDFF8A0914FF0000AC245E3
:1043300080F002810DF0FCFD89F8A2010DF002FE73
:1043400040F2ED23984205DD40F6CA039842A8BF2B
:10435000184601E040F2EE20A0F2EE20192390FB77
:10436000F3F00AF1010A89F8A30109F10209DEE775
:1043700080460DF0DDFD04EB080308F10108B8F1FB
:10438000080F83F88A01F4D1D6E053794FF007097A
:10439000B3FBF9F9C9EBC9029B1A13F0FF0F7FF4C5
:1043A00012AC5FFA89F909F1FF395FFA89F9B9F1BD
:1043B000FF0F00F0C1800DF0BBFD5FFA80FA4FFAED
:1043C0008AF00AF0A5FB804600283FF4FCAB80F899
:1043D00000A00DF0B7FDA8F802000DF0A9FD88F8C7
:1043E00004000DF0A5FD88F805000DF0A1FD88F88A
:1043F00007000DF09DFD88F80600D4E7DFF8C880BF
:1044000008F140090DF09EFDA8F8B0020DF090FDF6
:1044100088F8B2020DF08CFD08F1040888F8AF02AC
:10442000C845EFD188E00DF083FD1F2880463FF698
:10443000CAAB3B685B79082B7FF4C5AB0DF082FDFE
:1044400008F18C0804EB880900F03F00A9F802008D
:104450000DF078FDB9F80230800100F4FE501843E9
:10446000A9F802000DF064FD000104F828000DF029
:104470005FFD14F8283000F00F00184304F82800FE
:104480000DF056FD89F801000BF076FE54E00C4B60
:10449000012283F835204FE0100E0020281800205C
:1044A0002E1800202C1800202A1800208A0F002027
:1044B0008C0F00209C0F0020940F0020540E002031
:1044C000E00E0020301800202C1000200DF030FDF0
:1044D000FF2881461BD100238DF81F309DF81F3027
:1044E000052B29D89DF81F00704A9DF81F30012127
:1044F00002EBC3035B6852F83000994089B248224E
:1045000003F016FA9DF81F300133DBB2E4E705280B
:104510003FF659AB00200DF05DFD0DF037FDD8F8EA
:1045200000000AF012FD18B932200AF034FCF6E758
:104530004FFA89F003F00AFA00200DF04BFDFFF767
:104540008DB95B4B98590AF000FD18B932200AF07A
:1045500022FCF6E70AF084FE03F090FF554A564B22
:10456000DA60FFF787B90C283ED00A2845D1534DB1
:1045700053480DF0B3FD2846232113F09EF908B1EE
:10458000401B20602368002B5AD14C480021302268
:10459000236013F05CF9039B1B7843BB494B1B68FA
:1045A0009B0614D5484B49491B688A6B9A1A002A06
:1045B0000DDB474A1278042A09D903F5123303F5B3
:1045C000F873444A8B63D36883F01003D360424B83
:1045D0009B68002B67D04148984764E006F0E0F9FB
:1045E000FFF73CB90C2804D13D480DF077FD3D485C
:1045F0000DE07F2812D1FFF79CB80D28B7D07F2897
:1046000009D12E4A013B002137482360D1540DF0D7
:1046100065FDFFF78EB82F2B3FF68BA8A0F1200287
:10462000D2B25E2A3FF685A813B920283FF481A8AC
:104630005A1C2260214AD0540DF048FDFFF779B88A
:104640005A1EA95C202901D113469CE71B4A002170
:104650002360D154254B264DD3F80090D5F800A007
:10466000DFF85880504613F036F906465146324678
:10467000404613F039F91F4A28B918F806304B4460
:104680005B78580703D010359542E7D306E0954292
:1046900004D2701CEB684044984702E016480DF0C5
:1046A0001DFD002371E709B0BDE8F08FDCC80108EB
:1046B000841E00200400FA0500ED00E020290020FF
:1046C000C3D401082418002000340020E00E00208C
:1046D0002E180020000C0140341F00201C0F002069
:1046E0007EC5010879C50108A5C50108680000203C
:1046F00058AD010838AF010889C501082DE9F04718
:104700004B28A0B0044600F0408600F2B480302868
:1047100000F0CA8651D8222800F08C8423D80328C0
:1047200000F0608114D8012800F05081022840F088
:10473000268704200DF04EFC43200DF016FC4C2083
:104740000DF013FC46200DF010FC4C2000F051BE83
:10475000042800F05181052840F011871A200DF03F
:1047600039FC00245BE1282800F0DD8515D82428D9
:1047700000F0C485262840F00287B54C06200DF0D5
:1047800029FCB4F85C010DF028FCB4F85E010DF0D2
:1047900024FCB4F8600100F0AEBD2C2800F0D685F2
:1047A0002E2800F051862A2840F0E98601200DF0DD
:1047B00011FCA74B587900F01CBE3D2800F01C836B
:1047C0001ED8362800F026860BD8322800F00B863B
:1047D000342840F0D48648200DF0FCFB002500F082
:1047E0004BBC3A2800F0BA823B2800F01C843828E1
:1047F00040F0C58604200DF0EDFB954C00F084BD23
:10480000452800F0A98627D8402800F0F5854228E1
:1048100040F0B5868E4C10200DF0DCFB60790DF079
:10482000A4FBA0680DF0E2FB94F892010DF09DFB53
:10483000B4F85C010DF0D1FBB4F85E010DF0CDFBD6
:10484000B4F860010DF0C9FBB4F882010DF0C5FBAE
:10485000B4F8840100F04FBD472800F05B86C0F03B
:104860004886492840F08B8602200DF0B3FB784B38
:10487000988900F040BD702800F0F18258D869286E
:1048800000F04C822AD8652800F0FE8015D84D280B
:1048900000F08A85642840F0728607200DF09AFBAC
:1048A000E7200DF062FB6A4B58790DF05EFB0020AB
:1048B0000DF05BFB042000F05EBE672800F0B181C4
:1048C00000F21F8212200DF085FB624B00241B8832
:1048D000B3F5806F8CBF0825012584E16C2800F0BA
:1048E000308217D86A2800F08D846B2840F0478604
:1048F00005200DF06FFB584B18880DF06EFB574BE1
:1049000018880DF06AFB564B93F86A0000F001001E
:1049100000F06FBD6E28524D00F0278200F27782C2
:1049200006200DF057FBA86D0DF060FB4D4B13E218
:10493000782800F0838119D8742800F0BE830BD842
:10494000722800F01F84732840F0198608200DF0AB
:1049500041FB012400F04FBC762800F0738400F284
:10496000F1832F200DF036FB3F4C54E3A42800F0D8
:104970008E8414D87B2800F0F482A02840F0FF85B4
:104980000C200DF027FB394B18680DF02FFB384B2E
:1049900018680DF02BFB374B186800F0ECBDF128C0
:1049A00000F08881FE2800F09984F02840F0E78527
:1049B0002B4C04200DF00EFBE36BB3F85A000DF006
:1049C0000CFBE36BB3F8580000F095BC03200DF02E
:1049D00001FB00200DF0C9FA20460DF0C6FA0D20AB
:1049E00000F007BD0DF0F6FA01200DF0BEFA0A2026
:1049F0000DF0BBFA00F049BC06200DF0EBFA4120A7
:104A00000DF0B3FA46200DF0B0FA4E200DF0ADFADD
:104A100041200DF0AAFA184B187800F06CBC174B27
:104A2000185D01340DF0A1FA0B2CF8D10024144BC1
:104A3000185D01340DF099FA082CF8D10024114BBF
:104A4000185D01340DF091FA072CF8D100F095BDF6
:104A50002C10002028000020A2180020A4180020FC
:104A6000200F0020141000200FA30108E8F7FF1FFB
:104A7000ECF7FF1FF0F7FF1F1B340020C4C1010833
:104A8000D0C10108A5C10108CA4C0B200DF0A2FA43
:104A900020880DF0A2FA608880B20DF09EFAC64B15
:104AA0001B68C3F3C000C3F38002800040EA4200E9
:104AB000C3F340021043C3F3401240EAC20003F0C4
:104AC000100318430DF089FABC4B1A88636802F092
:104AD000080103F4475949EA010903F4804149EA0E
:104AE000010903F4004149EA010903F4803149EA6C
:104AF000010903F4003149EA010903F4802149EA7C
:104B0000010903F4002149EA010903F4801149EA8B
:104B1000010903F0007349EA0303DFF8D89212F0A9
:104B2000010F99F8009018BF4FF00208C9F38009EF
:104B300008BF4FF0000843EA090312F0020F43EAEE
:104B4000080314BF4FF0040C4FF0000C12F0040FD8
:104B500043EA0C0C14BF4FF0100E4FF0000E12F091
:104B6000400F14BF202700274CEA0E0E12F0100F42
:104B700014BF4FF4007600264EEA070712F0200F0C
:104B800014BF4FF4806500253E4312F4807F14BFAC
:104B90004FF400600020354312F4007F14BF4FF43F
:104BA00000110021284312F4806F41EA000114BF74
:104BB0004FF080630023002019430346247AA34268
:104BC0000AD27F4A9D5C012202FA05F50D421CBF04
:104BD0009A4010430133F2E70DF008FA794B93F84D
:104BE000B80700F006BC784B33F91400013490FB91
:104BF000F5F080B20DF0F1F9032CF4D16D4CA08CDE
:104C00000DF0EBF9E08C0DF0E8F9208D6F4C0DF014
:104C1000E4F920880DF0E1F960880DF0DEF9A08854
:104C200069E310200DF0D6F90024694B185D0134BA
:104C30000DF09BF9102CF8D100F09FBC70200DF006
:104C4000C9F900260E2474435A4D0136EB6B2344F8
:104C5000B3F819010DF0C1F9EB6B2344B3F81B0154
:104C60000DF0BBF9EB6B2344B3F81D010DF0B5F962
:104C7000EB6B234493F81F010DF077F9EB6B2344A2
:104C800093F820010DF071F9EB6B234493F82101A7
:104C90000DF06BF9EB6B234493F822010DF065F9ED
:104CA000EB6B1C44D4F823010DF0A0F9082EC9D1F8
:104CB00000F063BC70200DF08DF9424C04F17005DA
:104CC00094F8D4000DF051F994F8D5000DF04DF999
:104CD00094F8D6000DF049F994F8D7000DF045F995
:104CE00094F8D8000DF041F994F8D9000DF03DF991
:104CF000073494F8D3000DF038F9AC42E0D100F05D
:104D00003CBC10200DF066F90024324B185D0134D4
:104D10000DF02BF9102CF8D100F02FBC2E4D0024F3
:104D20002878400000F0FE000DF054F92B789C42EA
:104D300080F02384294B33F814000DF04EF9013430
:104D4000F4E7274C06200DF045F920880DF045F9D1
:104D500060880DF042F9234B1888CCE204200DF056
:104D600039F9144BD86D00F006BC07200DF032F96C
:104D70001D4B1888FF28A8BFFF20C0B20DF0F5F822
:104D80001A4B186880F3100080B20DF026F9B5F8C0
:104D900060000DF022F90B4B93F88721144B186833
:104DA00022B10A23584380F3100001E000F30F0002
:104DB00080B2A0E2200F002024180020EC18002070
:104DC000290F00202C1000200E100020502C002055
:104DD0004A0F0020600F0020201F0020602F0020BD
:104DE0001C2F00201C100020141800202018002068
:104DF0001C18002019340020BF4C02200DF0EAF8E6
:104E000094F8E2010DF0B1F894F8E101F1E20B2021
:104E10000DF0E0F86B6E002618780DF0A6F86B6EBA
:104E200058780DF0A2F86B6EB44C33441879013603
:104E30000DF09BF8032EF6D1636ED8790DF095F83E
:104E4000636E98780DF091F8636ED8780DF08DF858
:104E5000636E58890DF0C1F8636E187AC9E2A74CE9
:104E60001E200DF0B7F8E36B00251B78022B65D1EF
:104E7000E36B05F1080253F82200A1490EF0A8FFE8
:104E800012F0F2FE80F30800C0B20DF06EF8E36B92
:104E90009C4903EB8503D86A0EF09AFF12F0E4FEFA
:104EA00080F30800C0B20DF060F8E36B05F10E026C
:104EB00053F8220094490EF08BFF12F0D5FE80F3D8
:104EC0000800C0B201350DF050F8032DD0D1072DE8
:104ED000E36B21D1586C8A490EF07AFF12F0C4FEC0
:104EE00080F30800C0B20DF040F8E36B8449986C81
:104EF0000EF06EFF12F0B8FE80F30800C0B20DF0A5
:104F000034F8E36B93F84C000EF00AFF12F0ACFE9D
:104F100080F30800C0B20BE02B4458780DF025F860
:104F2000E36B2B44D87A0DF020F8E36B2B44587DCB
:104F300001350DF01AF80A2DC9D11EE3E36B2B449D
:104F400058780DF012F8E36B2B44D87A0DF00DF879
:104F5000E36B2B44587D01350DF007F80A2DEDD198
:104F60000BE33C200DF036F80024644D04F10802F8
:104F7000EB6B654953F822000EF02AFF12F074FE25
:104F800080B20DF02AF8EB6B5F4903EB8403D86A1B
:104F90000EF01EFF12F068FE80B20DF01EF8EB6BF3
:104FA00004F10E0253F8220057490EF011FF12F0DF
:104FB0005BFE013480B20DF010F8032CD5D1072C24
:104FC000EB6B16D1586C50490EF002FF12F04CFEFC
:104FD00080B20DF002F8EB6B4B49986C0EF0F8FEC6
:104FE00012F042FE80B20CF0F8FFEB6B93F84C002D
:104FF0000BE0234458780CF0F0FFEB6B2344D87A95
:105000000CF0EBFFEB6B2344587D01340CF0E5FF13
:105010000A2CD4D1B1E214F8010F002800F0AD82BF
:105020000CF0A3FFF7E701200CF0D4FF334BDB6B50
:105030001878DEE150200CF0CDFF00252F4B0C211D
:10504000DC6B324B04EB850494F87920013501FBCD
:10505000023393F838000CF088FF94F87A000CF0D3
:1050600084FF94F87B000CF080FF94F87C000CF037
:105070007CFF142DE2D180E2204BDC6B062303FB86
:10508000054494F8CE000CF070FF94F8C9000CF0C1
:105090006CFF94F8CA000CF068FF94F8CB000CF099
:1050A00064FF94F8CC000CF060FF013594F8CD005B
:1050B0000CF05BFF0C2DDFD15FE24FF00008012602
:1050C00000270E4B1A7A974233DA0933FA5C002430
:1050D0000C2363430D4D05F13001595C914207D11A
:1050E0002B44586B12F0F7FB82468EB9B14611E0A3
:1050F00001341C2CECD11AE02C100020200F0020D1
:10510000000020410000C84200007A4410A30108BA
:1051100080440CE0D1450ADA0C2303FB04535B6B9B
:1051200013F809000CF021FF09F10109F2E701373A
:10513000C7E7002E00F021825FFA88F00CF04AFFEA
:105140000026BDE7CB4D0024287A0CF043FF2B7AD4
:105150009C4280F01282C84B0021E65C0C2202FBCC
:1051600001F3C64800F13007DA5DB24205D10344CD
:1051700093F838000CF0F9FE02E001311C29EDD162
:105180000134E4E7BE4C16200CF024FFB4F898017B
:105190000CF023FFB4F844010CF01FFFB4F84601F3
:1051A0000CF01BFFB4F848010CF017FFB4F8DA015B
:1051B0000CF013FF94F8EF010CF0D7FE00200CF078
:1051C000D4FE94F8F0010CF0D0FE94F887010CF0B6
:1051D000CCFE94F894010CF0C8FE00200CF0C5FE43
:1051E000A44B0A20DB6BB3F9563093FBF0F080B28E
:1051F0000CF0F3FE88E0E0B201340CF0B6FE092CAE
:10520000F9D1BAE110200CF0E5FE9E4B9E4C1878C7
:1052100000F002000CF0A9FE9C4B18780CF0A5FEE3
:1052200020680CF0E3FE60680CF0E0FE984B1888F4
:105230000CF0D3FE974B18880CF0CFFE8D4BB3F8D3
:10524000680058E00CF074FE074612200CF0C2FE15
:10525000884C17B9E66E256F05E0102F19BF0025A1
:105260002E46666FA56F38460CF07FFE30460CF078
:10527000BDFE28460CF0BAFEE06F0CF0B7FE002031
:105280000CF0ABFE00200CF0A8FE0020B1E0794D40
:10529000002495F880002E4680000130C0B20CF04A
:1052A00099FE95F880000CF060FE96F880309C42E4
:1052B00080F06381784D285D0CF057FE05F11003F6
:1052C000185D0CF052FE05F12003185D30350CF02E
:1052D0004CFE285D0CF049FE0134E6E708200CF096
:1052E00079FE00200CF079FE00200CF076FE002004
:1052F0000CF073FE00200CF070FE3EE104200CF078
:1053000069FE5F4B986836E194F87C010CF02DFE45
:1053100094F880010CF029FE94F87F010CF025FE32
:1053200094F8810165E0564C07200CF053FEB4F868
:1053300082010CF052FEB4F884010CF04EFE94F899
:1053400086010CF012FEB4F88801D4E74C4C0C2016
:105350000CF040FE94F892010CF007FEB4F89C01AA
:105360000CF03BFEB4F898010CF037FEB4F89A014B
:105370000CF033FE94F893010CF0F7FDB4F89E01A5
:105380000CF02BFEB4F8A001B5E73D4C04200CF066
:1053900021FE94F8D8010CF0E8FD94F8D9010CF046
:1053A000E4FDB4F8DA01A6E73C4C3D4D2078002638
:1053B00000EB4000C0B20CF00DFE237802359E4297
:1053C00080F0DB8015F8020C0CF0CFFD15F8010C15
:1053D000013600EB800000EB800000F2EE2080B28E
:1053E0000CF0FBFDE9E701200CF0F4FD244B93F8F1
:1053F00094010CF0BAFDC0E008200CF0EBFD002495
:105400001F4B234493F88A0101340CF0AEFD082CA5
:10541000F6D1B2E0174B1A4C93F8C10004F12805FD
:10542000C0EBC000C0B20CF0D5FD94F8F60100232B
:105430001C4AD25C904200F0A4800C333C2BF7D184
:105440000834AC42F1D198E040200CF0C3FD0C4C84
:1054500004F14005B4F8B0020CF0BFFD94F8B202BC
:105460000CF083FD043494F8AF020CF07EFDAC42E6
:10547000F0D182E0200F0020290F002010A30108A6
:105480002C10002028180020301800202E18002092
:105490002C1800202A180020A10F0020201F002017
:1054A000CE110020E42B0020E0200CF093FD424CB4
:1054B00004F18005B4F83202043400F03F000CF02F
:1054C0008CFDB4F82E02C0F386100CF086FD94F823
:1054D0002C0200090CF049FD94F82C0200F00F009A
:1054E0000CF043FD94F82D020CF03FFDAC42E1D1ED
:1054F00043E0324C0D200CF06DFD08F02BF90CF060
:1055000034FD20880CF072FDE0680CF06FFD07F0B0
:1055100021FD30E00CF020FD054684200CF05AFD02
:1055200028460CF063FD254BDC6805F18003A3429F
:105530008CBF641B802407F0C7FD284622466946BD
:1055400008F03CF905460024AC4216DA1DF80400C8
:105550000CF00BFD0134F7E713200CF03BFD0024A9
:10556000174B185D01340CF000FD0B2CF8D1002016
:105570000CF03CFD00200CF039FD012018E000206B
:1055800016E00CF0F2FCB4F8F8010CF026FD94F8EB
:10559000FA010CF0EAFC94F8FB010CF0E6FC94F83C
:1055A000FD010CF0E2FC94F8FC010CF0DEFC47E796
:1055B00020B0BDE8F08700BF2C10002018000020AC
:1055C000C4C101086B4B6C4A2DE9F04F5E89146829
:1055D0004FEA062AB4EB0A0A9C884FF000054FEA0E
:1055E00004481C894FF0000BA4FB0A6765EB0B0B0A
:1055F00004FB0B77F40944EA476418EB04065C8863
:105600004FF000094FEAE7154FEAC438DC8849EB50
:10561000050787B0CDE90467A4FB0A6704FB0B7795
:10562000340A44EA076418EB04064FEA27259C89EC
:105630004FF0000949EB0507CDE90067AAFB0467B5
:1056400004FB0B77F40D44EA472414F5FA664FEA9D
:10565000E75545F10007B6F5FA6F77F10003CDE99C
:105660000267964666DADDE90489A4FB046704FB59
:1056700005F34FF0050C07EB4307A6FB0C230CFBCF
:1056800007335F104FEA3206B8EB06084FEA92067E
:1056900046EA837669EB07099F10DDE90023921B38
:1056A00063EB0703CDE90023DDE90267334A4FF0DE
:1056B000FF33964277EB0303CDE9048927DA40F6FE
:1056C000AC520023A4185D4104FB05F3A4FB044580
:1056D0006FF0060205EB4305664202FB0566A4FB7C
:1056E0000223334418EB020649EB0307CDE90467B4
:1056F0000B26A4FB062306FB0533DDE900455B1002
:105700004FEA3202A41A65EB0305CDE90045DDE955
:1057100002450AFB0BF3AAFB0AAB0BEB430B4FEA68
:10572000DA7242EA4B02A41A4FEAEB7365EB030507
:10573000CDE90245DEF80440009B019DA4FB032354
:1057400004FB05334FEA525848EAC3284FEA63592D
:10575000DDE90423B8EB020269EB03039946D30B9E
:1057600043EA494300B1036009B1029B0B6007B0F3
:10577000BDE8F08F541F0020E40F002024FAFFFF43
:105780002DE9F04FDFF8589285B00746D9F80800A8
:105790000E460EF0C9FA8E4C804620880EF0C0FAF4
:1057A0004FF05C51054640460EF012FB4FF064513D
:1057B000824628460EF00CFB014650460EF0FEF9DC
:1057C0004FF06251824640460EF002FB4FF06A51A4
:1057D000804628460EF0FCFA014640460EF0EEF9EF
:1057E0000546B4F902000EF09FFA014628460EF075
:1057F000EFFA5146054650460EF0EAFA8046B4F9F3
:1058000004000EF091FA014640460EF0E1FA01461E
:1058100028460EF0D5F980460EF0A0FC6D490546ED
:10582000A06140460EF088FBD9F80C30804628462F
:1058300001930EF079FA4FF07C510EF0C9FA6649E7
:105840000EF0BCF90546E389B4F90A0002930EF0A4
:105850006BFA29460EF0BCFA29460EF0B9FA4FF061
:1058600058510EF0B5FA8146B4F90800B4F810B0FA
:10587000B4F80CA00EF058FA29460EF0A9FA014629
:1058800048460EF09DF94FF058510EF0A1FA4FF036
:1058900060510EF09DFA4FF07E510EF091F9814665
:1058A000E0880EF03DFA014648460EF091FA0021DC
:1058B00081460EF021FC00287BD1294628460EF0B7
:1058C00087FA03900FFA8BF00EF02EFA039B014635
:1058D00018460EF07DFA4FF060510EF079FA8346CB
:1058E000BDF908000EF020FA014628460EF070FAC5
:1058F00001460EF065F9014658460EF061F94FF089
:105900007A510EF065FA834601980EF00DFA0146C1
:105910004FF093400EF052F905460FFA8AF00EF060
:1059200003FA4FF08F410EF053FA014658460EF03D
:1059300047F94FF066510EF04BFA014628460EF03B
:105940003DF926490EF044FA49460EF0F5FA0546AF
:10595000B4F916000EF0E8F929460EF039FA294696
:105960000EF036FA4FF040510EF032FA8146B4F99B
:1059700014000EF0D9F9014628460EF029FA4FF02E
:1059800060510EF025FA014648460EF019F981469D
:10599000B4F912000EF0C8F9014648460EF010F9AD
:1059A0004FF076510EF014FA014628460EF008F931
:1059B00000E0002017B10EF0D1FB38602EB1404658
:1059C0000EF0CCFB64235843306005B0BDE8F08F87
:1059D000B41F00200000A04500007A470050C345D6
:1059E000E40F0020704770472DE9F041324C334DF1
:1059F00062892B8AB4F904809A1A2389B4F902E0E7
:105A00005A43B4F91230D613B4F91420DB023244ED
:105A100093FBF2F232440A26E2615643A2F57A621F
:105A200002FB02F3B4F90EC002FB0EFE02FB08F209
:105A3000B4F90C801B130CFB03FC03FB08F31B14D1
:105A400003EB62320232E388921002F500425343C4
:105A50004CF25032B4F920704FEAEE2EB4F9004007
:105A60000EEBEC2C0CEB8404BC406D690234A5EB0E
:105A7000A4043A4162434FEAD3384EBFB2FBF8F375
:105A80005400B4FBF8F340F6DE3448BF5B001A1252
:105A9000524362430A4C08365C43241404EB22420E
:105AA00002F6CF62361103EB221300B1036001B19D
:105AB0000E60BDE8F08100BF681F0020E40F0020E9
:105AC00043E3FFFF024B4FF480521A80704700BF40
:105AD00028000020044A137E23B101230370002311
:105AE0001376704703707047E40F00207720482139
:105AF00001220BF0DFBC7720582101220BF0DABC29
:105B00007620F42131220BF0D5BC074B002193F80D
:105B10002020064B9201343259767720F42102F08E
:105B2000FC020BF0C7BC00BF681F0020E40F002080
:105B3000034B00225A767720F4212E220BF0BABCB8
:105B4000E40F002008B50F21082218200BF0B2FC4A
:105B50000E22182010210BF0ADFC024B4FF48052A6
:105B60001A8008BD2800002008B5134B53201B786D
:105B70002D2108227BB10BF09DFC31210A225320FC
:105B80000BF098FC2C210C2253200BF093FC53209B
:105B90003821902209E00BF08DFC31210A2253209C
:105BA0000BF088FC53202C210A220BF083FC40F2DE
:105BB0000912024B1A8008BD501F00202800002047
:105BC00007B5002101AB032277200BF033FC9DF8D1
:105BD00005309DF804001B0243EA00439DF80600CF
:105BE000184303B05DF804FB08B5FFF7E9FF014B6C
:105BF000586008BDE40F002008B5FFF7E1FF014B36
:105C0000186008BDE40F002007B5F7216B46062297
:105C100076200BF00FFC9DF800309DF801101B035F
:105C200043EA01139DF80210094A43EA1113D360B5
:105C30009DF803309DF804101B0343EA01139DF8FF
:105C4000051043EA1113936003B05DF804FB00BF35
:105C5000E40F00200F4B13B51B780F4C0BB1637E84
:105C6000B3B1032201AB7720F6210BF0E3FB9DF8E3
:105C700005309DF804201B0243EA02439DF80620EC
:105C80001343064AB2F92020C2F10802D3406361EF
:105C900002B010BD33000020E40F0020681F002078
:105CA0000A4B13B51B780A4C0BB1637E63B1022219
:105CB00001AB7720F6210BF0BDFB9DF804209DF889
:105CC000053043EA0223238202B010BD33000020D6
:105CD000E40F002013B506220446432168206B46DA
:105CE0000BF0A8FBA8B19DF800209DF80130012021
:105CF00043EA022323809DF802209DF8033043EA03
:105D0000022363809DF804209DF8053043EA0223B6
:105D1000A38002B010BD13B5062204463B216820C3
:105D20006B460BF087FBA8B19DF800209DF8013071
:105D3000012043EA022323809DF802209DF80330CE
:105D400043EA022363809DF804209DF8053043EA6E
:105D50000223A38002B010BD13B501220DF1070389
:105D600004461A2168200BF065FB9DF8073003B14B
:105D70000123237002B010BD13B5022204461B217B
:105D8000682001AB0BF056FB70B19DF804209DF824
:105D9000053043EA022303F54E5310334FF48C725F
:105DA00093FBF2F32333238002B010BD13B5062218
:105DB00004461D2168206B460BF03CFBA0B19DF80A
:105DC00000209DF8013043EA022323809DF8022041
:105DD0009DF8033043EA022363809DF804209DF878
:105DE000053043EA0223A38002B010BD13B506229A
:105DF000044601211C206B460BF01CFB08B39DF8E8
:105E000001309DF80020042143EA022242F38D0272
:105E100092FBF1F29DF8023022809DF8032042EAC5
:105E2000032242F38D0292FBF1F29DF8043062806E
:105E30009DF8052042EA032343F38D0393FBF1F31E
:105E4000A38002B010BD13B506220446022118201B
:105E50006B460BF0EFFAB8B19DF800309DF80120C9
:105E60009B0803EB022323809DF802309DF803205A
:105E70009B0803EB022363809DF804309DF8052006
:105E80009B0803EB0223A38002B010BD314B2DE928
:105E9000F3411B780546002B3BD0002426462746BD
:105EA000A04601345320322108226B46E4B20BF0A5
:105EB000C1FA08B9002049E09DF801209DF80030A2
:105EC000202C03EB02231BB29DF8032098449DF87D
:105ED000023003EB02231BB21F449DF805209DF8FE
:105EE000043003EB02231BB21E449DF8073003F07D
:105EF0007F0301D0002BD4D198FBF4F897FBF4F783
:105F000096FBF4F6144BA5F800806F80AE809C766B
:105F10001CE05320322106226B460BF08BFA00283E
:105F2000C8D09DF801209DF8003003EB02232B80A0
:105F30009DF803209DF8023003EB02236B809DF84F
:105F400005209DF8043003EB0223AB8002B0BDE8CE
:105F5000F08100BF501F0020E40F002008B54FF46F
:105F6000804009F0D3FD012801BF044B4FF480426B
:105F70005A61034B08BF587608BD00BF00040140BA
:105F8000E40F002010B5074C2368186909F0BEFD26
:105F900030B123681A69044B5A61044B01221A7606
:105FA00010BD00BF4C1F002000040140E40F002082
:105FB00013B500222A211C200BF07CFA0E210222AC
:105FC0001C200BF077FA0F2103221C200BF072FA31
:105FD0002B2112221C200BF06DFA164A0224936921
:105FE000154843F0040393612023ADF804300423E3
:105FF0000DEB03018DF806308DF8074007F071FABC
:1060000022462C211C200BF055FA2D2101221C20A8
:106010000BF050FA2E2100221C200BF04BFA2A2103
:1060200005221C200BF046FA044B4FF480721A80B4
:1060300002B010BD001002400008014028000020FE
:10604000F8B50F461646074C4FF48055656140F091
:1060500080000CF06DFA3846002132460CF032FA1E
:106060002561F8BD000C014013B501220DF10701B7
:1060700004463820FFF7E4FF052008F081FE9DF874
:10608000073003B10123237002B010BD13B50446DD
:10609000694643200622FFF7D3FF9DF800209DF8B4
:1060A0000130012043EA022323809DF802209DF85D
:1060B000033043EA022363809DF804209DF80530F5
:1060C00043EA0223A38002B010BD13B5044669461B
:1060D0003B200622FFF7B4FF9DF800209DF8013019
:1060E000012043EA022323809DF802209DF803301B
:1060F00043EA022363809DF804209DF8053043EABB
:106100000223A38002B010BD70B50E46054C4FF4BB
:10611000805565610CF00CFA30460CF009FA2561E7
:1061200070BD00BF000C01401D4B07B51A681D4B28
:106130009A420ED14FF40053ADF8043002238DF88B
:106140000730042318480DEB03018DF8063007F0E3
:10615000C8F980216B20FFF7D7FF642008F01BFEF1
:1061600000216B20FFF7D0FF642008F014FE6B20A5
:106170000121FFF7C9FF1B201821FFF7C5FF1C20D5
:106180001021FFF7C1FF094B1A201978FFF7BCFF58
:1061900019200021FFF7B8FF03B05DF804FB00BF32
:1061A00044000020001BB700001001403200002016
:1061B000F0B5254D85B0EB7E002B43D1234C2368F1
:1061C000002B3FD01A68224E12B1B1690A43B26166
:1061D0009A889868ADF8002002228DF8032069465D
:1061E00004228DF8022007F07CF9B369002743F000
:1061F0000103B36123680126197D187B07F05CF960
:10620000144808F08DFE2368134A1B6953610293FA
:1062100008230DEB03008DF80D308DF80C708DF810
:106220000E6009F043FC236801A85B7D8DF80670C1
:106230008DF8043003238DF805308DF807600CF0DD
:1062400023F9EE7605B0F0BDE40F00204C1F0020CE
:1062500000100240855F00080004014008B5FFF708
:10626000A7FF6B21802268200BF024F9642008F03E
:1062700092FD6B21032268200BF01CF90F2008F01F
:106280008AFD124B19211A7868200BF013F90F20A0
:1062900008F081FD0E4B1A211A7868200BF00AF9DC
:1062A0001B21182268200BF005F91C211022682000
:1062B0000BF000F93721002268200BF0FBF8BDE855
:1062C00008406820382101220BF0F4B8D01F0020CC
:1062D0003000002008B5FFF76BFF074B1B7813B1A8
:1062E000012B03D008BD4FF4006201E04FF480524F
:1062F000024B1A8008BD00BF511F0020280000205B
:1063000008B5192008F047FD6820152100220BF080
:10631000D1F810B9022008F0B9FD0C4B16211A78FB
:10632000682042F018020BF0C5F8172100226820FF
:106330000BF0C0F83D21012268200BF0BBF8BDE84E
:10634000084068203E2101220BF0B4B83100002043
:106350000AF0FCBE0BF022B80AF0F8BE0BF01EB833
:1063600073B51D4C237F53BB1C4A1D4D93694FF4DD
:10637000805643F00803936110238DF806302846B9
:10638000032301A98DF80730ADF8046007F0A9F8E0
:10639000144A2E61138823F040031B041B0C138046
:1063A000138823F038031B041B0C43F008031380ED
:1063B00013889BB243F04003138001232377752099
:1063C00001A90122FFF73CFE9DF80400A0F1700333
:1063D0005842584102B070BDE40F00200010024046
:1063E000000C01400038004007B5232008F0D3FC22
:1063F0006820752101220DF107030BF01BF828B16D
:106400009DF80700A0F168035842584103B05DF8B9
:1064100004FB00BF2DE9FF47CB4C07462378CB4E4A
:10642000002B00F0E78132686368D31A7C2B40F2BE
:10643000E181237A6260013323724FF0000808F192
:106440002400C14DC0B20CF02FFC05F10A0333F952
:1064500018000DF069FCBE4B814618880DF064FCF5
:10646000014648460DF068FDBA490DF0B1FC0DF04B
:1064700075FE08F1010800B20CF004FCB8F1030F3E
:10648000DDD130200CF010FCB5F910000CF0FAFB57
:106490000CF002FC2B7A9A072CD141F288336A68FF
:1064A0009A4218D910200CF0FFFB68694FF064087D
:1064B00090FBF8F000B20CF0E5FB21200CF0F4FBAF
:1064C000686990FBF8F308FB13000028B8BF40424E
:1064D00000B20CF0D7FB14200CF0E6FBB4F9180066
:1064E0000CF0D0FB1C200CF0DFFB00200CF0CAFBF2
:1064F0000CF0D2FB237ADFF850825B0740F0578123
:1065000002200CF0D1FBD8F81C006423323090FB41
:10651000F3F000B20CF0B6FBB8F926504FF0050AC4
:1065200095FBFAF503200CF0BFFB8B4BADB21B784B
:10653000DFF8389213F0040F0DD008F5D970394602
:1065400008F0BFFB28B9D9F8003013F0100F18BFBE
:10655000002528B205E0D8F80C389889B0FBFAF08D
:1065600000B20CF08FFBD9F800309F076ED5DFF832
:106570000092B4F8102899F800304FF0640808FB36
:1065800002325B00B2FBF3F3B4F8127806203F014D
:10659000BFB247EA0327BFB2C3F303231F430CF084
:1065A00083FB38B20CF06EFBB4F8123899F8001087
:1065B00001339BB293FBF1F201FB1233A4F81238C2
:1065C000D4F81438604D9B7B012B05D139200CF099
:1065D0006BFBB5F910081AE0B5F810586E235D434F
:1065E000152795FBF7F53A20AFB20CF05DFBB7FB32
:1065F000F8F528B208FB15750CF044FB3B200CF0B5
:1066000053FBA8B2451D0A2095FBF0F000B20CF038
:1066100039FB28200CF048FBD4F818380A2093FBEB
:10662000F0F000B20CF02EFB04200CF03DFBD4F88F
:106630000C389B8913B109F053FC04E0424BD3F8AA
:106640001C0880F3100000B20CF01CFBD4F82038BA
:106650003D4F9D0640F1A08097F8243898071DD53E
:1066600011200CF021FBB7F826084FF4F3656843BE
:106670003A4B90FBF3F000B20CF004FB19200CF045
:1066800013FBB7F826084543642095FBF0F595FB0E
:10669000F0F300FB135000B20CF0F4FA94F8243835
:1066A000B4F8285813F0020F08BF002501200CF0A1
:1066B000FBFA28B20CF0E6FA09200CF0F5FA0020FB
:1066C0000CF0E0FA264B94F82A581A88B2F5967F17
:1066D0000AD91D4B1B7A03F00F03072B04D842F293
:1066E0000F75954228BF154605200CF0DDFAD4F849
:1066F00014385B7B0BB928B216E0A5F120000DF031
:1067000013FB18490DF018FC002105460DF0FEFCA6
:1067100010B94FF07C5101E04FF03F4128460DF099
:106720004FFA0DF01BFD00B20CF0ACFA94F82428DF
:10673000054B910703D493F82B28012A1AD1012382
:1067400084F82B3808482EE004100020482F002041
:106750002800002000007A4419340020A08601009F
:10676000560000206666E63F30180020242F0020E7
:1067700054000020D3F81458C04968680DF028FB75
:106780000DF0ECFCBD490290A8680DF021FB0DF066
:10679000E5FC039002A806E0B94A02AB92E80300C8
:1067A00083E8030018460CF08FFA0CF075FA237A90
:1067B000282B1FD1B34B00221A7233684FF47A7022
:1067C000B3FBF0F83C2717200CF06EFAB8FBF7F596
:1067D000B5FBF7F007FB1050000200B20CF052FAC4
:1067E00018200CF061FA07FB158000B20CF04AFA91
:1067F0000CF052FA94F83438A24D002B00F061816D
:1068000008F0A2FAD5F838389F4AC31A93420746CF
:1068100040F2C780002385F83E3885F84038B5F847
:106820001038DAB21B0A85F85A2885F85B3885F8E3
:10683000502885F85138D5F8682833689A1AD5F861
:106840006C38D97B4FF47A734B439A420ED38F4BFB
:106850001B68C5F8683895F87038013B012B9FBF5D
:10686000102385F83E38022385F84038D4F81828DC
:106870000A20D4F81C3892FBF0F293FBF0F384F872
:106880005828121284F8592884F85C3894F824287F
:106890001B1284F85D3894F82A389207794984F8F5
:1068A0008B3803D42D2381F88C3878E0D4F82C98D9
:1068B0007748DFF8E8C199FBF0FA0CFB0A924FF039
:1068C000060E042B0EFB02F28CBF3323322381F819
:1068D0008C38704BD4F8306892FBF3F196FBF0F0F3
:1068E00003FB1122642592FBF5F20CFB006C0EFBFE
:1068F0000CFE84F87D28121284F87E289EFBF3F2A9
:1069000003FB12E393FBF5F30AEB8A0A4FFA81F8D3
:106910000AEB8A0A08EB8A0189B284F87B1800EB3B
:106920008000090A84F87C1800EB800051B201EB6A
:10693000800292B284F88028120A84F8812884F8B0
:106940008238B4F826281B1284F883382423534352
:1069500093FBF5F5B4F89E380A2284F884381B0AB4
:1069600084F88538B4F828384FEAD979B3FBF2F3C4
:1069700003F5FA739BB284F886381B0A84F88738CB
:10698000B4F8A038F60F84F87858C5F3072584F8D2
:106990007A9884F87F6884F8795884F88D38C4F838
:1069A000387894F8A288374DB8F1000F0DD1D5F89A
:1069B000A80808F0D3FA012807D90228364E00F0BB
:1069C0005C820CF051F90123B370D4F8AC282D4D42
:1069D000002A76D095F8A2683EB140F6B731D5F8D6
:1069E000B438FB1A8B4219D86BE00123D5F8A808FC
:1069F00085F8A23801F07EF8D5F8B838082193F967
:106A0000000002238DE8480032464FF4964301F01F
:106A100085F885F8BC68C5F8A80850E095F8B06816
:106A2000CEB9D5F8A808C5F8AC6885F8A26801F019
:106A300061F8D5F8B838082193F9000001238DE8F2
:106A4000480032464FF4964301F068F8C5F8A808AC
:106A50000CF00AF933E0013EF6B285F8B06895F81B
:106A6000BC1895F8BD38DEB94A1C013385F8BC283E
:106A700085F8BD38D5F8A8081FE000BF8096184BF0
:106A80009CA40108041000203F0D0300482F0020A3
:106A90008096980040420F0028000020806967FF20
:106AA00012F8016B01337018314685F8BC08D5F82F
:106AB000A808C5F8AC2885F8BD3808F052FAC4F823
:106AC000B47894F8BE38A04DDBB1D5F8C038C3B166
:106AD000D5F8C438ABB1C5F8C8381B689B4AC5F8AF
:106AE000CC38D5F8D0381344187AFDF707FE0BF0F0
:106AF0004DFAD5F8D0380133092B88BF0023C5F8EB
:106B0000D038934D94F8D4282E688F4B002A00F08B
:106B1000EF81D3F8D828002A00F0EA8193F8DC3816
:106B2000013B012B00F2E481D4F8D808864F08F02D
:106B300015FAE0B1D7F8D80808F00DFA97F8DD3863
:106B400080467E2BD5F800900ED102231B2887F8B3
:106B5000DC3809D1D7F8D80808F000FA20B90123A9
:106B6000C7F8E09887F8E43884F8DD88DCE7D7F8E0
:106B7000E0282B689B1A41F6583293421ED9032312
:106B800087F8DC38B4E1734A32F8130010B90346D1
:106B90004FF403600133B0F5C06FDBB279D01ED97A
:106BA000B0F5006F7FD032D9B0F5036F3FD184F8D4
:106BB000E538D4F82038644F99063FD494F8E418A7
:106BC00094F8E538002900F055812A68921B012AC3
:106BD000D9D984F8E538002384F8E43888E1B0F5A1
:106BE000007F43D007D8B0F5807F49D0B0F5887FCB
:106BF00000F08B80E6E7B0F5806F00F0AF80B0F575
:106C0000826F00F0F480B0F5047FDBD123E0B0F5B3
:106C1000E26F00F08B80B0F5E46F00F08C80B0F58F
:106C2000E06FCFD184F8E538B4F90A1087E0B0F509
:106C3000046F74D0B0F5026FC4D104E197F8243822
:106C40009A07BBD5B7F8261824234B436421123387
:106C500093FBF1F108E184F8E5383F4B3A4F1B68AC
:106C60009B07ABD5B7F810380A21FCE084F8E5386B
:106C7000394B354F1B681905A0D5D7F81818F3E024
:106C800084F8E538D4F820382F4F5A0796D579691B
:106C9000EAE084F8E538304B2B4F1B681B058DD597
:106CA000D7F81C18E0E0D4F82018274A8F0684F89B
:106CB000E53883D592F8241888077FF57FAFD90788
:106CC00011D5D2F83038192283EAE371A1EBE371D0
:106CD00001EB5101B1FBF2F1002BACBF41F00041DF
:106CE00041F040410EE0D2F82C38192283EAE371DA
:106CF000A1EBE37101EB5101B1FBF2F1002BB8BF45
:106D000041F080414FF400608CE084F8E538D4F81D
:106D100020380D4F5B077FF551AF3969A4E084F847
:106D2000E538B4F91830642159437BE084F8E5383C
:106D3000B4F90C1003E0B4F90E1084F8E5382C23F4
:106D400091FBF3F16EE000BF041000209CA4010849
:106D5000482F0020C6C60108242F002084F8E538FB
:106D600094F8E638644A0133DBB2032B88BF012371
:106D700082F8E63842F2107394F8E61859435F4BF4
:106D80001B78D80748BF01319A0748BF02315F0717
:106D9000B4F8E83848BF0431D80748BF0A319A0729
:106DA00048BF14311F0648BF2831D80548BF2831D5
:106DB0005A0748BF64311F0748BFC831980548BF0C
:106DC00001F5C8719A0648BF01F57A71DF0648BF20
:106DD00001F5FA61580648BF01F57A614FF4806009
:106DE0000BF00EFF444B002283F8E428E6E6D4F8CB
:106DF0002018DFF8048111F0200784F8E53817D057
:106E000098F8242812F0020F14BF4FF47A71002171
:106E100012F0010F14BF4FF4FA6300230B4494F8EF
:106E20002A1819440BF0ECFE002384F8E438C5E678
:106E3000334B1B6819067FF5C1AE39460BF0E0FEF7
:106E400088F8E478BAE684F8E538D4F820382A4F90
:106E50009A067FF5B3AE97F824389B077FF5AEAE60
:106E6000B7F82838642159430BF0CAFE002387F88D
:106E7000E438A3E684F8E5383AE0B37823B1C5F8FE
:106E8000A47886F80280A0E5D5F8A438FB1AB3F5FB
:106E90007A6FFFF49AAD0123D5F8A808B37008F013
:106EA0005AF80646D5F8A80808F055F876067FF493
:106EB0008CAD8A2802D08E280DD086E5D5F82038F2
:106EC00098067FF582AD95F8A238002B7FF47DAD52
:106ED00005F6710306E095F8A238002B7FF475AD36
:106EE00005F63C03C5F8AC382D2385F8B0386CE5C1
:106EF00004B0BDE8F08700BF041000201934002062
:106F0000242F0020F8B504460E46174600252046DB
:106F1000202110F0D2FC0446D0B10134204610F0FC
:106F20002FFDB0F5617F05DB40F634039842A8BF22
:106F3000184601E04FF46170A0F56170192390FBD1
:106F4000F3F00DB9307000E070703B7801333B70A6
:106F50000DB90125DBE72046F8BD30B505460C46E6
:106F6000134629462246BDE83040014801F0EAB800
:106F7000B8C701087FB504780646E4B9354B192136
:106F8000186800EB840090F87B5090F879204D430E
:106F900005F5617590F87A30009590F87C004143D2
:106FA00001F5617101912C482146013401F0CAF8C4
:106FB000142CE3D14BE010F0E3FC1328054641DC30
:106FC000244B701C1C68202100238DF80F3010F01A
:106FD00074FC1E35064670B10136304610F0D0FC08
:106FE0001A289FBF04EB850358709DF80F300133BA
:106FF00098BF8DF80F303046202110F05EFC064619
:1070000070B10136304610F0BBFC0D289FBF04EB79
:10701000850398709DF80F30013398BF8DF80F30BD
:1070200004EB85043046E11C0DF10F02FFF76AFF07
:107030009DF80F30042B0AD0601C0021042210F0B0
:1070400006FC04E0054800211322FFF786FF04B088
:1070500070BD00BF5C0F0020D7C70108ECC7010856
:1070600001480BF03BB800BFF2C701082DE9F0431F
:1070700004788FB00546002C59D17B4B0021142297
:1070800009A807AED3F8008010F0E1FB07223046D4
:10709000002110F0DCFB00231A46A70005A8059389
:1070A00008EB070583807149B5F802E031F813C099
:1070B0001CEA0E0F0AD00E310DF1380C595C02F1AA
:1070C000010E624402F81C1C5FFA8EF20133072B9A
:1070D000E9D100210B46664AB5F802E011F802C07A
:1070E0001CEA0E0F0AD006320DF1380C8A5C03F14F
:1070F000010E634403F8242C5FFA8EF30131062954
:10710000E9D118F807308DE841006A7859490292B0
:1071100009A81A0903F00F0300F0FFFF21465648A3
:1071200009AA013401F00EF8202CA6D198E010F045
:1071300027FC1F28044600F3868028462021E4B25D
:1071400010F0BBFB1F2C02D9FFF78AFF88E0464BEB
:10715000451C1B68002103EB84042046042210F028
:1071600076FB0027454B09AE304600210A2217F86E
:1071700003905FFA87F810F06AFB002315F8012BE3
:1071800032B10A2B04D04A4502D0F2540133F5E75C
:107190004A455ED108F1FF33032B09D8DFE803F03D
:1071A0001005023F0DF1230134E00DF123011EE033
:1071B000304610F0E5FB2378C0B243EA001006E049
:1071C000304610F0DDFB237800F00F0018432070EC
:1071D00031E00133062B0AD0244800F11B069E5DE6
:1071E0009642F6D103445A7D63881343638011F8B5
:1071F000012F02B30023EFE70133072B0AD01B480E
:1072000000F10E069E5D9642F6D130F81320638899
:107210001343638011F8012F6AB10023EFE7304672
:1072200010F0AEFB0F2804DC304610F0A9FB6070B4
:1072300001E0002363700137052F93D1012408F08A
:107240009BFF6CB980E70E4800211F22FFF785FEE7
:1072500006E020460021042210F0F9FA0024EEE7AF
:107260000FB0BDE8F08300BFF0180020B0A4010803
:10727000C5A4010800C801080FC80108D1A401086D
:10728000ECC70108F8B50478064674B9304D2146BC
:10729000B5F8C621B5F8C8312E48013400F052FFC8
:1072A000042C05F10405F2D1F8BD2B4910F0D8FAF1
:1072B000A8B9274B4FF47A714FF4FA62A3F8C611BC
:1072C000A3F8C821A3F8CA11A3F8CC21A3F8CE11C2
:1072D000A3F8D021A3F8D211A3F8D421F8BD3046E9
:1072E00010F04EFB032805462BD83046202110F025
:1072F000E4FA044630B10134204610F041FB012687
:10730000074600E006462046202110F0D6FA10B9C4
:10731000BDE8F840A4E6013010F032FB012EF7D1B1
:1073200040F2DC53A7F2EE229A42F1D8A0F2EE220C
:107330009A42EDD8064B703503EB8503DF80188148
:10734000F8BD064800210322BDE8F84005E600BF6D
:107350002C1000201BC801082EC801080BD60108FC
:107360002DE9FF4104780546002C34D16D480AF020
:10737000B5FE6D4D686900210CF0BEFE002840F09E
:10738000CE802146694800F0DDFE6869694600F05C
:107390005FFD0146664800F0D5FEA869694600F029
:1073A00057FD0146624800F0CDFEE869694600F0ED
:1073B0004FFD01465E4800F0C5FE286A694600F0B0
:1073C00047FD013401465B4800F0BCFE0C2C05F182
:1073D0001005CFD1A3E05849052210F085FA38B93D
:1073E000514B002203441030C0285A61F8D196E076
:1073F00028465249042210F077FA04462846002C09
:107400003FD1202110F059FA002800F08880451C57
:10741000284610F060FA0746494B53F824601EB91D
:1074200048480AF05BFE7AE028463146FAB210F08E
:107430005BFA01340028EFD13B4B0021C218103019
:10744000C02851619E46F7D13F4B03EBC402D2F8EE
:1074500004C09846BCF1000F04D131463B4800F00F
:1074600071FE53E0002718F834309F42F5DA3B01F3
:107470000EEB0305143563440FCB013785E80F008D
:10748000F1E710F07DFA0B28064643DC2846202160
:1074900010F013FA054648B10135284600F042FCC9
:1074A000214B012403EB0613586100E004462846F3
:1074B000202110F002FA054640B10135284600F0BF
:1074C00031FC194B013403EB061398612846202147
:1074D00010F0F3F9054640B10135284600F022FCD2
:1074E000114B013403EB0613D8612846202110F01C
:1074F000E4F910B9FFF7B4FD11E0013000F012FC1F
:10750000094B032C03EB06163062F3D11048FFF74A
:1075100027FF04E00F4801210C22FFF71EFD04B0F5
:10752000BDE8F08134C801082C1000204FC80108C4
:1075300055C8010867D301082EC8010859C80108B9
:1075400038AF01085EC80108E8C601086DC8010827
:10755000A8C50108ECC70108F0B5047887B0064655
:1075600014BB514B19201968062303FB041191F831
:10757000CA5091F8CE20454305F5617591F8C930A0
:10758000009591F8CB50C831684300F561700190C7
:10759000087902904979454803912146013400F069
:1075A000D1FD0C2CDDD17CE010F0EAF90B2804466B
:1075B00072DC3D4B701C1D68202100238DF81730B4
:1075C00010F07BF9064680B10136304610F0D8F94C
:1075D00003289FBF062303FB045383F8CE009DF8C6
:1075E00017309CBF01338DF817303046202110F042
:1075F00064F9074680B10137384610F0C1F90D280B
:107600009FBF062303FB045383F8C9009DF817307E
:107610009CBF01338DF8173006266643A9193846FA
:10762000CA310DF11702FFF76DFC202110F045F96A
:10763000074670B10137384610F0A2F914289FBFF1
:107640009DF817307619013386F8CC0098BF8DF875
:1076500017303846202110F030F978B1013010F0A1
:107660008FF90D289FBF062303FB045383F8CD0039
:107670009DF817309CBF01338DF817309DF81730F7
:10768000062B0ED0062202FB04500021C93010F058
:10769000DEF8FFF7E5FC04E0054800210B22FFF7C8
:1076A0005CFC07B0F0BD00BF5C0F002079C801088A
:1076B000ECC70108F0B5027887B08AB94A4C04F1EA
:1076C000280694F8F6210023484950B259568142C1
:1076D0006DD00C333C2BF7D10834B442F1D180E0AB
:1076E000002204920592451C10F04AF9C4B260B21F
:1076F00007F00EFA074618B18DF81040012400E09B
:1077000004462846202110F0D8F8054638B1013546
:10771000284610F035F90134ADF81200E4B2002625
:107720002846202110F0C9F8B0B3451C284610F0B7
:1077300027F900222E495FFA82FE51F82230834257
:1077400004D00132082AF5D1002300E0734651F835
:107750002320824220D1022E0FD0032E12D05A1E97
:10776000012ED2B204D0042A13D88DF814300EE0C2
:10777000042A0ED88DF8153009E0052B09D88DF8AC
:10778000173004E09A1E052A03D88DF8163001340C
:10779000E4B20136042EC3D1052C03D807B0BDE8EE
:1077A000F0405DE404AB03CB3860796019E094F8F5
:1077B000FB010F4B94F8FA5153F82000B4F8F8216C
:1077C000009094F8FD0153F82000019094F8FC011A
:1077D00053F8200053F825300290064800F0B2FC20
:1077E0007AE707B0F0BD00BF2C100020E42B00208A
:1077F000D0A9010899C801082DE9F3470478074684
:107800004CB9204601A90BF0F3F80134FFF7F4FF5F
:10781000122CF6D17FE010F0B3F8C5B2112D75D857
:107820003E4C05F1D00604EB4603781C202193F86A
:10783000028010F042F83A4F034630B9A8F1020234
:10784000D2F1000848EB020848E007F1260800F1F1
:10785000010A5978404610F030F868B1032D8CBF0A
:1078600003230023C8EB0000C0B23B44184490F847
:107870002A90B9F1030F02D1FFF7F2FB4BE0A9F117
:107880000203D3F1000850464FF0200148EB0308F3
:1078900010F013F8D8B1B8F1000FEDD0013010F0AE
:1078A0006FF840F2ED2380B2984205DD40F6CA033E
:1078B0009842A8BF184601E040F2EE20A0F2EE2068
:1078C000192290FBF2F004EB4603D87002E0B8F105
:1078D000000FD1D104EB460383F8029004EB460479
:1078E000A3781F4497F82620B8F1000F09D0E1785B
:1078F00019234B430B48294603F2EE2300F022FCE8
:1079000009E02946084800F01DFC04E00748002172
:107910001122FFF722FB02B0BDE8F0872C100020F7
:10792000B0A40108B8C80108CAC801080BD60108EC
:1079300007B50123ADF8041001A98DF806208DF8D4
:10794000073005F0CEFD03B05DF804FB2DE9F047EC
:10795000814672B6514C4FF400774FF480616161FB
:10796000204667614822FFF7E3FF39462046102290
:10797000FFF7DEFF1FFA89F6494A4FEAC60802EB15
:107980000803596852F83650464B4FEAD10E05EBC2
:107990008E00586055F82E0001F0070198608900AC
:1079A000D8600F208840C043D3F80CC052F839A0EB
:1079B00000EA0C0CC3F80CC0D3F808C002EBC909EC
:1079C00000EA0C009860D8684FF0080C0CFA01FC33
:1079D0004CEA0000D860D3F808C0012000FA01F199
:1079E00041EA0C019960996845F82E10D9F8041005
:1079F000994600FA01F5CAF8105027611746A368A6
:107A00005805FCD4D9F80830D9F8042008211360AF
:107A10004FF40073CAF814506361234B19611021AD
:107A2000596140F60553A16849051AD4013BFAD1C2
:107A3000D9F80C3057F83600136007EB080252688B
:107A4000C168012393400B43C3604FF40071134896
:107A50001822FFF76DFF62B6BDE8F047322007F04D
:107A60009AB94822CAF810505046A9B2FFF760FFF1
:107A70000D4B10221A61A268084B5205C2D5DAF8E4
:107A800008204FF400701542074A4FF0080115BF57
:107A90001861586111615161EDE700BF00080140B4
:107AA000DCC80108F0180020000C014010B50446A5
:107AB000204607F04AFA18B90A2007F06CF9F7E7F0
:107AC00010BD30B5094900220B78094C1557854285
:107AD00002BFFF25155503F1FF3302F10C0208BF69
:107AE000DBB23C2AF1D10B7030BD00BFE10F0020AA
:107AF000E42B0020002208490C2303FB02135968E1
:107B0000814204D10022C2621A725A607047013267
:107B1000052AF0D1704700BFE42B00202DE9F74380
:107B2000064689469DF8288011461A469DF82C3055
:107B300000250C2068431D4FC419C057B04202D124
:107B4000207A20B12BE00135052DF2D127E0022E5D
:107B50000FD005DC56B1012E21D1009314480AE064
:107B60001E2E0DD01F2E1AD1012009E000931148BE
:107B700001E011480093434603F014F9044605E080
:107B800001F0F0FE4146044607F0DCF94CB10C234D
:107B900003FB0575267185F808906C6001E00020F4
:107BA00000E0204603B0BDE8F08300BFE42B0020D6
:107BB000004400400038014000480040F0B5012476
:107BC000B0FBF4F58D4201D34C43F9E70026D4B164
:107BD000B0FBF4F504FB1500B4FBF1F41EB9002D65
:107BE00001DC002CF3D1092D03F1010EEFB204DD0D
:107BF000002A14BF3725572500E030253D441D706D
:107C000001367346E3E71C70F0BDF0B50124B0FB0C
:107C1000F4F58D4201D34C43F9E70026D4B1B0FB13
:107C2000F4F504FB1500B4FBF1F41EB9002D01DCE2
:107C3000002CF3D1092D03F1010EEFB204DD002A6F
:107C400014BF3725572500E030253D441D7001360F
:107C50007346E3E71C70F0BD03685A1C026019709C
:107C600070472DE9F843089E002B074688461446C6
:107C7000334614BF4FF030094FF0200913F8012BA1
:107C80000AB9254603E0002CFBDD013CF6E7002D98
:107C900004DD38464946C047013DF8E7354624EA49
:107CA000E474A01B284415F8011B11B13846C047E5
:107CB000F7E7BDE8F883024B186807F052B900BF38
:107CC000100F0020F8B507460C46486800211546FD
:107CD0001E460CF011FA58B128460CF025F8104950
:107CE0000CF076F801464FF07E500CF025F96060FC
:107CF000616830460BF064FF014630460CF01CF919
:107D000025680646294638460BF058FF014630469E
:107D10000CF05EF8014628460BF052FF2060F8BDDB
:107D2000DB0FC9402DE9F04102780346202A00F11B
:107D30000100F9D0092AF7D02D2A02D10346414D7E
:107D400004E02B2A08BF03464FF07E551C46002650
:107D5000234614F8012BA2F13007F9B209290DD8F6
:107D6000394930460CF034F8064638460BF0DCFF53
:107D7000014630460BF024FF0646E9E72E2A17D1CC
:107D8000314F234614F8010B3038C2B2092A0FD8FC
:107D90000BF0CAFF39460CF0CFF8014630460BF025
:107DA0000FFF2949064638460CF012F80746E8E767
:107DB0001A7802F0DF02452A39D15A782D2A02D1E9
:107DC0000233012704E02B2A14BF013302330027BA
:107DD000013B002413F8012F303AD1B2092903D80E
:107DE0000A2101FB0424F5E7B4F59A7F28BF4FF47C
:107DF0009A74A0464FF07E53B8F1070F07D9184682
:107E000012490BF0E5FFA8F108080346F4E704F077
:107E1000070434B118460C490BF0DAFF013C034665
:107E2000F7E719462FB130460CF086F804E04FF022
:107E30007E5130460BF0CCFF014628460BF0C8FFC0
:107E4000BDE8F081000080BF0000204120BCBE4C96
:107E500030B5054687B00C4603A800210C220FF070
:107E6000F6FC284600210CF06FF920B1284628497D
:107E70000BF0A6FE03E0284625490BF09FFE25499E
:107E80000BF0A6FF0CF06AF9054680EAE07069463F
:107E9000A0EBE5700AF0ACFD002DACBF20232D2334
:107EA00068468DF80C300FF016FD012807D13023FD
:107EB0008DF80D308DF80E308DF80F300CE0022863
:107EC00005D130238DF80D308DF80E3004E00328F5
:107ED00004BF30238DF80D30694603A80FF0DEFC97
:107EE00003A80FF0F8FC0338C5B22A4603A92046C0
:107EF0000FF01CFD00236355204607490FF0CEFC10
:107F000003AB204659190FF0C9FC204607B030BD1D
:107F10006F12033A00007A440CC9010870B5064696
:107F2000B6FBF2F40846154614B12046FFF7F6FFFB
:107F300005FB1464024B1B5D00F8013B70BD00BFE4
:107F40000EC901082DE9F04F81468A4616461C46A7
:107F500089B000253178002900F0DB80252902D086
:107F60000136484674E072784FF00008302A0CBFA2
:107F7000B278B71CA2F1300312BF4FF0000BF71C10
:107F80004FF0010B092B19D8A2F13003D9B20929FE
:107F900005D80A2202FB083817F8012BF4E7A2F1F2
:107FA0006103052B02D8A2F1570305E0A2F14103BA
:107FB000052B03D8A2F137030A2BEADD6C2A30D156
:107FC0003A787E1C642A00F083800BD8252A3DD0A5
:107FD00003D8002A00F09D80BCE7582A0CD0632A01
:107FE00019D0B7E7732A22D002D86E2A37D0B1E76A
:107FF000752A5CD0782AADD1271D2068A2F15804DB
:1080000062424FF01001624155E02CD9582A32D01B
:10801000632A2AD13E4648462178271DD04701359C
:108020000FE0642A63D00ED9732A14D13E46236828
:1080300048460093514642460023FFF712FE271D93
:1080400005443C4686E7252ADFD13E4648462521A1
:10805000D04701357EE70AD86E2A06D13E4623680E
:1080600004341D6076E7002A53D03E4672E7752A35
:1080700026D0782AF9D1A2F1580304F1040C5A420F
:108080002068CDF80CC04FF010015A4105ABFFF746
:1080900095FDDDF80CC03E46644605AB00934846AE
:1080A000514642465B46FFF7DCFD054452E7206837
:1080B000271D0A21002205ABFFF7A7FD3C46ECE790
:1080C00004F1040CCDF80CC020680A210022DDE781
:1080D0002068271D002808DA2D238DF8143040422F
:1080E0000DF115030A210022E6E705ABFAE7206847
:1080F00004F1040C00280ADA2D238DF814304042D4
:108100000DF11503CDF80CC00A210022BFE705AB25
:10811000F8E7284609B0BDE8F08F0EB40FB505ABFF
:1081200053F8042B0190064901A80393FFF70AFFB7
:10813000019B00221A7004B05DF804EB03B0704795
:10814000597C00080FB413B50B4904AB08680B4900
:1081500053F8042B09680193FFF7F4FE0446084B1B
:10816000186806F0F2FE0028F9D0204602B0BDE8FB
:10817000104004B0704700BF6C0800206808002061
:10818000100F002080EAE073A3EBE0738B4206DB64
:10819000002801DD401A704702D0084470470020D3
:1081A000704770B504460BF0D9FF2030402857D8EF
:1081B00020462C490BF0C8FF28B120462A490BF075
:1081C000FDFC0446F4E7204628490BF09FFF28B148
:1081D000204625490BF0F4FC0446F4E720462449E8
:1081E0000BF0B2FF30B1224920460BF0E7FC01460C
:1081F0001F480AE020461F490BF088FF40B11C4988
:1082000020460BF0DDFC01461A480BF0D7FC044673
:10821000214620460BF0DCFD0546204629460BF0A2
:10822000D7FD1549064628460BF0D2FD13490BF041
:10823000C5FC014628460BF0CBFD11490BF0C0FCF4
:10824000014628460BF0C4FD0E490BF0B7FC014671
:1082500030460BF0BDFD014620460BF0B1FC70BD71
:10826000002070BDDB0F4940DB0FC940DB0F49C068
:10827000DB0FC93FDB0FC9BF9A7C2E36FAAF4F39EF
:108280003587083CA4AA2A3E08B503490BF098FCA0
:10829000BDE8084085E700BFDB0FC93F2DE9F04F7F
:1082A000056885B0814628460C46FFF7EDFF8046FD
:1082B0002846FFF776FFD9F8045006462846FFF710
:1082C000E3FF07462846FFF76CFFD9F808900546FC
:1082D0004846FFF7D9FF82464846FFF762FF41460E
:1082E000814650460BF074FD4146834648460BF0EC
:1082F0006FFD5146019030460BF06AFD49460290F1
:1083000030460BF065FD3946039050460BF060FD9A
:108310004946206007F100400BF05AFD2946606095
:10832000A56002980BF054FD014601980BF048FC43
:108330002946E06003980BF04BFD014658460BF0D0
:108340003DFC3946206106F100400BF041FD294615
:10835000606158460BF03CFD014603980BF02EFC83
:108360002946A06101980BF033FD014602980BF0FD
:1083700027FC4146E06138460BF02AFD206205B03B
:10838000BDE8F08F2DE9F04107688AB0466885683E
:108390000446084601A9FFF781FF019938460BF012
:1083A00017FD0499804630460BF012FD0146404609
:1083B0000BF006FC0799804628460BF009FD0146A4
:1083C00040460BF0FDFB0299206038460BF000FDA3
:1083D0000599804630460BF0FBFC014640460BF009
:1083E000EFFB0899804628460BF0F2FC0146404618
:1083F0000BF0E6FB0399606038460BF0E9FC069948
:10840000074630460BF0E4FC014638460BF0D8FB3B
:108410000999064628460BF0DBFC014630460BF076
:10842000CFFBA0600AB0BDE8F081074B10B51A88F9
:108430001C4622EA00009042188002D0012006F07B
:108440000DFD208810BD00BFEC180020064B10B5B4
:108450001A881C4610439042188002D0012006F072
:10846000FDFC208810BD00BFEC180020024A936874
:1084700023EA0000906070472C10002008B5104BD4
:108480001A780023D9B2914207D20E49002051F840
:108490002310013309680880F4E7322006F07BFCE2
:1084A000094B1B685A0309D5084B9B685B0305D42D
:1084B000BDE8084040F2DC5006F06DBC08BD00BFCE
:1084C0005C2A00202C2A0020242F00202C100020C1
:1084D0002DE9F3410BF0C6F84B4A6923137040F2C3
:1084E000E4735380BE231371EF2382F8E137002336
:1084F0001946164682F8E237F25C0133514040F2E9
:10850000E4729342F8D1404B404A83F8E217404B63
:1085100004275A6002F188325A600020013F17F0A8
:10852000FF075ED03A4B34223A4CDA6004F17848C7
:10853000A8F5FC38C8F3090353B100234FF40050E9
:1085400056F80880019307F08DF90428E6D11CE065
:108550004FF4302007F086F90428DFD12C4D4FF47A
:1085600030202B6943F002032B616C612B6943F0CF
:1085700040032B6107F076F941F6FD732A69042860
:1085800003EA02032B61D8D0C8E7214D4FF4005015
:108590002B6943F001032B611FFA88F3238007F056
:1085A00061F9042813D1A31C0193019B4FEA1848D9
:1085B000A3F800804FF4005007F054F941F6FE7321
:1085C0002A69042803EA02032B6106D0A6E741F6D4
:1085D000FE732A6913402B61A0E70F4B04349C42C1
:1085E000A4D10B4A0428136943F08003136102D11C
:1085F00008F0BCF910B9052006F048FC0BF01CF897
:1086000002B0BDE8F08100BF2C10002023016745B7
:108610000020024000F80108E4FF01082DE9F041C4
:1086200008F0A4F910B9042006F030FCC04C0BF09F
:1086300019F8C04940F2E47220460FF0FDF894F8B2
:10864000B8374FF4CC71022B84BF002384F8B837BD
:1086500094F8B827B84D01FB02F303F53C702044B1
:108660002344286093F8440301FB0242022803F5E7
:10867000507384BF0020187192F84433AF4A1370CE
:108680000C2202FB0343AE4A03F2BA73136046F2B4
:108690000902A3681A401AB9A54A43F4005393602B
:1086A000A368DF0703D54FF40050FFF7DFFEA36890
:1086B0005E0409D50820FFF7D9FE4FF40050FFF7FC
:1086C000D5FE0120FFF7D2FEA368180706D54FF4A8
:1086D0000050FFF7CBFE0120FFF7C8FEA368990406
:1086E00013D54FF40040FFF7C1FE914B93F886314C
:1086F000012B03D14FF40060FFF7B8FE4FF4803038
:10870000FFF7B4FE4020FFF7B1FEA3685A0603D579
:108710004FF48030FFF7AAFEA36803F40852B2F5C5
:10872000085F0AD11B0508D5814B93F88631012BD0
:1087300003D14FF40060FFF799FE94F8E0217C4BE1
:108740002AB193F8E42112B1002283F8E4214FF01A
:10875000000C67467B4E7C4B1E6004EB0C03B3F8A9
:10876000F8E14FEA5E0101F077314FEA9E0303F032
:108770003333C1EB0E00C11A4FEADE0303F01133AD
:10878000CB1A03EB231303F00F32FF2392FBF3F317
:108790001EF00108C3EB032318BF0137A2EB03034C
:1087A00018BFFFB2012B0ADD022B40F0BE80B8F1EA
:1087B000000F00F0BA801EF0BC0F00F0B6800CF184
:1087C000080CBCF1280FC8D1013F012F00F2AD8089
:1087D00008F0A9F8302200215C480FF038F85C4F0F
:1087E0005C4BD5F800801F605B4B002108F17900DD
:1087F000C3F8008006F054FA584B80F0010018705E
:10880000574B07F126021A60564B07F1DC021A603B
:1088100098F8000006F066FE2868534B00F5C57214
:108820001A6004F09FFA514B94F8D81107F19402A2
:108830001A6064224A434E4BC8325A6000229A6042
:10884000DA601A615A619A61DA6183F8202083F84C
:108850002120484B2D6807F12C021A60464B05F287
:1088600019121A60454B05F289121A60444B07F140
:1088700008021A60434BDFF848811F60424B07F142
:10888000A0021A6007F1AA03C8F800303F4BB4F801
:1088900066011E600BF044FAC8F80800B4F86801DD
:1088A0000BF03EFA95F85C3008F1040288F80430C9
:1088B00095F87830C8F80C0088F8053094F8E33162
:1088C000286E88F81030324BC8F814501A60314BBB
:1088D00005F164021A6030490BF07AFA01464FF054
:1088E0007C500BF029FBB5F816412C4B1860204644
:1088F0000BF01AFA01462A480BF01EFB29490BF02F
:1089000067FA294A294B1560294A186005F168035E
:108910001360284A05F211151560274A1760274A87
:10892000BDE8F04113600AF087BE01F0E7FA4FE7B7
:108930002C10002000F801085C0F0020DC2E002025
:10894000840F0020B611002090330020140E002068
:1089500070110020480E00204C0E00201400002052
:10896000680100202C0D0020580E0020EC33002060
:108970009C330020142D002058290020980300204B
:10898000002B0020042B0020AC02002070030020EC
:10899000D0010020FC010020DB0F4940F80100203D
:1089A000000061444C3D0F44340100208C2B00201A
:1089B000280100209C020020A402002000010020C9
:1089C0000019002008B5FFF783FDFFF727FEBDE87B
:1089D0000840012006F042BA344B354A1B68126841
:1089E00010B51A60334A11685960516892689960ED
:1089F000DA60314A116819615168926859619A6167
:108A00002E4A1168D9615168926819625A622C4ADB
:108A100011881985518859859188D2889985DA8578
:108A2000284A118819865188598692889A86264A3A
:108A30001188D986518892881987194621F83A2FCA
:108A4000224A10780022824206DA214C34F8124081
:108A5000013221F8024FF6E71E4A1288A3F864207B
:108A60001D4A1288A3F866201C4A1188A3F86C10CE
:108A700051889288A3F86E10A3F87020184A3B2101
:108A800012689A66174A126892FBF1F2B2F5967F65
:108A9000C8BF4FF0FF325A67134A1288A3F87820F4
:108AA000124A5289A3F85E2010BD00BF8830002012
:108AB00000340020CC290020D8290020E4290020FF
:108AC00024100020440F00200E1000205C2A0020FB
:108AD000600F0020822C0020040F0020502C00206A
:108AE0001810002000000020800F00204A0F0020F6
:108AF0002DE9F84305460E460D4B002493E880030C
:108B0000B44213DA7B1933F9140008EB050333F987
:108B1000142009EB050333F9143001341344022205
:108B200093FBF2F3C01A08F080FAE9E7BDE8F88396
:108B30008830002010B5134B014693F8E037012B25
:108B400019D1114B114C1878421CD2B21A7012066E
:108B500044BF00221A700E4A1B78127821549342A7
:108B600036BFC2F180029B1A9B183F2B09D9BDE882
:108B7000104004F0C5BA074BBDE81040186806F075
:108B8000F0B910BD2C1000200C2E00200E2E00205D
:108B90000D2E00207030002070B54720FFF7CAFF6F
:108BA000174B1B681B0307D5164B174A5B681068E9
:108BB0001B68C01A08F029FA144E154C154D307870
:108BC00008F023FA23682868C01A08F02EFA6368B0
:108BD0006868C01A08F029FA0F4B188808F015FACF
:108BE0000E4B188808F011FA0D4B188808F00DFA92
:108BF000337823742B68A3606B68E36070BD00BF9B
:108C00000C32002088300020003400202E18002074
:108C100074300020301800202C1800202A18002062
:108C2000880F00207FB5264C264E274D2749284A1D
:108C3000284B20B128480088B0F5805F31D23088B9
:108C400091F820101278ADF8040028781C4D1B789C
:108C50008DF806008DF807108DF8082001A8294628
:108C600006228DF809300EF0D7FD30B30198BDF81B
:108C700008302860AB805320FFF75CFF208808F0A5
:108C8000C4F9A07808F0C1F9E37801A80193237929
:108C900002936379039308F01DF90F4B00221A80A9
:108CA0000BE0308891F820102080127828781B780B
:108CB000A070E17022716371DDE704B070BD00BF88
:108CC00018190020EC180020281800209C330020E0
:108CD0007F0D0020E40D00202C3200200A4A13886A
:108CE00001331380094A136801331360084A13885B
:108CF00001339BB2202B01BF00231380054A138848
:108D000008BF0133138070472C320020143200203A
:108D1000183200201A32002038B5394B05461B782E
:108D20000C46083B012B6AD84520FFF703FF284675
:108D3000FFF700FF0C2D23D004D80A2D0AD014D839
:108D400035B138BD0E2D4BD02ED3FF2D50D038BDB0
:108D5000206849E02078FFF7EDFE62796378002A09
:108D600014BF80200020184300E02078FFF7E2FEC7
:108D7000A078FFF7DFFEE078FFF7DCFE20793BE02C
:108D8000B4F9000008F036F9A078FFF7D3FEE078D8
:108D9000FFF7D0FEB4F9040008F02CF9B4F906008E
:108DA000BDE8384008F026B9637820788BB180F0B0
:108DB0008000FFF7BFFEA468E0B2FFF7BBFEC4F37C
:108DC0000720FFF7B7FEC4F30740FFF7B3FE200EFE
:108DD00012E0FFF7AFFE6068BDE8384008F025B943
:108DE000206808F012F96068BDE8384008F00DB955
:108DF000044808F01EF90020BDE838409AE638BD66
:108E00006C30002033C901082DE9F04FBE4B8BB008
:108E10001A880193BD4F002A40F0A98042F2010355
:108E2000B7F8DE07BA4EC21A50425041FFF7FAFEB9
:108E3000FFF7D2FD346849202546FFF77BFEB54B8E
:108E400004F11C09186808F0E0F855F8040B08F064
:108E5000DCF8284601F006F804F1100001F002F8F1
:108E60004FF01008AC4D01232A6803FA08F31342AF
:108E700003D0D9F8000008F0D8F808F10108B8F1DB
:108E8000130F09F10409EDD104F1280000F0DAFF15
:108E9000B7F84431B4F92E00C01A08F0B6F82B68C0
:108EA000DB0408D59D4BB4F864001B88181AC0F386
:108EB0000D0008F0AAF82B68980403D5B4F86600F2
:108EC00008F0A3F82B68590503D504F16C0000F0F5
:108ED000B9FF2B681A0502D5A06E08F0A6F82B681A
:108EE0005B0402D5606F08F0A0F82B68180403D566
:108EF000B4F8780008F089F8A04604F1300000F0DA
:108F0000A1FF04F1360000F09DFFB7F8443138F9B5
:108F10003C0F0127C01A08F078F8814B1B789F425C
:108F200008DA38F9020FB4F93C300137C01A08F0FA
:108F30007CF8F2E72B68990505D5B4F95E00A0F23C
:108F4000DC5008F072F8326876487260B260121A2B
:108F50009110754A4A43531C032293FBF2F202EB31
:108F600042029A1A7C2303FB02033360D6E16F4B63
:108F70006F4A1B6811688B4206D00AA941F8203D50
:108F800000201360FFF7C8FE019B97F8DE171B88CF
:108F900097F8DF070B44013BB3FBF0F200FB123301
:108FA0008B4280F086815A4F0120FFF73BFEFFF78E
:108FB00013FD50203E687D68FFF7BCFDBA683B6832
:108FC00010681B687A680344106806F11C0BA3EB59
:108FD000400008F02AF86A68736802A89B1A029396
:108FE000AA68B36805F11C089B1A0393EA68F36842
:108FF00010249B1A049300F035FF2A69336902A8F4
:109000009B1A02936A6973699B1A0393B369AA69ED
:109010009B1A049307F05EFF3F4901220B68A240B0
:109020001A428A4606D0DBF80000D8F80030C01A91
:1090300007F0FBFF0134132C0BF1040B08F10408BB
:10904000EAD106F1260005F12601002331F9024F8D
:1090500030F9022F121B02AC44F823200133042BF9
:10906000F4D103214FF000094FEA89035FFA83F935
:1090700002AB53F821206AB102F108000F2802D890
:1090800049F0010906E08032FF2A94BF49F0020945
:1090900049F0030911F1FF31E6D248460024FFF7F9
:1090A00049FDA0460DF1080B09F00302022A16D073
:1090B000032A1DD0012A4ED1B8F1000F05D1DBF8EB
:1090C000004090462401E4B245E0DBF800004FF098
:1090D000000800F00F002043FFF72CFD3BE0B8F143
:1090E000000F0CD0DBF80000C0F3031020432CE08D
:1090F000B8F1000F1ED19BF80100FFF71BFD9BF894
:109100000000FFF717FD26E0183200202C10002089
:1091100088300020143200200C3200200832002059
:109120005C2A002094300020DF7BEFBD203200203D
:109130001C320020DBF80000C0F303302043FFF7AF
:10914000F9FCDBF80000C0F30710FFF7F3FCDBF8D5
:1091500000402401E4B20BF1040B06AB9B454FEA3F
:109160009909A1D1B8F1010F02D12046FFF7E2FC25
:10917000DAF8003013F480541FBFB6F86420B5F855
:1091800064100124521A18BF02929A040AD50AAA3E
:1091900002EB8401B5F86600B6F866200134121AB5
:1091A00041F8202C580513D502AA02EB840C06F1D5
:1091B0006A0E05F16A0000223EF9021F30F9028FA3
:1091C000C8EB01014CF822100132032AF4D1033418
:1091D000190508D50AAA02EB8400A96EB26E013403
:1091E000521A40F8202C5A0408D50AAA02EB84002F
:1091F000696F726F0134521A40F8202C18040BD595
:109200000AAB03EB8402B5F87810B6F87830013475
:109210005B1A42F8203C00E0FCB1012C03D102981B
:1092200007F003FF19E0631E002002AA52F8232072
:109230004000C0B20AB140F00100013BF5D5FFF794
:1092400079FC4FF0000802AB53F8280008B107F092
:10925000ECFE08F10108A045F5DB30200321FFF703
:1092600047FC36200321FFF743FC2F4B3C201978A5
:10927000FFF73EFCDAF80030990506D5B6F95E0036
:10928000B5F95E30C01A07F0D0FE3A6827487B680F
:109290007A60121A9110264ABB604A43531C03227B
:1092A00093FBF2F202EB42029A1A7C2303FB0203C5
:1092B0003B60204B1B681A0630D51F4C1F4D22689F
:1092C0002B689A420BD162686B689A4207D1019B66
:1092D0001B88102B11D11A4B1B885B060DD148201F
:1092E000FFF728FC206807F0A0FE606807F09DFEED
:1092F00023682B6063686B600EE0124A0F4B117895
:109300002A7C914208D1104A99681068884203D19A
:109310005268DB689A4201D0FFF73EFC07F0C8FDB7
:109320000BB0BDE8F08F00BF5C2A00209430002015
:10933000DF7BEFBD242F00208C0F00207430002035
:109340001A3200202E180020301800202DE9F84F86
:109350000C9EC2EB030B394C0B9B002914BF4FF042
:10936000060A4FF0040AF61A636805460133904670
:1093700013D1236853455ED2314A032B98BF294647
:1093800052F823202F4807F0BFFE63680022013304
:1093900063602D4B05469A7113E0002511E02B4ABE
:1093A0001278954240DA0B9BE3B109FB06F2995C17
:1093B00001228A40264909680A4213D163680133B1
:1093C0006360D4F804900A9B1C4F9945E7DB2BD1CE
:1093D0000A20FFF7AFFB3B6801333B604FF0FF33E0
:1093E0007B6021E0184A917921B12C20FFF7A2FB84
:1093F000013501E00121917109FB0BF3226808EBB3
:10940000030752B958F8030007F013FE97F9041048
:1094100005444B1CD2D00F4802E03A440E48117963
:1094200007F072FE0544C9E7206850452CBF0020B4
:109430000120BDE8F88F0020BDE8F88F243200201D
:10944000A0A901083EC901081819002064000020E5
:109450000C3200204DC90108A7D20108426A806A77
:10946000131A5842584170474171704743799B071E
:109470000AD5436A8269D154436A01690133B3FB57
:10948000F1F201FB123343627047437913F0010399
:109490001FBFC36803F1FF32C369006A1DBF181AFA
:1094A0001040C0B218467047437910B513F001035D
:1094B00004460DD0FFF7E9FF58B1236A6269E168FD
:1094C000D05C0133B3FBF1F201FB1233236210BD18
:1094D000184610BD90F83B3210B57BB990F83A327F
:1094E00090F83942A34209D2B0F8401201229A40C2
:1094F0000A430133A0F84022DBB2F3E710BD8379C1
:10950000DB0748BFB1FA81F1D0F8343148BF4909CF
:109510005A681B8909B1136170475361704710F88D
:109520000A3C0133DBB20A2B84BF10F8131C054A36
:1095300000F80A3C82BF002322F8113000F80A3CF0
:10954000704700BFE8320020334A70B5136C906852
:10955000194440F68C23081A98429160D0605160FB
:1095600013463BD9127893F9451010468A420BD125
:10957000111F082908D893F84610182901D801317D
:1095800003E083F8442002E0002183F8461093F9B9
:1095900044402149A24219D191F84740B4B10C315D
:1095A0000024944206DA51F8046F1C4D25F814602B
:1095B0000134F6E70C2805D01849002421F81040A2
:1095C0000130F7E7164801780131017083F8452032
:1095D000002201211A7083F8471070BD92F84710DD
:1095E000C9B140F2DA51A0F2EF248C4208D81178C8
:1095F0000B2905D80B1D0131117042F8230070BDF5
:10960000002283F84720074B03F13002002143F882
:10961000041F9342FAD170BD94080020E832002064
:10962000DC000020A0080020024A136C013319441A
:109630001164704794080020024B53F820301B68D7
:10964000198070472C2A0020074BA1F57A7153F836
:1096500020301A681B8959434FF47A7391FBF3F158
:1096600089B21180704700BF2C2A00201FB501234A
:10967000ADF80830ADF80410002301A9ADF80A30A8
:10968000ADF80C30ADF8062006F0FDF805B05DF839
:1096900004FB38B5A0F513746379A579DB0745D5CC
:1096A00094F8383205F00105F3B1226B1068838D10
:1096B000C3F34E03838494F83C3223B1B4F84232AE
:1096C0000133A4F84232917A6A00FFF7CFFF0123F9
:1096D00084F83B32002384F8393284F83A3284F833
:1096E0003832A4F8403238BD94F83B322046012B82
:1096F00004BF94F8393284F83A32FFF7EBFE94F85D
:109700003B22236B3AB9012284F83B221868997AEC
:1097100005FA02F207E0002284F83B22954218681D
:10972000997A08BF0222BDE838409FE738BD10B5DE
:10973000A0F5127494F83C22BAB9A36A616A9942FE
:1097400028D0591CA069A162C35C2069DBB25B0010
:1097500043F400738142A4F83E324FF00A0384F8C8
:109760003D3228BFA262012312E094F93D327BB161
:10977000B4F83E1220464B08A4F83E3201F0010135
:10978000FFF7BDFE94F83D32013B84F83D3201E025
:1097900084F83C3294F83832002B4ED194F83932A8
:1097A0000133DBB2092B84F8393203D12046BDE8FE
:1097B00010408FE60A2B40D194F83B322BB9B4F815
:1097C000403243F00103A4F840326379D9071CD535
:1097D000B4F84002820501D4C30705D4B4F844327A
:1097E0000133A4F8443210E0E36AC0F347000BB140
:1097F00098470AE0E3696269D054E369E16801339C
:10980000B3FBF1F201FB1233E361012284F8382249
:1098100094F83B220023012A84F839320DD1A27931
:1098200084F83B32236B12F0010F1868997A0CBF51
:1098300002220022BDE8104018E710BDF0B5046D0B
:109840008279A389467923F4005312F0020F4FEA7C
:1098500003434FEA13430CBF00214FF4005112F0B1
:10986000040FA38114BF4FF4806E4FF0000E16F06A
:10987000010F8768054614BF04200020B307238A20
:1098800048BF40F008029BB223F4405343EA01036F
:109890002382A18948BF90B289B221F4B05121F04E
:1098A0000C014EEA010140EA0102A281A38A87B0BD
:1098B00023F440731B041B0CA38201A805F088FF4E
:1098C000039B049E254A944218BF1E46A389192271
:1098D00072431BB2002BB4BF7E00BE00B2FBF6F693
:1098E0006427B6FBF7F00001010907FB1163A289A9
:1098F00012B2002AB7BFD9001A013231B1FBF7F218
:10990000A7BF3232B2FBF7F302F007021043A8BF41
:1099100003F00F03AA79A8BF184380B212F0010F19
:1099200020812B6D06D00E498B4202BF042001F529
:109930004841086112F0080F9A8A0BBF22F0080212
:1099400092B2120442F0080208BF120C9A829A895D
:1099500092B242F400529A8107B0F0BD0038014043
:10996000004400402DE9F04F504C4FF4147685B080
:10997000804691461D4606FB0046274608B94C4BDB
:1099800002E0012804D14B4B33631033C6F8343165
:109990004FF4147303FB08F3474AFC18FA500322F0
:1099A0006271224603F59C733B44E162A36100218E
:1099B0004FF48070D4F8343134324FF0010B6261CF
:1099C0002162E161A162616284F83C1284F839127B
:1099D000A4F84212A4F84412C4F80890A571E060FB
:1099E000206184F838B284F8468258681B890222C4
:1099F000ADF80C3003A910238DF80E308DF80F2030
:109A0000019203F06EFD236B019A597B58681B8904
:109A10008DF80E1003A9ADF80C308DF80F2003F06F
:109A200060FD30465946FFF76AFD322005F0B3F974
:109A3000224BD4F834A11B681A46B2FBF9F1B1F5F8
:109A4000803F03D3012AF8D95208F6E71C4A504652
:109A5000B3FBF2F289B2D2B201F0D8F84FF414702D
:109A600000FB08F0174B07EB000800F512703C18DC
:109A70000022C8F848325046214601F00FF9D8F8C4
:109A8000307015F0010F0CBF022200223868B97A3D
:109A9000FFF7ECFD0C4B3846C8F84C32211D002274
:109AA00001F0FCF8304605B0BDE8F08F2019002029
:109AB000D4C40108F4C40108B8A90108600000205A
:109AC00040420F002F9700089396000803460A466D
:109AD00090F84602D96A9B7944E71FB50123ADF897
:109AE00008300023ADF80C30ADF80A30084BADF863
:109AF00004101B7801A9012B08BF0323ADF8062031
:109B000008BFADF80C3005F0BEFE05B05DF804FBF3
:109B10009008002038B510F80E2C044650F8043C8C
:109B200052B9012200F80E2C20F80C1C997A186802
:109B30000222BDE83840D0E730F80C2C20F80A1C8F
:109B4000891A89B220F8081C074A10F80F0C002562
:109B500022F8101004F80E5C1868997A2A46FFF76C
:109B6000BCFF04F8065C38BDE8320020044B53F813
:109B700020301BB107289CBF1B681980704700BFAD
:109B8000BC0900202DE9F7438E460546DFF8A09278
:109B9000114699F8A0440068164698467246631C20
:109BA00089F8A03400F0DEFF2B8901A9ADF804305C
:109BB00018238DF80630686802238DF8073003F00B
:109BC00090FCAB7A09F2A447240127442A6849464D
:109BD0000C2B00F2F680DFE813F00D00F400F40027
:109BE000F4005100F400F400F4008A00F400F400E2
:109BF000F400C200138CDFF83CC223F001031B0405
:109C00001B0C1384138CB2F804E0108B624520F017
:109C100073004FEA00404FEA10409BB21FFA8EFEDD
:109C200040F0700014D00CF5006C624510D00CF5BB
:109C3000406C62450CD00CF5806C624508D00CF588
:109C4000806C624504D023F0020343F0030307E075
:109C500023F00E032EF4407E43F003034EF4807E87
:109C6000A2F804E01083A2F834801384138B23F04D
:109C700008031B041B0C43F0080336E0138CDFF8C9
:109C8000B4C123F010031B041B0C1384138CB2F813
:109C900004E0108B624520F4E6404FEA00404FEAB2
:109CA00010409BB21FFA8EFE40F4E04008D00CF545
:109CB000006C624504D023F0200343F0300307E03A
:109CC00023F0E0032EF4406E43F030034EF4806E38
:109CD000A2F804E01083A2F838801384138B23F4D5
:109CE00000631B041B0C43F40063138369E0138CB3
:109CF000DFF840C123F480731B041B0C1384138C06
:109D0000B2F804E0908B624520F073004FEA004007
:109D10004FEA10409BB21FFA8EFE40F0700008D050
:109D20000CF5006C624504D023F4007343F44073D7
:109D300007E023F460632EF4405E43F440734EF476
:109D4000805EA2F804E09083A2F83C801384938B99
:109D500023F008031B041B0C43F0080330E0138CB2
:109D6000DFF8D0C023F480531B041B0C1384108C29
:109D7000B2F804E0938B20F4005023F4E6431B0474
:109D800000041B0C000C62451FFA8EFE43F4E043F6
:109D900040F4405003D00CF5006C624503D12EF422
:109DA000804E4EF4804EA2F804E09383A2F84080E7
:109DB0001084938B23F400631B041B0C43F4006397
:109DC00093832B7B43B1B2F844306FEA43436FEA8D
:109DD00053439BB2A2F8443013889BB243F0010373
:109DE0001380AB7A0C2B19D8DFE803F0071818188A
:109DF0000B1818180F18181813000B1902F134005B
:109E00000AE00B1902F1380006E00B1902F13C00E0
:109E100002E00B1902F14000C3F8A40438460C44D8
:109E2000A4F8AC64C4F8A82403B0BDE8F08300BF74
:109E300020190020002C014003F022BA03F020BAC0
:109E400003F01EBA10B50446B0F9000007F0EDF8B3
:109E5000B4F9020007F0E9F8B4F90400BDE81040D5
:109E600007F0E3B810B50446006807F0DEF8606854
:109E700007F0DBF8A068BDE8104007F0D6B82DE980
:109E8000F74F012004F07EFE002480B3012C2ED871
:109E90004FF04C0A0AFB04F7DFF85C8008EB070B75
:109EA0000BF14806B57815B10134E4B2EDE790F94D
:109EB000003090F804E018460E4B03228DE8240091
:109EC00001212A4653F82E30FDF728FE814650B175
:109ED0005846294652460DF0BAFC01231C4448F866
:109EE0000790B370E4B2012004F030FECDE703B078
:109EF000BDE8F08FD0A90108841E002000212A228D
:109F000010B511480DF0A3FC104B00221946104863
:109F10000424105C013283F8F601052083F8FB412C
:109F200082424FF0000483F8FA0183F8FD4183F880
:109F3000FC0103F10803EAD10123A1F8F83152230F
:109F400081F8F43110BD00BF201200202C10002039
:109F500071C9010870B50646441E14F8011F89B185
:109F6000094D28460DF0A9FC0028F6D005F108039C
:109F700098423FBF054B401BC018A31B38BF80F859
:109F80008A31EAE770BD00BF2EDF01082C100020E7
:109F900007B51C4B03F19C02C3F898201A4A92F8AB
:109FA00092215AB1012A14D1032183F89E1007216E
:109FB00083F8A02083F89F100C2208E0022183F888
:109FC0009E10032183F8A02083F89F10072283F8B6
:109FD0009C200E4A0E4B40201A6004F0D3FD70B155
:109FE0000122002390F9000040218DE80C00094A6D
:109FF0004FF4E133FDF792FD003018BF012003B0AC
:10A000005DF804FB841E00202C1000200933010899
:10A010002C000020B93301082DE9F04F8DB01F4608
:10A02000BDF95830B34C01939DF86030039205465A
:10A030000C220E4604F1A400002102930DF007FC4F
:10A040000021142204F1B0000DF001FC002384F87B
:10A05000C430A94B93F800909846A84B03F118021E
:10A06000B9F1010F88BF1346C4F8C830FCF7BCF93A
:10A070008246834670B3A24BB5F5807FC4F8B030FA
:10A08000A04BC4F8B430A04BC4F8BC309F4BC4F80C
:10A09000C0309F4B01D1002216E0BB2D01D9012217
:10A0A00012E0612D01D902220EE0292D01D90322EF
:10A0B0000AE0132D01D9042206E0092D01D9052259
:10A0C00002E0002DE7D006221A71012384F8C43083
:10A0D00002236AE0192004F05EFE68201521524632
:10A0E00007F0E8F978B38B4A622DC4F8B0208A4AA9
:10A0F000C4F8B420894AC4F8B820894AC4F8BC20FE
:10A10000824AC4F8C020824A0FD004D80A2D13D046
:10A11000142D0FD00CE0BC2D05D0B5F5807F07D1F4
:10A1200082F805A00AE0012300E00223537105E054
:10A130000323FBE70423F9E70523F7E7012384F86A
:10A14000C430042331E0B9F1030F40F0F983FCF788
:10A1500007F9002800F0F483724BBB2DC4F8B0302F
:10A16000714BC4F8B430714BC4F8BC30674BC4F8C1
:10A17000C030674B01D901220FE0612D01D90222C5
:10A180000BE0292D02D983F806900AE0132D01D99E
:10A19000042202E0092D02D905229A7101E006226B
:10A1A000FBE7012384F8C4300723614A1370614A36
:10A1B000136843F0010313605F4B00221A70994645
:10A1C000082E33D8DFE806F0383238101D22102D63
:10A1D0002D004FF0000A0CAB03F818AD5320514688
:10A1E000012207F027F960BB444B98F8001003F1F7
:10A1F0001802012988BF1346C4F8C830FCF7F4F8E8
:10A2000080BB98F80030012B40F2A08000210CABFD
:10A2100003F8181D1820012207F00CF9002840F05F
:10A22000B58098F80030032B00F0C080012E40F27A
:10A23000D380414B00261E7098F80030012BD3D8F4
:10A24000C7E79DF81830E52BCED13C4B84F8CCA065
:10A25000C4F8A4303A4BC4F8A830042389F800307D
:10A260000223B2E006210A4606AB682007F0E2F8B6
:10A270009DF81D1001F001029DF81B1001F0010175
:10A280004B0043EA82019DF8192002F001030B43C1
:10A290000AD05BB2012B01D1002302E0022B0ED1C8
:10A2A000012384F8CD3011E005AB68200C21012298
:10A2B00007F0C0F89DF8143013F00F0303D103200A
:10A2C00004F0E4FD02E0042BEAD1E5E71D4BC4F8FD
:10A2D000A4301D4BC4F8A83094F8CD30002B0CBF2F
:10A2E0006F236E2384F8AC30012389F800300323F8
:10A2F0006BE000BF841E00201B340020F0A9010881
:10A300005D620008D55C0008D55A000890C1793D0F
:10A310002C00002001630008AD5D0008795D000895
:10A32000595D0008296100088D6000086960000817
:10A3300058000020241800201A340020695B00080F
:10A340008D5E0008D5620008175D000800220CAB86
:10A3500003F8182D1C200D21012207F06BF80028AE
:10A360003FF454AF9DF818302A2B02D01A2B7FF4FB
:10A370004DAFD34A84F8CE30C4F8A420D14A02238A
:10A3800089F80030C4F8A82004231EE09DF8183096
:10A39000FB2B7FF446AFCC4BC4F8A430CB4BC4F8B6
:10A3A000A830012389F8003005230EE0FBF7D8FF21
:10A3B00000283FF43BAFC64BC4F8A430C54BC4F8EB
:10A3C000A830012389F800300823C34A5370C34AD8
:10A3D000136843F00203136098F80030012B05D195
:10A3E00008F0CCF8BE4B4FF400525A61042F00F233
:10A3F000CD81DFE817F00500D40169000500920166
:10A400000A2004F0C8FC7720A021012205AB07F048
:10A4100011F8002858D01E210122772007F04AF8B1
:10A420004FF42F6004F0ACFC0027A7F16001002678
:10A43000C9B2022206AB77208DF818608DF819603A
:10A4400006F0F8FF9DF819309DF8182043EA022223
:10A45000A44B03F1D0017A520237102FE5D1B3F8A3
:10A46000DE10324601F00F0701F47F41A3F8DE1041
:10A4700033464FF0010E22F001002044B0F8D00026
:10A48000002818BF4FF0000ED60703D5C0B24340D6
:10A49000082002E083EA1023FAE71E0448BF83F491
:10A4A000C05301384FEA4303F7D10132102AE2D1F9
:10A4B00039438C4AA4F8DE10BEF1000F04D1C3F377
:10A4C00003339F4200F0178294F8E060002E40F0C2
:10A4D0002F82834F08F052F84FF48048282405A9B2
:10A4E0003846ADF814808DF8164002F0FAFF4FF4AC
:10A4F00000533B617C4804F013FD0E21022002F062
:10A50000DBFF0823CDF8188006A84FF001088DF86E
:10A510001D308DF81C608DF81E804FF0030905F08A
:10A52000C5FA04A88DF810408DF811908DF81260CE
:10A530008DF8138007F0A8FF142004F02CFC42468D
:10A540007720D02105AB06F075FF664C3A4600280F
:10A5500000F09F809DF81430A4F80491552B84F8E6
:10A56000FB3040F09680D121424605AB772006F0C3
:10A5700061FF9DF81430772003F00F021B0984F867
:10A58000FC2084F8FD30162206ABAA2106F052FF0B
:10A590009DF818209DF8193043EA0223A4F8E4300E
:10A5A0009DF81A209DF81B3043EA0223A4F8E630F8
:10A5B0009DF81C209DF81D3043EA0223A4F8E830E2
:10A5C0009DF81E209DF81F3043EA0223A4F8EA30CC
:10A5D0009DF820209DF8213043EA0223A4F8EC30B6
:10A5E0009DF822209DF8233043EA0223A4F8EE30A0
:10A5F0009DF824209DF8253043EA0223A4F8F0308A
:10A600009DF826209DF8273043EA0223A4F8F23073
:10A610009DF828209DF8293043EA0223A4F8F4305D
:10A620009DF82A209DF82B3043EA0223A4F8F63047
:10A630009DF82C209DF82D3043EA0223A4F8F83031
:10A6400041F27073A4F8083146F67813A4F80A3181
:10A65000264BC4F80C31264BC4F81031254BC4F8F6
:10A660001431254BC4F81831244BC4F81C3194F82C
:10A67000E03043B9FBF75CFA42F6E06004F080FB9F
:10A68000BE68C6F380361E4BDE71012384F8E030CD
:10A690004EE11C49D4F820010B6823F480430B6081
:10A6A000114B1049984209D0D1F8240198422BD07F
:10A6B000D1F8281199422DD1022326E0002324E06D
:10A6C000B15F0008ED5D0008455B0008475E0008CB
:10A6D000C55A0008CB60000858000020241800204C
:10A6E00000100140841E00205D5F0008315B0008FF
:10A6F000A15C00080B5B0008555C0008E9590008E4
:10A700002C00002000040140012304EB83040023FB
:10A71000C4F820314FF4005353618B4C94F82C61F2
:10A72000002E40F0FF80142004F035FB04F22D13BE
:10A730007620D021012206F07DFE94F82D31582B91
:10A740002DD104F5987388211822762006F072FE28
:10A750007620F421312206F0ADFE012384F82C315D
:10A760007A4BA4F80861C4F81031794BC4F80C3165
:10A7700045F6D813A4F80A31764BC4F81431764B59
:10A78000C4F81831754BC4F81C31CBE0012F06D04A
:10A79000734B744A9F70136843F004031360714E47
:10A7A000694C336813F0020F02D0D4F8A4309847F4
:10A7B000029B63B315F0FF0F336809D140F2596271
:10A7C00013F0020F40F2712318BF13467D2208E0F8
:10A7D0009A0759BF4FF47A731A464FF4FA634FF44D
:10A7E0007A721799994205DBB1F57A6F0B46A8BFCB
:10A7F0004FF47A63511E0B44B3FBF2F3013BDBB21F
:10A8000003FB022284F84C31C4F8502106E09DF885
:10A81000083084F84C31179BC4F85031D4F8B0306C
:10A820009847514B039F93F80090504B03F1180247
:10A83000B9F1010F94BF994691464D4D00232B70FD
:10A840000FB1022F70D14FF000080CAB03F8188D38
:10A850001E200A210122DFF8F0B0C4F8549106F05E
:10A86000E9FD98B19DF81830482B63D1414B022285
:10A87000CBF85831404BCBF85C3103232B70384B6D
:10A88000DA70336843F00803336001E0804651E03A
:10A890003A4B93F858210AB184F8C42093F859210F
:10A8A0000AB137490A7093F85A3103B12B703368F3
:10A8B0001B071AD5019B642693FBF6F5284609F081
:10A8C00033FA019B074606FB153000B209F02CFA5B
:10A8D0002C4909F07DFA0146384609F071F92A49F8
:10A8E00009F076FAC4F8600102E00023C4F8603190
:10A8F0004FF0010B24E042F21073A2F80831A2F8E5
:10A900000A31224B0327C2F80C31214BC2F8103117
:10A91000204BC2F81431204BC2F818311F4BC2F83B
:10A920001C3135E7042733E7012FB1D91F4684E7EF
:10A9300002272DE7012FABD9002785F8008082E799
:10A9400058460DB0BDE8F08F841E0020E559000880
:10A95000E7590008015B0008095C000881570008FE
:10A9600058000020241800201B34002020AA0108D1
:10A970001C34002047D50008E5D100082C10002029
:10A980001A3400208988883C00002041F75A0008CA
:10A99000F95B0008ED5A0008E95B0008C55500089E
:10A9A0000120002107F0F8BA026D70B51588044641
:10A9B000ADB2A90613D5036B8BB9C36A1BB19088DE
:10A9C00080B298470BE0E169928840694E1CD2B290
:10A9D000E6614254E169E268914228BFE3612B06D7
:10A9E00013D5636AA26A9A42236D0AD0511CA069EA
:10A9F000A162825C9A802369994206D30023A362F4
:10AA000070BDDA6822F08002DA6070BD026B034626
:10AA1000C16810B5406942B11A6C8C1A013A08BF7E
:10AA20000A46005D1A64C0B210BD1A6A805C013229
:10AA30008A4228BF0022C0B21A6210BD436B13B114
:10AA400090F844007047836A406A1B1A5842584184
:10AA50007047036B13B15B68016C01E0C369016A65
:10AA60008B423CBFC2689B18581AC0B27047836AB9
:10AA70008169426B1944D160416A994297BF01696B
:10AA8000CB1ACB1A536096BF0023536083624FF0FA
:10AA9000000380F84430136888BF816243F00103EB
:10AAA00013607047436A8269D154436A0269013373
:10AAB000934228BF00234362436B1BB11B68DB0733
:10AAC00005D4D4E7026DD36843F08003D3607047A8
:10AAD0004171FEF7B3BE8160FEF7B0BE2DE9F041D3
:10AAE00005460E46078A83899BB21F40002F37D048
:10AAF000B7FA87F24FF00043D340DB4399B21F40CF
:10AB0000A2F11B032982042BF0D8DFE803F0221FF7
:10AB10001C190300746A24B1013C0023A4B27362BF
:10AB200001E0AC8DA4B2D6F82080B8F1000FDDD0E2
:10AB3000D8F80030404621469847D8F80480F4E71A
:10AB40003068A98E08E07068298F05E0B068A98F89
:10AB500002E0F068B5F84010036889B29847C5E78D
:10AB6000BDE8F081254B10B55A43254B254C1B6899
:10AB70000139B3FBF2F20388013AA04289B292B2E2
:10AB80009BB212D004F50064A0420ED0B0F1804F09
:10AB90000BD0A4F59834A04207D004F58064A042FD
:10ABA00003D004F58064A04202D123F070039BB26D
:10ABB000154CA04206D004F58064A0421CBF23F4CB
:10ABC00040739BB203800F4B8185984202850FD062
:10ABD00003F5006398420BD003F54063984207D019
:10ABE00003F58063984203D003F58063984201D156
:10ABF000002303860123838210BD00BF40420F0063
:10AC000060000020002C01400010004073B5054694
:10AC10000068FFF7A7FF2A680124138800269BB26B
:10AC200043F001031380EB7A01A88DF804308DF80E
:10AC300005408DF806608DF8074007F025FCEB7A9B
:10AC40001B2B0BD1192301A88DF804308DF805407A
:10AC50008DF806608DF8074007F016FC02B070BD55
:10AC60000C4B800A98420CD004D8B0F5801F0CD150
:10AC700001207047084B984205D04933984206D0CE
:10AC800003E00220704703207047FE207047002039
:10AC9000704700BF01001000020010002DE9F843CA
:10ACA00004680746204688469146FFF7D9FF0328E7
:10ACB0004BD8BA7A9108B8F1000F06D1A589AEB287
:10ACC00002258D4026EA0505A5810A2303FB001312
:10ACD0001F4A42F82380043342F82390B8F1000F52
:10ACE00007D0BD7AA189AD080223AB400B439BB2CC
:10ACF000A3812823434303F120011144EFF312867B
:10AD0000502585F3128803F10C051C3315441344B8
:10AD100055F8047F17B10F60296804319D42F7D1BF
:10AD200000230B60F3B283F31188282303FB002078
:10AD3000036A23B1A3899BB243F0010304E0A38912
:10AD400023F001031B041B0CA381BDE8F88300BFA3
:10AD5000602A0020004827E6E81F0020004823E67C
:10AD60003C20002000481FE6902000200B4B4FF4B1
:10AD700000525A604FF6FE730948D0F8DC20116883
:10AD80000B401360D0F8CC20D0F8D0309A4201D0DC
:10AD9000A8306CE6012380F8EC30704700000240D8
:10ADA000E81F00202DE9F0431D46A64B8DB09842C8
:10ADB000884617469DF850605CD1A34BA34AA4492E
:10ADC000C3F8A82003F1FC02C3F8BC2003F5FE720F
:10ADD000C3F8C0204FF48072C3F8B420C3F8B82081
:10ADE0009C4AC3F8B070C3F8D820A2F54842543A40
:10ADF000C3F8F420C3F8F020C3F8F800C3F8DC105F
:10AE0000954B9A6942F480429A615A6942F0010274
:10AE10005A6102238DF803304FF40073ADF800300F
:10AE2000330701D51C230FE0AC0706D518238B4848
:10AE300069468DF8023002F054FBE8070AD54FF45A
:10AE40008063ADF800304823844869468DF80230AD
:10AE500002F047FB0E238DF804300022012301A8E5
:10AE60008DF805308DF806208DF807307C4C07F002
:10AE70000BFBA1E07B4B98424ED1734B734ADF65CD
:10AE80005A654FF480721A665A6603F53F729A66E5
:10AE900003F57F72DA66744AC3F8A400C3F89C20F5
:10AEA000C3F8A0206C4B3107DA6942F40032DA6152
:10AEB0005A6942F001025A614FF002038DF80330E3
:10AEC0004FF00403ADF8003001D51C230EE0AA07B3
:10AED00006D51823614869468DF8023002F001FB5F
:10AEE000EB0709D50823ADF8003048235B486946D5
:10AEF0008DF8023002F0F5FA26238DF80430002296
:10AF0000012301A88DF805308DF806208DF8073053
:10AF1000564C07F0B9FA4FE0554B984240F0ED809F
:10AF2000494B4A4A9F601A6003F2FC425A6103F29D
:10AF3000FC529A614FF48072DA601A614D4A1865CA
:10AF40009A64DA64444B3407DA6942F48022DA61A5
:10AF50009A6942F008029A614FF002038DF80330BB
:10AF60004FF48063ADF8003001D51C230FE0A80733
:10AF700006D51823404869468DF8023002F0B1FA30
:10AF8000E9070AD54FF40063ADF8003048233A488A
:10AF900069468DF8023002F0A4FA27238DF80430B8
:10AFA0000022012301A88DF805308DF806208DF8C8
:10AFB000073007F069FA244C4FF00009012384F8A8
:10AFC0004430C4F82090C4F81C90C4F82890C4F809
:10AFD0002490C4F82C806571A760A6712046FEF706
:10AFE0002DFCEA0752D5206B002847D0E36CCDF842
:10AFF0000C9001934FF480530A9380230693E368E7
:10B00000CDF814900493202309936369CDF81C9024
:10B010000293CDF82090CDF82C9004F061FB01A9AB
:10B02000206B04F03FFB226B216D136843F001039A
:10B0300013608B8A9BB243F040038B8253689BB2B0
:10B04000236423E000380140E81F002050AA0108D3
:10B050004400024058000240001002400008014035
:10B060009020002000440040044400403C20002088
:10B070000048004004480040000C01404FF6DF72D9
:10B08000236D1A80DA6842F02002DA60AB072CD513
:10B09000606B28B3A36C002501934FF480530A938F
:10B0A0008023069323690295049310230393059547
:10B0B0000795089509950B9504F012FB606B01A9A3
:10B0C00004F0F0FA636B1A6842F002021A60226D13
:10B0D0005D605D60938A9BB243F08003938204E0DD
:10B0E000226DD36843F08003D360226D204693899C
:10B0F0009BB243F40053938100E000200DB0BDE803
:10B10000F08300BF08B507480CF0E5FBC0B2142877
:10B11000044B04D8421C20211954D0B2F7E7002276
:10B120001A5408BDA82E00202DE9F74F03F00CFE9D
:10B13000A64C804626686568A768861BF643451BB3
:10B14000C71BED43FF43F60FED0FFF0F2EB93FB9BD
:10B15000002D00F08782B9462CE04FF0000929E06D
:10B16000B14627E003EB8A0BBBF802301A050ED478
:10B1700013F4805F1DBF964A9BF801101268954A30
:10B18000954B14BF52F82120126843F82A20BBF8CF
:10B190000230D80516D499050AD5904B1B7813F0C8
:10B1A000040F0CBF8E4A8F4A8B4B126843F82A203B
:10B1B00009F10109207B5FFA89FA8B4982450B6806
:10B1C000D0D326E0894A5046594604F065FF884BA3
:10B1D0001B885A0603D550465946864A16E058073A
:10B1E00003D550465946844A10E0190703D5504606
:10B1F0005946824A0AE09A0703D550465946804A82
:10B2000004E0DB07D4D5504659467E4A04F044FF9B
:10B21000CEE7DFF808E20093BEF906307822A3F506
:10B220007A7353434FF47A7293FBF2F3F34603F2CB
:10B230002B13019300225FFA82FE864517D2009BF2
:10B2400003EB820EBEF802E01EF4806F0DD040F2D8
:10B25000671ADFF88491019B39F822E09E449EFB37
:10B26000FAFC0AFB1CEE29F822E00132E3E74DB3B9
:10B2700008F5C333A0336360637B544A13BB9373F5
:10B28000614B1B6813F0020F0AD0DFF894E19EF8BF
:10B2900000E0BEF1000F03D04FF0010E82F80EE087
:10B2A000DA0506D5594BDB781BB1A37B43F00203CB
:10B2B000A3734A4B1B7813F0050F02BFA37B43F027
:10B2C0000403A37394F80EE0BEF1000F03D13F4BCB
:10B2D0005B7B002B4FD094F80DC01CF0010FACF13C
:10B2E0000C031DD1BCF1030F07D8DFF8E8901EF066
:10B2F000040F3B4A08BF4A4600E0364AACF1040C52
:10B30000BCF1070F05D8DFF81CC11EF0010F18BFF4
:10B310006246DBB2032B0ED81EF0020F3C4B06E058
:10B32000DBB2032B06D82F4B2A4A1EF0020F18BFA0
:10B330001A4600E0274A4FF0000C5FFA8CF3834274
:10B340000DD20B6803EB8C035B881B0642BFD2F85F
:10B350000090214B43F82C900CF1010CEDE785B1E6
:10B36000BEF1000F08D0637B184A0133DBB2142B07
:10B3700006D1002304E025B1637B002BF3D100E06C
:10B380005373002E52D0234A3223B2F90250B2F93D
:10B390000020002DB8BF6D42002AB8BF524295FB75
:10B3A000F3F592FBF3F2EDB2D3B2AB4238BF2B46CA
:10B3B000194A13B192FBF3F300E0134643442360B0
:10B3C000E37B024A83BB01232FE000BFE426002079
:10B3D000542900206CC10108E20700201934002024
:10B3E00064B2010854B20108F018002068AA0108EC
:10B3F000EC1800206EAA010874AA01087AAA0108B4
:10B4000080AA010886AA0108242F00209C3300206E
:10B410006CB2010824100020400D0300602F0020B2
:10B420007418002074B201080023D3738F4D904B21
:10B430002D78E27BADB9002F00F00F818D4B267B7C
:10B440001A788D4B02F0040293F800C08B4BD2B2F5
:10B45000D3F800E00B680021894D03EB86060F4608
:10B46000B5E01AB9874A1A61002508E0864AFAE76A
:10B470000A68AB00D6187688760604D40135EBB29C
:10B480008342F5D3D7E7814EB6F90060192E25DD4A
:10B4900012F803E094F814C00EF00F09E145266994
:10B4A0000CDCDFF8CCC19CF815C0BCEB1E1FDEBF66
:10B4B000D6F800C0DFF8D8E143F80EC012F803E078
:10B4C00094F816C00EF00F09E14533DBDFF8A0C198
:10B4D0009CF815C0BCEB1E1F2CDC26E0193629DABF
:10B4E00012F803E094F814C00EF00F09E145266944
:10B4F0000CDCDFF87CC19CF817C0BCEB1E1FA2BFA0
:10B50000D6F800C0DFF888E143F80EC012F803E077
:10B5100094F816C00EF00F09E1450BDBDFF850C1BF
:10B520009CF817C0BCEB1E1F04DBD6F800E0584E99
:10B5300043F806E0554EB6F90260192E1BDD12F8ED
:10B5400003C094F814E00CF00F09F14526690CDCF7
:10B55000DFF81C9199F81590B9EB1C1FDEBFD6F8E7
:10B560000090DFF82CC143F80C90D25C02F00F0C75
:10B57000F4451EDD82E7193680DA12F803C094F82C
:10B5800016E00CF00F09F14526690CDBDFF8E090BE
:10B5900099F81590B9EB1C1FDEBFD6F80090DFF8C4
:10B5A000F0C043F80C90D25C02F00F0CF445FFF6AB
:10B5B00065AF94F817E0BEEB121FA2BF3668344A9D
:10B5C0009E505BE75888000504D404330435B34229
:10B5D000F8D122E04AB101EB0C0A06209AFBF0F9FF
:10B5E00000FB19A001280DDC01E057B9012793F8F1
:10B5F00001900EEB89003EF829A090F80290C078E7
:10B6000003E01746002081468246013125F802AC4E
:10B6100085F800906870C9B2D7E7174A1378013BE4
:10B6200013F0FF0308BF06231370124B1B785B0750
:10B6300041BFBBF906304FF47A72A3F57A7303EB7E
:10B64000C30348BF93FBF2F3124A46BF0133DBB298
:10B65000012392FBF3F34344A36003B0BDE8F04F32
:10B6600001F04CBE03B0BDE8F08F00BF7F0D00209D
:10B67000E426002019340020340000205429002042
:10B68000E407002070B201086CC1010824100020FA
:10B69000E2070020400D03002DE9F04F054690F829
:10B6A00050008DB008910592099318B13228A8BFB7
:10B6B000322000E0012008F037FB0146AA4808F0DC
:10B6C0003BFCAA4B04461888002808BF012008F05C
:10B6D0002BFBA749069008F07BFB019001992046BF
:10B6E00008F06EFA0146019808F026FCA14B07907D
:10B6F0001B889A0724D5A049B1F90030B1F902009E
:10B7000083EAE37280EAE071A2EBE372A1EBE071FD
:10B7100091420C46B8BF1446B4F5E17F12DA91426B
:10B7200003DD0028D8BF404203E0002BCCBF184601
:10B73000584208F0F9FA914908F0FEFB064603E08A
:10B74000002601E04FF07E564FF0000903950024DB
:10B75000CDF8089063000493894B33F9140008F086
:10B76000E3FA884908F034FB08F0F8FC08F0DCFA4A
:10B77000854908F02DFB804B824633F9140008F010
:10B78000D3FA7C4B07461B889B077ED0014608F006
:10B7900017FA7E4B804633F9140008F0C5FA0146CB
:10B7A000404608F00DFA08F0D9FC059B5B42984230
:10B7B00003DB059B8342A8BF0346754A0499885E54
:10B7C000099A1B1A32F91400184408F0ADFA8046A1
:10B7D00007F08EFF70B16F4B40466F4914F803902D
:10B7E00008F0AAFB0146484606F0E4FE6A4908F064
:10B7F000EFFA8046287F08F093FA684908F0E8FAE3
:10B800008346287A08F08CFA0146404608F0E0FAB0
:10B81000634908F0DDFA08F0A1FC81460BF1004015
:10B8200008F09CFC814505DB584608F097FC48452C
:10B83000A8BF484608F078FADFF88891029001998D
:10B84000404608F0C5FA59F8241008F0B9F95549EE
:10B850004FEA840B804608F059FC38B940465249FB
:10B8600008F072FC20B1DFF8408101E0DFF834819C
:10B8700049F80B80A87C08F053FA0146404608F0CE
:10B88000A7FA4A4908F0A4FA81463A4BB3F800B047
:10B890001BF0010F40F09880394B049ADFF81C81AF
:10B8A000D35E002BB8BF5B42B3F5206F4FEA840331
:10B8B0000A9303DD002348F824302AE03C49384647
:10B8C00008F086FA039B0B90587808F029FA0B9A37
:10B8D0000146104608F030FB514608F06FF9019917
:10B8E00008F076FA58F8241008F06AF931498046D1
:10B8F00008F00CFC38B940462F4908F025FC20B16F
:10B90000DFF8B48001E0DFF8AC802C4A0A9B42F8F3
:10B910000380039BD87A08F003FA284B53F82410CD
:10B9200008F056FA264908F053FA1BF0020F804639
:10B930004CD03846029908F041F90146304608F0EB
:10B9400047FA0146029808F03BF949460746404647
:10B9500008F034F90146304608F03AFA0146484604
:10B9600008F02EF9804631E083F9223E200F0020B6
:10B97000BD378635EC180020241000200000E1437C
:10B98000440F00200000A03ECDCC4C4014340020D9
:10B990001C2F002088B10108000020410000A040B9
:10B9A0006F12033C0000F0C10000F0410AD7A33D34
:10B9B0000000A043000040C30000404304270020D3
:10B9C0000AD7233CFC260020C846029F8B4B185DFB
:10B9D00008F0AAF90146504608F0FAF9884908F03B
:10B9E000F7F90146384608F0E9F895F85120034682
:10B9F0003AB18449844B01EBC4011B68FCF762F93E
:10BA00000346824F504657F824100A9308F0D6F8A0
:10BA1000019908F091FA47F824A007F1080A5AF8AA
:10BA200024B01037594608F0C9F80146079808F0C5
:10BA3000CFF90146584608F0C3F883464AF8240077
:10BA4000385D08F071F90146584608F0C1F97049AF
:10BA500008F0BEF907460A9B4146184608F0B0F8C0
:10BA6000394608F0ABF80CF0FFF86A4A049B0492E0
:10BA7000D0520A9BDFF8C0B1184608F06FFB4BF8B4
:10BA80002400404608F06AFBDFF8B0A1DFF8B0817F
:10BA90004AF8240007F1004008F060FB039B049A79
:10BAA000013348F82400039317460CB9012451E6EA
:10BAB000089A594B9479B3F90430640028345C43F4
:10BAC000564B6411B3F9040008F02EF94FF07A5187
:10BAD00008F07EF90CF0C8F8201A08F025F9002CBF
:10BAE000B8BF6442322C06464D4C02DD0023A360F1
:10BAF00025E0069808F032FB20F0030008F014F966
:10BB00000190687B08F00CF90146304608F060F9B6
:10BB1000019B81464349184608F00EFA0146484603
:10BB200008F056F908F01AFBA36818443E4B9842F7
:10BB3000A8BF18463D4B9842ACBFA060A360A36865
:10BB40006FF0FF005B13B3F5807FA8BF4FF48073E5
:10BB50009842B8BF184608F0E7F80446304608F0A7
:10BB6000FDFAEB785843801108F0DEF8304B0646BA
:10BB70001B78032B12D9B5F84E90B9F5FA7F0DD288
:10BB800008F0ECFAC9F10003984203DB484503468C
:10BB9000A8BF4B46184608F0C7F8064695F851204E
:10BBA0006AB1530803D09A42A8BF1A4600E00122A6
:10BBB000154B30461F491B68FCF784F806462146A2
:10BBC000304607F0FDFF08F0C9FA80B2B88000B235
:10BBD00008F0AAF80CF048F8B880304608F0BEFA31
:10BBE000CBF80800204608F0B9FA0023CAF808008C
:10BBF000C8F808300DB0BDE8F08F00BF1027002056
:10BC0000A69B443B602900207829002014270020AF
:10BC1000F7CC9238C429002024100020440F0020C3
:10BC20007C29002000803B45FEFFFF0F020000F052
:10BC30005C2A002070290020CC290020D82900206F
:10BC4000E42900202DE9F04F89B00593BE4B002672
:10BC5000B3F90290B3F90030B9F1000FB8BFC9F1E0
:10BC60000009002BB8BF5B429945B8BF9946804692
:10BC7000B2463446B9F5FA7F04910392A8BF4FF457
:10BC8000FA79019000960296B04D2B88990754D00E
:10BC9000AD4B610033F91420AD4B33F9143003EB95
:10BCA0004202039B5B429A4203DB039B9342A8BF81
:10BCB0001346A84A8F5E059ADB1B32F914001F1841
:10BCC00007F016FD90B1A44B384613F804A008F015
:10BCD0002BF8A24908F030F90146504606F06AFCFC
:10BCE0009E4908F075F808F039FA074698F80830C8
:10BCF00064227B4393FBF2F398F81C206FF0040A54
:10BD00000AFB02FA534504DB02EB820A9A45A8BFFC
:10BD10009A4642F21072924B53F8240038449042F3
:10BD2000A8BF10468F4A9042B8BF104643F824007F
:10BD300098F812305843031302932D8805F003033B
:10BD4000012B38D0804B884933F91430A60000937A
:10BD5000019B51F8247093F801E0844B33F91400EF
:10BD600080EAE073A3EBE073B3F5206F16DC009A72
:10BD700050235A4392FBFEF3042290FBF2F0181A70
:10BD80000744B7F57A5F7A4BA8BF4FF47A579F42C2
:10BD9000ACBF41F8247041F8243002E0002341F8A0
:10BDA00024308B597D2693FBF6F6019BDB7A734397
:10BDB000402693FBF6F6AA0712D5009A09FB06F572
:10BDC00009FB02F70298C9F5FA7303FB0A7703FB34
:10BDD00000534FF4FA7297FBF2F193FBF2F505E092
:10BDE000EB0755BF354651460099029D5F4B04272E
:10BDF00033F914305F4A93FBF7F3A25C6FF04F07FF
:10BE0000534393FBF7F398F851204FEA440BCF18B4
:10BE100072B13846069207F087FF5749574B01EB3E
:10BE2000C401069A1B68FBF74DFF08F097F9074617
:10BE30004E4B534A3BF803003BF9021003B25B1A26
:10BE4000042193FBF1F102F1040E5EF824302BF88B
:10BE500002000C3252F8240042F8243098F85020A6
:10BE600018444FEA840C08444EF8241082B1CDF8EF
:10BE70001CC0069207F058FF4249404B01EBC40139
:10BE8000069A1B68FBF71EFF08F068F9DDF81CC076
:10BE90003D4BDFF810E11B5D7A195843202390FBDE
:10BEA000F3F3D21A2BF80E20384A5B424CF80230DA
:10BEB000019B3748374901334CF801504CF800706A
:10BEC000019375460CB90124DEE61F4B0427B3F934
:10BED0000440049B244E9B79D6F808E00F335B00A6
:10BEE0006343224C5B11B4F90440002B94FBF7F739
:10BEF000A3EB0707B8BF5B42322B98F80D400BDC71
:10BF000004FB07E4244BA342A8BF2346234CA342CF
:10BF1000ACBFB360B46001E00023B36098F80340A5
:10BF200004FB07F31E4C9B112478032C3DD9B8F871
:10BF30004E40B4F5FA7F38D26742BB4234DBA342AD
:10BF4000A8BF234631E000BF24100020EC180020D9
:10BF5000143400201C2F002088B10108000020416B
:10BF600028270020F0D8FFFF7C290020440F002064
:10BF700080C1FFFF102700206029002078290020C1
:10BF800030270020AC29002024270020E4290020AD
:10BF9000CC290020D8290020FEFFFF0F020000F06E
:10BFA0005C2A0020C42900203B46B4686FF0FF06DD
:10BFB00044F34F34B4F5807FA8BF4FF48074B4428B
:10BFC000B8BF344683601E190023AE808C60936036
:10BFD00009B0BDE8F08F2DE9F04F87B00393B44B63
:10BFE00081461D88029105F00205ADB2019295B11E
:10BFF000B04BB3F90250B3F90030002DB8BF6D4219
:10C00000002BB8BF5B429D42B8BF1D46B5F5007F0F
:10C01000A8BF4FF40075CB460026A64BA64933F9BE
:10C020001620A64B4FEA460A33F91630520083EA2F
:10C03000E374A4EBE374B4F5206F4FEA860851F87B
:10C04000260011DC042493FBF4F3D31A0344B3F564
:10C050007A5F9B48A8BF4FF47A538342ACBF41F844
:10C06000263041F8260002E0002341F8263051F83E
:10C0700008709BF80B30FF119BF801405F438C4B1D
:10C0800054431B88BF119B074FEAA41456D08D4B15
:10C090003AF903301A44019B5B429A4203DB019B4D
:10C0A0009342A8BF1346884A3AF902209B1A039A82
:10C0B00032F916201A44049207F01AFB049A98B138
:10C0C000824B10469B5D049307F02EFE804907F0DB
:10C0D00033FF049B0146184606F06CFA7C4907F0D2
:10C0E00077FE08F03BF8024642F21070794958F8A2
:10C0F000013013448342A8BF034677488342B8BF48
:10C10000034648F8013099F8081099F81C004A4392
:10C1100000EB8000D21141428A4203DB8242A8BF79
:10C120000246114699F81220641A53431B13FF1A52
:10C130006F436C4303EB672701EB64245F4B0422DE
:10C140003AF9033093FBF2F2644B9B5D534399F849
:10C150005120A4EBA31472B12046049207F0E4FD31
:10C160005F49604B01EBC601049A1B68FBF7AAFD0F
:10C1700007F0F4FF044651495B4B3AF801003AF9E5
:10C1800003E002B2CEEB02024FF0040E92FBFEF28D
:10C190002AF803009E440C3358F80EC058F80300E8
:10C1A00048F80E206044104499F8502048F803C025
:10C1B0008C467AB10591049207F0B6FD4B49494B84
:10C1C00001EBC601049A1B68FBF77CFD07F0C6FF74
:10C1D000DDF814C0464BDFF834E19B5DE2194343C0
:10C1E0005B11D21A2AF80E2042484349434A5B4267
:10C1F00048F8004048F8017048F802300BF1010B94
:10C2000074460EB9012608E72A4B0427B3F90450F7
:10C21000029B294E9B79D6F808E00F335B006B43F5
:10C22000BCF904505B1195FBF7F7002BA3EB070754
:10C23000B8BF5B42322B99F80D500BDC05FB07E5CC
:10C240002F4BAB42A8BF2B462E4DAB42ACBFB360C9
:10C25000B56001E00023B36099F8035005FB07F3D4
:10C26000294D9B112D78032D0CD9B9F84E50B5F5F9
:10C27000FA7F07D26F42BB4203DBAB42A8BF2B461B
:10C2800000E03B46B5686FF0FF0645F34F35B5F566
:10C29000807FA8BF4FF48075B542B8BF3546836034
:10C2A0005E190023A6808D60936007B0BDE8F08F13
:10C2B000EC180020241000207C290020440F0020CE
:10C2C00080C1FFFF143400201C2F002088B101081A
:10C2D0000000204128270020F0D8FFFF1027002071
:10C2E000602900207829002044270020AC29002064
:10C2F00024270020CC290020D8290020E429002070
:10C30000FEFFFF0F020000F05C2A0020C42900207D
:10C310002DE9F04F89B00593AE4B0027B3F90280A9
:10C32000B3F90030B8F1000FB8BFC8F10008002B16
:10C33000B8BF5B429845B8BF98468246B946BB46EF
:10C340003C46B8F5FA7F0492A8BF4FF4FA78029001
:10C350000397A14D2B88990757D0022C55D09D4BA0
:10C36000610033F914209D4B33F9143003EB420282
:10C37000049B5B429A4203DB049B9342A8BF134693
:10C38000974A8E5E059A9B1B32F914001E1807F01F
:10C39000AFF990B1934B304613F804B007F0C4FCEA
:10C3A000914907F0C9FD0146584606F003F98E4948
:10C3B00007F00EFD07F0D2FE06469AF80830642218
:10C3C000734393FBF2F39AF81C206FF0040101FB16
:10C3D00002FB5B4505DB02EB82029342A8BF1346DA
:10C3E0009B4642F21072814B53F824003044904235
:10C3F000A8BF10467E4A9042B8BF104643F82400BA
:10C400009AF81230584303130393298801F0030369
:10C41000012B01D1022C3DD16E4B764D33F9149096
:10C42000029BA00093F801E0734B55F8247033F998
:10C43000146086EAE673A3EBE673B3F5206F1CDCA9
:10C44000022C14D0502303FB09F292FBFEF30422CA
:10C4500096FBF2F69E1B3744B7F57A5F674BA8BF91
:10C460004FF47A579F42ACBF2F502B5007E089EA18
:10C47000E973A3EBE973642BE4DD00232B505D4BE0
:10C480007D27C35893FBF7F7029BDB7A7B4340275A
:10C4900093FBF7F78A0713D5022C11D008FB07F599
:10C4A00008FB09F60398C8F5FA7303FB0B6603FB58
:10C4B00000534FF4FA7296FBF2F193FBF2F508E0A9
:10C4C000CB0704D5022C02D0039D594601E03D461E
:10C4D000494663000193484B042633F91430484A17
:10C4E00093FBF6F3A25C6FF04F06534393FBF6F316
:10C4F0009AF85120CE18E2B1022C069230460BD1A8
:10C5000007F012FC069A530803D09A42A8BF1A46B5
:10C5100000E001223B4905E007F006FC3A49069A93
:10C5200001EBC401394B1B68FBF7CCFB07F016FE8F
:10C530000646314B019A0198D15A354B0AB2C05E7A
:10C540004FEA840C121A042092FBF0F20198C152B7
:10C5500003F10801143351F824E053F8240041F8A2
:10C560002420704410449AF8502043F824E082B10B
:10C57000CDF81CC0069207F0D7FB2649234B01EBF0
:10C58000C401069A1B68FBF79DFB07F0E7FDDDF889
:10C590001CC0214B214A1B5D01995843202390FB6D
:10C5A000F3F073191B1A8B521D4B40424CF8036079
:10C5B0001C4B01344CF803501B4B032C4CF803006C
:10C5C000029B03F1010302937FF4C3AE09B0BDE8FF
:10C5D000F08F00BF24100020EC180020143400203D
:10C5E0001C2F002088B101080000204128270020CE
:10C5F000F0D8FFFF7C290020440F002080C1FFFFFE
:10C6000010270020702900206029002078290020B0
:10C6100058270020AC29002024270020C42900200E
:10C62000CC290020D8290020E429002010B507F0EB
:10C630007BFB0021044607F087FD08B1204601E09E
:10C6400004F10040054907F077FC054907F0C0FBFD
:10C65000FBF71AFE034B186010BD00BF8096184B05
:10C6600035FA8E3C4C000020F8B59C4B04461B6804
:10C67000187818B1012800F06A819AE2242C984DAC
:10C680000CD006D80A2C00F0D9800D2C00F0D680F2
:10C6900048E12A2C06D02C2C04D043E12870687085
:10C6A000A87050E18F4B69782F7800208C4A58543D
:10C6B0002FBB1978D770472921D1597850291ED11D
:10C6C0009978472907D1D978472904D1197941297F
:10C6D00001D10121D1709978824A522903D1D178B0
:10C6E0004D2900F0688299787E4A472907D1D17890
:10C6F000532904D11279562A04BF0322EA70EA783A
:10C70000774E022A39D0032A4CD0012A40F0858086
:10C71000BA1E072A00F28180DFE802F004080F1336
:10C720001A257F2A06F0B8F8686076E01B78532B4C
:10C7300073D16B685B426B606FE006F0ADF8A86088
:10C740006BE01B78572B68D1AB685B42AB6064E051
:10C750001B78302B644B1A788CBF42F0020222F017
:10C7600002021A7059E0002006F0F6F8287354E02F
:10C77000002006F0F1F8E8814FE0072F06D0082FDF
:10C780004BD1012006F0E8F8708246E0012006F067
:10C79000E3F841F2184358434FF47A73B0FBF3F0D7
:10C7A00030823AE0022F07D0032F0AD1002006F092
:10C7B000D3F84E4B187030E0002006F0CDF83075FD
:10C7C0002BE02AD93A1F9210337D0132D2B2013BBD
:10C7D00002EB8303DBB2102B1FD8F91EC2F101025A
:10C7E00001EB8202D2B2012A0BD0042A11D100201F
:10C7F0005E1E06F0B1F83E4B002298553D4B9A550F
:10C8000007E03D4A5E1E0020935506F0A5F83B4B1D
:10C8100098553B4A136801331360314B2A2C18BFDB
:10C820009A7807F101074FF000000CBF0122544035
:10C830002F7068700CBF5A759C7084E0687D00286A
:10C8400048D0304B13F8012D2F495A708B42F9D143
:10C85000244A234C13785278402B85BF373B1B0169
:10C860001B01DBB298BF03F0F003402A8CBF373ABC
:10C87000303AD2B21344AA78DBB29A4227D12123AC
:10C880000B702249E0780B68012803F101031E4A6E
:10C890000B600AD002281CD172231370228A1C4B11
:10C8A0001A80628A1B4B1A8013E0672313700E4BA9
:10C8B0001B789F070ED5184B62681A60A2685A60F1
:10C8C000227B164B1A70E289154B1A8002E03F2337
:10C8D0000B70002000236B7535E000BF6001002065
:10C8E00078270020502F002028180020A00F0020BB
:10C8F000D10F0020C10F0020A10F0020B10F002098
:10C90000C82E0020000A0020EC090020D42E0020B0
:10C910002A180020880F0020301800202E18002030
:10C920002C1800206B78687D0E2B9FBFA54A591CE0
:10C930005170A54A98BFD454A24A18B993785C4064
:10C94000947000E00020003018BF0120F8BD9D4B1E
:10C950000022997D082900F22C81DFE801F0050B07
:10C960000F15202B475D6700B52C40F02281DA754A
:10C97000012239E0622C08BF022235E003229A75B9
:10C980001C765C769C7614E104229A755A7E997E18
:10C990002244D2B25A760A449A76DC7609E105221C
:10C9A0009A755A7E997E2244D2B25A760A449A7671
:10C9B0009C83FEE006229A755A7E997E2244D2B26A
:10C9C0005A760A449A769A8B02EB0424A4B2B4F500
:10C9D000AC7F82BF7B4A0121D17500229C83DA8320
:10C9E000002C40F0E68007229A75E2E05A7E997E9C
:10C9F0002244D2B25A760A449A76DA8BB2F5AC7FE8
:10CA00003EBF7049891881F820400132998B92B25B
:10CA10009142DA83E7D9CCE008229A755B7EA34283
:10CA200000F0C780674B0122DA750DE0674D9A75FB
:10CA300015F8012D6A70664A9542F9D1997E614ACE
:10CA4000A14206D03F232B70624A536801335360E2
:10CA5000AFE06148016801310160D07D10B13E2333
:10CA60002B70A6E021212970D17E062941D004D85F
:10CA7000022907D0032923D0F8BD122959D0302923
:10CA800067D0F8BD5021546A297054494C60946AAB
:10CA90000C60116B4FF47A7491FBF4F1504C2180CF
:10CAA00092F878114F4A19B1117841F0020102E071
:10CAB000117821F002011170012283F8792169E0D7
:10CAC0005321297092F82510CE0705D592F824201D
:10CAD000D51E6A426A4100E0024602F0010183F875
:10CAE0007811002A56D13F490A7822F002020A70D2
:10CAF00050E04F21297092F82B10CC0705D592F801
:10CB00002A20D11E4A424A4100E0024602F00101B9
:10CB100083F8781122B933490A7822F002020A70A8
:10CB200093F84F10304A1170B3F84C102F4A11800F
:10CB300030E05621546B29702D490C8042F210745C
:10CB4000916B91FBF4F12B4C2180012182F87A1139
:10CB500020E04921297092F82410274A102988BF23
:10CB600010211170254914780022A2420ED20E7AAB
:10CB7000234D56554E7A234D5655CE7A224D565555
:10CB800011F80C6F214D56550132EEE720490A6825
:10CB900001320A6093F879310A4A002B3AD092F8B0
:10CBA0007A31BBB3002182F8791182F87A111846E4
:10CBB000F8BD0020F8BD1279432A7FF494AD02221B
:10CBC000EA7090E578270020502F0020000A00200E
:10CBD000EC09002040010020D42E00203018002055
:10CBE0002C180020281800202E18002056000020A5
:10CBF0002A180020880F0020A00F0020982700206E
:10CC0000A10F0020B10F0020C10F0020D10F002084
:10CC1000C82E0020F8BD0449044B09680022187092
:10CC20005A6199611A777047482F0020400100200F
:10CC3000F8B5101A0D461F4607F076F80446781B23
:10CC400007F072F8174B079E196807F0C1F82146E4
:10CC50000546204607F0BCF829460746284607F057
:10CC6000B7F80146384606F0ABFF0BF061FA0E4903
:10CC700007F0AEF807F098FA069B2946186004F111
:10CC800000400BF0C9F8094907F0A2F8084906F07E
:10CC900097FF07F063FA0028BCBF00F50C40A030F6
:10CCA0003060F8BD4C0000202C7D8E3FA00CB345B9
:10CCB00000A00C4644F25063984203DDA0F50C40FE
:10CCC000A0387047034B9842BCBF00F50C40A03021
:10CCD000704700BFB0B9FFFFF7B50368174C184D98
:10CCE00023600B68174E63600068FFF79FFC95E8B0
:10CCF0000300154B0196009394E80C00FFF798FF92
:10CD00003668124B60681E606B68114FC01A07F0DE
:10CD10000BF8104B196807F05BF807F01FFA2A6848
:10CD2000236878609B1A3B600B4B1E600B4B1B68A3
:10CD3000DA880B4B1A8003B0F0BD00BFAC2D002089
:10CD400030180020B82D0020B42D0020F42D002034
:10CD5000BC2D00204C000020EC2D0020580E00209F
:10CD6000E82D002070B50446407906F0D9FF1E4931
:10CD700007F0E2F81D4D1E4E2860E07B06F0D0FF64
:10CD8000194907F0D9F8EE606860A07906F0C8FF8D
:10CD9000184907F0D1F8184D2860207C06F0C0FF34
:10CDA000114907F0C9F86860A07E06F0B9FF134981
:10CDB00007F0C2F8EE60A860E07906F0B1FF0D4917
:10CDC00007F0BAF80E4D2860607C06F0A9FF06490E
:10CDD00007F0B2F86860E07E06F0A2FF074907F0AE
:10CDE000ABF8EE60A86070BD0000C842C42D002002
:10CDF0000000FA4400002041D42D002000007A44B5
:10CE0000F82D002010B50C4C23789B0713D50B4B45
:10CE10001B78042B0FD90A4A0A4B10685268186015
:10CE20005A60FFF703FC084B1A88084B1A802378D6
:10CE300043F00103237010BD281800202E18002095
:10CE4000301800208C0F00201C100020082E00201D
:10CE5000164B13B51B681B0325D5154B154C1B78BA
:10CE600015498DF80030154B20681B788DF801307E
:10CE700006F0AEFF07F098F911498DF802006068DE
:10CE800006F0A6FF07F090F98DF80300A06807F000
:10CE90008BF90C4B8DF804001B780A2069468DF83D
:10CEA0000530FBF739FF02B010BD00BF242F002072
:10CEB000162F0020382F002000002041342F0020A2
:10CEC00000007A441A2F0020054A137883F00103EA
:10CED0001370044A00231360034A1360B8E700BFCD
:10CEE0001A2F0020302F00202C2F0020094A137801
:10CEF00018441346C0B210F0800F18BF803810706D
:10CF0000054A19781378994201BF00231370014A2A
:10CF1000137070470D2E00200C2E002010B50A4B08
:10CF20000A4A1B7842609C18094A046012789A42A7
:10CF300025BFD31A0B60C3F1800300232EBF4B60C3
:10CF40000B604A6010BD00BF0D2E00200E2E002089
:10CF50000C2E00201FB5684602A9FFF7DFFF044B27
:10CF600002981B6803440398184405B05DF804FB5D
:10CF7000500D00202DE9F04F89B001930023824627
:10CF8000994602910392039A934205DA029A52F863
:10CF9000232001339144F6E7019B4D46002B56D1E7
:10CFA00000F0D8FB002852D101987DE00222404ECB
:10CFB0008DF81C201A0C4FF480578DF81D20062088
:10CFC0001A0A8DF81E208DF81F3000F0E7FB7761FC
:10CFD000062005F0ADFA374B01223761D0461A70B2
:10CFE00077612646002007A9042205F06BFA029F0C
:10CFF0004FF0000B039B9B451EDABC4657F8042BF1
:10D000004FEA8B03002A48D0B24236D332465AF850
:10D0100003100020CDF814C0049305F053FA049BCC
:10D02000DDF814C05AF8032032444AF80320DCF833
:10D0300000309E1BCCF800601D4B4FF480521A61EB
:10D040001D4A2D1B13681C44019B146053B34DB340
:10D05000194B1B68DCB22A19B2F5807F174A88BFCA
:10D06000C4F58074D26898BF2C4693429ED3144A6C
:10D0700000231370134A137014E00020D8F8001036
:10D0800005F020FA57F8043CD8F80020F61A1344AB
:10D09000C8F80030002347F8043C0BF1010B08F1FD
:10D0A0000408A7E7C5EB090009B0BDE8F08F00BF91
:10D0B000000C01404D0D0020500D002018000020F4
:10D0C0000C2E00200D2E002030B50B4C0B4D22787D
:10D0D0002B7885B09A420CD0684602A9FFF71EFF54
:10D0E0000123684602A90222FFF744FF00232B70A8
:10D0F000237005B030BD00BF0D2E00200C2E002087
:10D1000030B50E4D0E4C2A78237885B09A4211D056
:10D11000684602A9FFF702FF002302A9022268461F
:10D12000FFF728FFFFF7E2FE20782B781B1A584202
:10D13000584100E0012005B030BD00BF0D2E002099
:10D140000C2E002038B50E4C4FF4805545F20820C7
:10D1500000F024FB6561062005F0EAF9094B012285
:10D160002561C7201A70656105F0E2F9064A0023BF
:10D1700025611370054A1370054A136038BD00BF5E
:10D18000000C01404D0D00200C2E00200D2E002023
:10D19000500D002001480249FDF7A0BC00080040E6
:10D1A000D82A002001480249FDF798BC000400403D
:10D1B000B02A00204FF080400149FDF78FBC00BF2E
:10D1C000882A002001480249FDF788BC002C014054
:10D1D000602A002001480249FDF780BC002C014074
:10D1E000602A002037B5044603211E2006226B4624
:10D1F00004F020F978BB9DF801309DF80000174D30
:10D2000043EA002000B206F08FFD296806F0E0FD39
:10D2100006F0A4FF9DF8033020809DF8020043EA49
:10D22000002000B206F080FDA96806F0D1FD06F0EE
:10D2300095FF9DF80530A0809DF8040043EA00208A
:10D2400000B206F071FD696806F0C2FD06F086FFC7
:10D250006080012000E0002003B030BD38000020D5
:10D2600010B5054C2368186902F050FC18B123680A
:10D270001A69024B5A6110BDD81F002000040140FA
:10D2800038B50D4B0D4D99680D4B1A681C465288E8
:10D29000114203D001F058FD286007E001F054FD71
:10D2A0002B68984282BFC01A064B186023685A68E0
:10D2B000054B5A6138BD00BF000C0140F428002026
:10D2C0003C0100200000002000040140084A1368CF
:10D2D0009B020BD5074B002119704FF6FE730649D0
:10D2E000086803400B604FF400135360704700BFA1
:10D2F00000000240183400206C0002402DE9F04785
:10D30000664D6B686649581C0A788E4602F0FF0627
:10D310000AB10346F6E737466B60687CEB6895F820
:10D320001080AA7C39B2202900F09C80DFF880C1EF
:10D330000CEB8103DC789B783CF82110C3F1FF03F0
:10D340009BB2002B65D04FF03C0CB1FBFCF9C3F154
:10D35000FF0363431B12B9F1050F5DD8DFE809F045
:10D36000030B1A293A4AE01A4143B1FBFCF0DAB246
:10D370001044C0B251E0B1FBFCF00CFB101189B2BB
:10D38000DAB2C1F13C01E31A4B43B3FBFCFC20468B
:10D3900094442CE0B1FBFCF00CFB1011E21A89B2B2
:10D3A0004A43B2FBFCF25FFA83F84244D2B2204611
:10D3B00032E0B1FBFCF90CFB191189B2E01AC1F1A2
:10D3C0003C014843B0FBFCF05FFA83F84044C0B234
:10D3D000224621E0B1FBFCF80CFB1811D8B289B24F
:10D3E000E31A01FB03F2B2FBFCFC224684445FFA21
:10D3F0008CF412E0B1FBFCF80CFB181189B2D8B226
:10D40000C1F13C01E31A4B43B3FBFCF20244D2B23C
:10D4100003E02246204600E044464FEA042C4CEA52
:10D42000004C4CEA020C17234FF0010808FA03F8ED
:10D4300006F1170118EA0C0FA1EB0301DFF8748065
:10D4400014BF4FF011094FF0090989B213F1FF33EE
:10D4500008F80190E8D218360137B6B2BFB2114BC6
:10D46000A0465FE7EB6001238EF8003040F22A33DC
:10D47000AA740D4A69810D4985F8108068742E815F
:10D48000536000238B840B889BB243F001030B8015
:10D49000136843F001031360BDE8F087F42800200F
:10D4A00018340020042900206C00024000040040D1
:10D4B000E2070020010A002001F0030301F0FC0153
:10D4C00001F1804101F5803110B59B008C680F227D
:10D4D0009A4024EA02028A608A68984002438A607D
:10D4E00010BDF0B5B1F800E000234EFA03F2D50705
:10D4F00025D58E784FEAD30CF40648BFCC7806F0D9
:10D500000F0203F0070748BF2243BF0050F82C501A
:10D510000F24BC4025EA0404BA402243282E40F8D8
:10D520002C2005D1C46801229A4024EA020205E0B9
:10D53000482E04D1C46801229A402243C2600133BC
:10D54000102BD2D1F0BD2DE9F0437A4A87B0136891
:10D55000904693B11A681AB17749886902438A6183
:10D560009A889868ADF8002002228DF80320694659
:10D5700004228DF80220FFF7B4FF322001F00BFCEB
:10D58000002111221E2003F095FF012160221E20A0
:10D5900003F090FF642001F0FEFB002402A8FFF7D7
:10D5A00021FE274626460A25022101221E2003F0DD
:10D5B00081FF322001F0EFFB02A8FFF713FEBDF957
:10D5C0000820BDF90A1014448A42A8BF0A46BDF9D2
:10D5D0000C300F4493421E44A8BF134613F5805FDE
:10D5E00009DD564A013DD36883F01003D360DBD1D7
:10D5F0004FF0010901E04FF000091E200021122226
:10D6000003F058FF0A25022101221E2003F052FFD9
:10D61000322001F0C0FB02A8FFF7E4FDBDF90820AD
:10D62000BDF90A10A41A8A42A8BF0A46BDF90C30F7
:10D630007F1A9342A6EB0306A8BF134613F5805F3B
:10D6400007DD3E4A013DD36883F01003D360DAD191
:10D6500001E04FF00009204606F066FB014638481D
:10D6600006F06AFC374D20F000402860384606F08E
:10D670005BFB0146324806F05FFC20F0004068602A
:10D68000304606F051FB01462F4806F055FC20F0CD
:10D690000040A860002170221E2003F00BFF012132
:10D6A00020221E2003F006FF1E200221002203F08C
:10D6B00001FF642001F06FFBB9F1000F04D14FF0BE
:10D6C0007E532B606B60AB60D8F80030194E1A7B2C
:10D6D00062B31A7D52B3184900258A69012442F0C9
:10D6E00001028A61187B197DFFF7E6FE174801F0F9
:10D6F00017FC3368164A1B6904A8536104930C2372
:10D700008DF815308DF814508DF8164002F0CEF9D2
:10D71000336801A85B7D8DF806508DF80430032333
:10D720008DF805308DF8074004F0AEFE07B0BDE877
:10D73000F08300BFD81F002000100240000C014001
:10D7400000406F463800002001C05E4661D20008EC
:10D75000000401400F4B73B518781C4698B105239F
:10D760000D4D8DF800304FF4805600238DF80130B8
:10D7700001A86E616946022204F0A4FE2E619DF8A4
:10D78000050000F0010000F00100207080F00100B1
:10D7900002B070BD4D0D0020000C0140064B70B56D
:10D7A00006461C461D68FFF7D5FF18B923685B1BAA
:10D7B000B342F8D970BD00BF482F0020F7B503234E
:10D7C0008DF80430030C8DF805308DF80700030A3E
:10D7D00006200F4614468DF80630FFF7DFFF78B1BC
:10D7E000084D4FF4805601A904226E61002004F018
:10D7F00069FE38460021224604F064FE20462E6170
:10D8000003B0F0BD000C0140024640213C2003F073
:10D8100051BE70B500EB8000094CA0F1A1059C3809
:10D8200025440444074B15F8010F1E787040FFF79C
:10D83000EBFFA542F6D13046BDE87040E4E700BFFB
:10D840008CAA01081D34002010B5441E14F8010FE5
:10D8500010B1FFF7DEFFF9E710BD024680213C2042
:10D8600003F028BE10B5D420FFF7F7FF8020FFF7A4
:10D87000F4FFA820FFF7F1FF3F20FFF7EEFFD320D2
:10D88000FFF7EBFF0020FFF7E8FF4020FFF7E5FF81
:10D890008D20FFF7E2FF1420FFF7DFFFA120FFF745
:10D8A000DCFFC820FFF7D9FFDA20FFF7D6FF1220F0
:10D8B000FFF7D3FF8120FFF7D0FFCF20FFF7CDFF89
:10D8C000D920FFF7CAFFF120FFF7C7FFDB20FFF7E2
:10D8D000C4FF4020FFF7C1FFA420FFF7BEFFA62032
:10D8E000FFF7BBFFAF20FFF7B8FFA620FFF7B5FF9C
:10D8F000AE20FFF7B2FF2020FFF7AFFF0020FFF7B9
:10D90000ACFFB020FFF7A9FF4020FFF7A6FF0020E3
:10D91000FFF7A3FF1020FFF7A0FF4FF48064013C46
:10D920000020A4B2FFF770FF002CF8D18120FFF790
:10D9300094FFC820FFF791FFAF20FFF78EFF012073
:10D9400010BD08B55038C0B2FFF787FF0020FFF7C1
:10D9500084FFBDE8084010207FE710B50446503929
:10D96000C8B2FFF77AFF04EB4400400000F00E005D
:10D97000FFF773FF06206043BDE81040C0F30310BB
:10D9800010306AE7012828BF01202DE9F04F064634
:10D99000734F142000FB0671724BD1F8A4421E761F
:10D9A0005C61714BD1F8B422DD69B1F8AC822A43D5
:10D9B000DA61A288B1F8AEA222F44072D1F8A8527E
:10D9C000120489B0120C4AEA0809A28003A9C5F81A
:10D9D000109002228DF80E0028460193ADF80C90AD
:10D9E0008DF80F20FFF77DFD019B00971F464FF03C
:10D9F000080BAA6818EA020F03D10A2001F0C0F947
:10DA0000F7E70A20C5F8148001F0BAF9C5F81080CC
:10DA10000A2001F0B5F9BBF1010BEAD1C5F814A059
:10DA20000A2001F0ADF9C5F814800A2001F0A8F928
:10DA3000C5F810800A2001F0A3F90222C5F810A051
:10DA4000284603A98DF80F201C228DF80E20ADF872
:10DA50000C90FFF746FD454A03A894423A690BBF74
:10DA600042F4001242F480023A613A610BBF3A6913
:10DA70003A6922F4001222F480023A61A38823F466
:10DA800040731B041B0CA38023889BB243F001034B
:10DA90002380A58801F09CFE0599354B25F03F05B4
:10DAA000B1FBF3F32D042D0C1D43ADB2A5802288EC
:10DAB000002522F001021204120C22802D4A03A834
:10DAC000B1FBF2F100298AB208BF012242F4004101
:10DAD0004FF4967253434FF47A7293FBF2F301338F
:10DAE0009BB22384A1832388009A9BB243F0010355
:10DAF0002380238823F4816323F002031B041B0C7F
:10DB000023804FF480432381142303FB062696F8D9
:10DB1000B13201248DF80C308DF80D508DF80E5077
:10DB20008DF80F4004F0B0FC96F8B0329DF80F204D
:10DB30008DF80C308DF80D508DF80E501AB103A8E9
:10DB400004F0A2FC08E05A0903F01F039C4002F114
:10DB50002003094A42F8234009B0BDE8F08F00BF16
:10DB60008CAA0108F4280020001002400054004054
:10DB700040420F00804F120000E100E038B5002461
:10DB80000B4D6059254404F0A9FA696811B10948A0
:10DB9000FAF7D8FAA96811B10748FAF7D3FA074893
:10DBA000103404F09BFAB4F5F07FE9D138BD00BF22
:10DBB00058AD010876C901087CC90108C3D4010821
:10DBC00070B50546284609F086FE064658B91A4B38
:10DBD0001A485A791A4BBDE8704003EB8203D3F818
:10DBE000DC11FAF7AFBA28461649324609F07CFE36
:10DBF00060B9154804F072FA144C54F8041F19B1B6
:10DC00001348FAF79FFAF8E7124805E00024124B90
:10DC100053F8241021B91148BDE8704004F05EBAF1
:10DC20002846324609F060FE01340028EFD1024B4D
:10DC30000B4D5C71C6E700BF2C10002082C90108A3
:10DC400058AD01088EC9010893C9010834AF010815
:10DC5000A6C90108C3D4010838AF01085EC801088D
:10DC6000A8C50108F0B585B0044609F034FE0828BF
:10DC700026D1621EE01D1F4912F8013F09681944B0
:10DC8000497801F00301022908BF203B824213704A
:10DC9000F1D1254604F1080715F8016B1648314605
:10DCA00009F00BFE20B12846314609F006FE10B1FE
:10DCB000F9F7D6F91CE0BD42EED12046FCF74AF94F
:10DCC0000E4804F00BFA00230D4A04A91A4492F8F6
:10DCD0008A210A440849595C0133082B02F80C1CBC
:10DCE000F2D10023074801A98DF80C30FAF72AFA7F
:10DCF00005B0F0BD680000202EDF0108AAC90108A8
:10DD00002C10002067D301082A4B2B4C1E6880B5CD
:10DD10002068F9F7CBFE3046F9F7C8FE2068417954
:10DD20008D0703D441F0020101F00CF9234B0822C6
:10DD30001A61234D10221A612B689A0341BF0623F2
:10DD40006371E37923F0010344BF43F00203E371FD
:10DD5000206801F003F990B1184F08237B61164B3E
:10DD6000186801F0F8F88046FEF77EFC08B102F072
:10DD70005DFA3046414601F0F4F808233B61304635
:10DD800001F0ECF878B10D4F4FF01008C7F814808F
:10DD90003046D4F8009001F0DEF80146484601F024
:10DDA000E0F8C7F810802B689B03D1D503F003FC83
:10DDB000CEE700BFF82E002010290020000C014003
:10DDC000242F00202DE9F047054609F084FD2F4E51
:10DDD0000446D6F8088090B92D4804F07FF92D4B01
:10DDE00053F8241049B10123A34013EA080F02D0CD
:10DDF0002948FAF7A7F90134F1E7284822E0284634
:10DE00002749224609F070FD58B9264804F066F902
:10DE1000254C54F8041F0029EFD01F48FAF792F957
:10DE2000F7E72B784FF000092D2B03BF013504F1E4
:10DE3000FF344FF0010A4FF0000A164B53F82970D7
:10DE400027B91A48BDE8F04704F048B928463946D2
:10DE5000224609F049FDA8B9012000FA09F0BAF1FB
:10DE6000000F03D0FAF702FB114803E040EA080074
:10DE7000B060104804F032F93946BDE8F0470E486A
:10DE8000FAF760B909F10109D7E700BF2C100020AB
:10DE9000B0C90108A0AF0108A6C90108C3D4010890
:10DEA0008EC90108BAC901089CAF01085EC8010803
:10DEB000C6C90108CFC9010866D3010810B50848D2
:10DEC00004F00CF9074B00241C741C64064B1C70F6
:10DED00001F0EAF904F0A6FA044B1C6010BD00BF83
:10DEE000D7C90108102900201E340020F82E002078
:10DEF00070B5064600240B4BE518AA8816420AD0D6
:10DF0000E1580948FAF71EF92846002104F077F88D
:10DF1000064804F0E3F840F6BC4314349C42EAD1CE
:10DF200070BD00BF3CB4010803CA0108C3D4010896
:10DF300008B50848FAF706F9FFF704F9FFF70AFCF5
:10DF400018B9642000F027FFF8E70348BDE808404F
:10DF5000FAF7F8B80DCA01081ACA01082DE9FF41FD
:10DF60000A48068885684488B0F80480C768FEF7C8
:10DF7000F1FFCDF800800290019731462A462346F2
:10DF80000348FAF7DFF804B0BDE8F081180000207C
:10DF900022CA0108F0B504788BB005460CB1002404
:10DFA00036E04B4B19680E2303FB0411B1F91D51E8
:10DFB000B1F91921B1F91B31009591F8205101F502
:10DFC0008C70019591F8215101F59071029590F9AD
:10DFD0000700039091F902103E4804912146013454
:10DFE000FAF7B0F8082CDCD170E02D2B14D1072CF7
:10DFF0001BDC284609F0C4FC0AAB661C03EB440496
:10E0000024F8100C15F8013F303B092BFAD934469F
:10E010002B78002BE9D104E0A3F13002092A09D8BA
:10E02000E5E7082CBDF8182009D00BB0BDE8F0409A
:10E03000F9F716B8202BF8D101352646E7E7072A6D
:10E04000F3D840F2DC55BDF81A00214BA0F2EE21C6
:10E0500089B2A9421B68E8D8BDF81C10A1F2EE24D1
:10E06000A4B2AC42E1D8BDF81E6004B237B2A742F8
:10E07000DBDB0DB2AF42D8DCA542D6DBBDF82470A5
:10E0800007F16404A4B2C82CCFD8BDF826E00FFA7B
:10E090008EF4112CC9DCBDF82050B42DC5D8BDF8C4
:10E0A0002240B42CC1D812B24FF00E0C0CFB02333C
:10E0B000A3F81901A3F81B11A3F81D6183F82051DF
:10E0C00083F8214183F81F7183F822E10BB0F0BD82
:10E0D0005C0F00207FCA0108F0B504468FB02046CF
:10E0E00009F0F9FBC5B21DBBAB4803F0F7FFAB4C21
:10E0F00094F8D61009B9AA4853E049B294F8D4204C
:10E1000094F8D530009194F8D710A648019194F96D
:10E11000D8100734029194F9D210039194F8D310D7
:10E12000049129460135FAF70DF8102DE0D1E2E708
:10E1300020469D49052209F0D7FB0546B8B9294676
:10E140009A48702209F083FB2846994B19680E23E0
:10E1500003FB001301300022082883F8232183F8F1
:10E16000242183F8252183F82621F0D112E12046CD
:10E170009049042209F0B8FB05462046002D4AD1FB
:10E18000202109F09AFB002800F00481461C30464B
:10E1900009F0A1FB2C460746874B53F824502DB9B4
:10E1A00086480FB0BDE8F040F9F7CCBF30462946AD
:10E1B000FAB209F099FB01340028EDD1774A1646EE
:10E1C00002F17001002382F8DA3082F8D63082F84A
:10E1D000D53082F8D43007328A42F3D1784901EB46
:10E1E000C40191F8A022934210DAD1F8A472C3EBD3
:10E1F000C302B0183A44176800F1D401C0F8D470D3
:10E2000090880133888092798A71E7E729466D48C2
:10E21000F9F798FF8FE06C49072209F065FB054686
:10E220002046002D49D1202109F047FB064609F080
:10E2300052FBC4B26CBB6548F9F784FF21466448C1
:10E240000134F9F77FFF0E2CF8D15548F9F77AFF22
:10E25000002460482146F9F775FF0025544A012340
:10E2600011680E2202FB0412D2F82321AB401342A4
:10E27000594B5A495A4808BF19460135F9F762FF08
:10E280000E2DEBD146480134F9F75CFF082CE0D1A4
:10E2900080E03046534909F077FB2C4600284CD0EB
:10E2A000022C4FD009F06CFB06AB43F824004D491B
:10E2B000002009F069FB0134F0E74A4909F064FBEA
:10E2C000002460B1082C38D009F05AFB06AB43F8A3
:10E2D00024004449002009F057FB0134F1E7082CE1
:10E2E0002BD1069B0F2B28D8DDF81CE0BEF1070FC1
:10E2F00023D8089F0D2F20D8099E06F16402C82A52
:10E300001BD80A9DFF2D18D80B98642815D80C9996
:10E31000642912D8884210DA0D9C032C0DD8324A99
:10E32000C3EBC303134483F804E05F719E71DD7196
:10E33000187259729C722D4CD1E60FB0BDE8F040B6
:10E34000F8F78EBE069B072B20D807990D291DD8FC
:10E350000278722A0DD06E2A18D1154A0E20126842
:10E3600000FB032301228A40D3F8231121EA020291
:10E3700009E00F4A0E20126800FB032301228A40A5
:10E38000D3F823110A43C3F8232101E0F8F768FE0C
:10E390000D4CA4E60FB0F0BDA7CA01082C10002058
:10E3A000C3D40108D2CA01082EC8010800110020F8
:10E3B0005C0F002059C8010838AF01085EC8010889
:10E3C00058AD01086DC801089FCA010880C901083D
:10E3D000EECA0108A7D20108F8D701083ED7010804
:10E3E000F3CA0108F7CA0108FC100020A8C50108FB
:10E3F0002DE9F743047805468CB9324D95F8B312F0
:10E40000B5F8B02295F8B2322F4800912146013478
:10E41000F9F798FE102C05F10405EFD14EE009F054
:10E42000AFFA0F28044636DC2846202109F045FAC9
:10E43000264EE4B2D6F84480451CA40000272846A6
:10E4400009F09EFA5FFA87F9B9F1010F83B208D09B
:10E45000B9F1020F0BD0B3F5B47F24D2726C135311
:10E460000AE0FF2B1FD8736C2344987004E0FF2B45
:10E4700019D8736C2344D87028462C2109F01DFA52
:10E48000054608B1013502E0B9F1020F0BD10137A1
:10E49000032FD4D112E00E4800210F2203B0BDE8B3
:10E4A000F043F8F75ABD08EB04000021042209F0FC
:10E4B000CEF903B0BDE8F043F8F7D2BD03B0BDE834
:10E4C000F08300BF2C100020F9CA01081029002099
:10E4D000ECC701082DE9F04FAC498BB0044609F0B8
:10E4E000BFF9AB49002820460CBF0125072509F0DC
:10E4F000B7F9A8490028204608BF022509F0B0F95D
:10E50000002808BF0425E90740F1E780A24803F08E
:10E51000E5FD002003F0ECFBA04CA14803F0DEFD7C
:10E52000A04803F0DBFD62799F4BA04803EB820318
:10E53000D3F8DC11F9F706FE9D48F9F703FE2646ED
:10E540000027D6F814800021404605F0D5FD20B103
:10E550009848F9F7F7FD002669E039469648D6F85D
:10E5600018B0D6F81CA0D6F82090F9F7EBFD40467D
:10E57000002105F0CBFD10B1202003F0A7FD06A976
:10E580004046F9F765FC01468C48F9F7DBFD584633
:10E59000002105F0BBFD10B1202003F097FD06A976
:10E5A0005846F9F755FC01468448F9F7CBFD50462B
:10E5B000002105F0ABFD10B1202003F087FD06A976
:10E5C0005046F9F745FC01467C48F9F7BBFD484643
:10E5D000002105F09BFD10B1202003F077FD06A976
:10E5E0004846F9F735FC013701467548F9F7AAFDA9
:10E5F0000C2F06F11006A4D1AAE749B294F8D42052
:10E6000094F8D530009194F8D7106E48019194F9A0
:10E61000D8100734029194F9D210039194F8D310D2
:10E62000049131460136F9F78DFD102E03D094F890
:10E63000D6100029E1D1644803F050FD574B634CDC
:10E640009F6854F8041F19B16148F9F77BFDF8E79A
:10E650000E46604B53F826404CB10123B3403B4279
:10E6600003D05D482146F9F76DFD0136F1E75B48BF
:10E6700003F034FD2146494B0AAA0B4493F88A3132
:10E680001344574A8A5C0131082903F8102CF2D14F
:10E69000002306A953488DF82030F9F753FD52485E
:10E6A00003F01CFD5148F9F705F8514803F016FD39
:10E6B0004E48F8F7DBFC4F4803F010FD4B48FFF7DE
:10E6C00097FE4D48F9F73EFD4020FFF711FC4B48FF
:10E6D00003F004FD4548F9F78FF8AA0739D54848F3
:10E6E00003F0FCFC474803F0F9FC404803F040FB12
:10E6F000454803F0F3FC3D48F8F73CFC434803F081
:10E70000EDFC3A48F8F728FF4148F9F71BFD374878
:10E71000F8F7B8FD3F4803F0E1FC3448FFF73AFC56
:10E7200000260E27774300243B4A0123926CA34026
:10E730003A44D2F80A2013421ED101340E2CF3D1F0
:10E740000136082EEDD12C48F9F7FCFC8020FFF7AC
:10E75000CFFB6B0716D5314803F0C0FC304803F0FF
:10E76000BDFC224803F0DEFA2348F9F7EBFC4FF436
:10E770008070FFF7BDFB05E0314622462948F9F7D6
:10E78000E1FCDAE70BB0BDE8F08F00BF0DCB01086C
:10E7900085CF010814CB01081ACB01082C100020EA
:10E7A00028CB01083ACB010858AD010846CB010837
:10E7B00051CB01085ECB01086BCB01087FC9010872
:10E7C00067D3010883CB010873CB01089CAF010814
:10E7D000A2CB0108A0AF0108B0CB0108BDCB010856
:10E7E0002EDF0108C9CB0108D2CB0108A8C501085A
:10E7F000E1CB0108EDCB0108C3D40108FBCB010834
:10E8000008CC01081BCC010829CC010833CC010835
:10E8100042CC010850CC0108102900205CCC010832
:10E820006DCC01087FCC0108034B4FF4805208B136
:10E830001A6170475A61704700080140034B4FF45A
:10E84000805208B15A6170471A6170470008014050
:10E850002DE9F04F89B00593A04B80461B880492A8
:10E86000980737D540F2E632129B9D48DC89B0F913
:10E8700000301B1B03F2F315954203D8002BB8BFE1
:10E880005B4201E04FF4FA73B0F9022040F2E63047
:10E89000121B02F2F314844203D8002AB8BF52427A
:10E8A00001E04FF4FA729342B8BF13460522C3F554
:10E8B000FA7393FBF2F30A22643B534398F81C204B
:10E8C000D2105343642293FBF2F3134423EAE3731D
:10E8D000DBB200E06423C1460193CB1C0393002408
:10E8E000039B022C13F8016F7E4F03934FEA440AF7
:10E8F00005D1B7F904301B365E4376114AE07A4BF6
:10E9000037F9142033F9143003EB4202049B5B42C5
:10E910009A4203DB049B9342A8BF1346734A32F921
:10E920000A50059A5B1B32F9145003EB050B04F0F7
:10E93000DFFE88B16E4A5846155D05F0F5F96D4960
:10E9400005F0FAFA0146284603F034FE694905F05D
:10E950003FFA05F003FC8346604A1288D10714D4BD
:10E9600037F90A501B366E4393074FEA261611D526
:10E9700098F812509DF9042005FB0BF353436422D1
:10E9800093FBF2F306EB231604E098F8085005FB1E
:10E990000BF52E11584B042533F90A30574F93FBD2
:10E9A000F5F5751B99F80160E35D6E435E430293D4
:10E9B000642396FBF3F698F851B0F611BBF1000F03
:10E9C0001BD0022C30460CD105F0AEF95FEA5B0398
:10E9D00004D05B45A8BF5B461A4600E001224849C7
:10E9E00005E005F0A1F95A46391D01EBC401FB69A8
:10E9F000F9F768F905F0B2FB0646424B99F80B703F
:10EA000019883E4B01FB05F203F1200E5EF824004D
:10EA1000D21207FB02073C4AB7F5001FA8BF4FF40C
:10EA20000017974203F12C00B8BF174650F8242076
:10EA300040F824504FF6FF700909B0FBF1F1AA1A13
:10EA40004A4303F1380103F144054EF8247051F8AC
:10EA500024E055F8240045F824E098F8505092112D
:10EA600070444FEA840C7F13104441F824208DB188
:10EA7000CDF818C0079305F057F9079B2A4603F114
:10EA8000500101EBC401DB69F9F71CF905F066FBE5
:10EA9000DDF818C099F81530F2195843029B01347B
:10EAA00043431846642390FBF3F0184B00120244D2
:10EAB00023F80A2003F108024CF80260032C03F14A
:10EAC000140203F120034CF802704CF8030009F122
:10EAD00001097FF405AF09B0BDE8F08FEC18002004
:10EAE000602F002024100020143400201C2F002050
:10EAF00088B1010800002041440F00205C2900205B
:10EB000070290020200F00200000E0FFC429002011
:10EB100010B5084B0022196801EBC20393F90240BB
:10EB2000844201D1981C10BD0132052AF4D1002085
:10EB300010BD00BFE02B002038B1438811EA03006C
:10EB400003D08B420CBF01200220704730B50B4B25
:10EB50000B491C6891F89420042A0BD81346551CC5
:10EB600004EBC303EAB29D882842F5D081F89420D3
:10EB7000981C30BD81F89420002030BDE02B00208F
:10EB80005C290020024B002283F89420DEE700BFBE
:10EB90005C2900202DE9F047877890F803C0BBB2CC
:10EBA000C7F1640E03EB83065C42C3F178001C4D91
:10EBB0005FFA8EFE7600CCF16408A4B280B2A3B2F4
:10EBC0000FFA83F9B9F1000F04DC002B14BF3B46A8
:10EBD000012300E0734609FB09F25B4302FB0CF2E0
:10EBE00092FBF3F3434403FB09F30A2293FBF2F392
:10EBF00033449BB225F8023FB1F800904A880A34AA
:10EC0000C9EB020A1AB202FB0AF24FF47A7392FBC2
:10EC1000F3F3A4B24B4484422B80D0D1BDE8F087FB
:10EC2000F029002010B544780078002240F6C41185
:10EC300002FB02F3193B634303F6C41353434343FC
:10EC400093FBF1F3034921F812300132072AEDD189
:10EC500010BD00BF0A2A0020104B043033F9100009
:10EC6000B0F5617F05DB40F633039842A8BF184634
:10EC700001E04FF461700A7819235A4302F283329B
:10EC8000824208DA4A78534303F283338342B4BFA3
:10EC90000020012070470020704700BF602F002037
:10ECA00010B500F1500302788A4203D18478C2780B
:10ECB000944204D304309842F5D1002010BD0120C5
:10ECC00010BD0B4B1B6813F4805F0A4BB3F9063081
:10ECD00005D0C089421A934207DD084400E0008A4B
:10ECE0008342B4BF0020012070470120704700BF5D
:10ECF000242F0020602F00201FB5084B1B681B032A
:10ED000009D58DF80400039101230D2001A98DF888
:10ED10000530FAF701F805B05DF804FB242F002058
:10ED20001FB5084B1B681B0309D58DF80400029121
:10ED300000230D2001A98DF80530F9F7EDFF05B08E
:10ED40005DF804FB242F002010B50A4A0A4B116815
:10ED50009B6800BF12689142F7D1084A4FF47A705D
:10ED6000D2F8BC4000FB04F2D31AB3FBF4F300FB6F
:10ED7000013010BD482F002010E000E05C29002089
:10ED800038B50446FFF7E0FF0546FFF7DDFF401BFF
:10ED9000A042FAD338BD10B504462CB14FF47A70B6
:10EDA000FFF7EEFF013CF8E710BD024A136801339C
:10EDB00013607047482F002010B50024044B53F80F
:10EDC000243003B198470134032CF7D110BD00BFA4
:10EDD000A41F0020014B1B68184700BFFC33002014
:10EDE00010B50020FFF7F6FF074B00241C7004F05D
:10EDF0005BFC064B83F8C040C3F8C440A3F8C8408E
:10EE0000C3F8CC4010BD00BFC03300205C290020F7
:10EE100010B510B9BDE81040E2E700230C225A43B8
:10EE20000C4C1119125D824203D00133102BF5D125
:10EE300010BD094BD3F8CC0018B14A784078824213
:10EE400006D20022C3F8CC10A3F8C820C3F8C4200F
:10EE500010BD00BF9CB201085C29002010B5400025
:10EE60001428A8BF14200023074A022199540B44F8
:10EE700099181424834201F8014CF5DBFF21D15489
:10EE80000F20BDE81040C3E7FC2E00202DE9F84319
:10EE900081460B26013E37D01E4B10225A610822B4
:10EEA0001A6109F101074FF032080525194C0120BC
:10EEB000E36883F01003E360E36883F00803E36032
:10EEC000FFF788FF4046FFF766FFE368002083F006
:10EED0001003E360E36883F00803E360FFF77AFF61
:10EEE0004046FFF758FF45B1013DDFD14FF4FA70BE
:10EEF000FFF751FF4FF0FA08D8E7013FD6D14FF4A2
:10EF00007A70FFF748FFC5E7034A044BDA60BDE8B3
:10EF1000F88300BF000C01400400FA0500ED00E09A
:10EF2000074B1A6832B15A681AB19A682AB9022294
:10EF300000E0012243F8220070470020A6E700BF4E
:10EF4000A41F002003685B69184703681B69184702
:10EF50000368DB68184703689B68184703685B68A9
:10EF6000184703681B681847B0F902302DE9F74FBE
:10EF700093421CBF0023037090F800A004460E4685
:10EF80009146BAF1000F40F0AB80104604F0CCFE81
:10EF9000864904F01DFF864904F01AFF4FF07C51AA
:10EFA00004F016FF08F0C0FE0146054604F010FF0D
:10EFB00080498346284604F00BFF0346584619460D
:10EFC000019304F0FDFD4FF07E5104F0F9FD014680
:10EFD0004FF07E5004F0B0FF2946804604F0F8FE62
:10EFE000294604F0F5FE07460146606004F0E8FD9E
:10EFF000E7604FF07E572946A0602761284604F05D
:10F00000DFFD294604F0E4FE4FF0804104F0D6FD18
:10F010000146404604F0DCFE019B606119465846FB
:10F0200004F0CCFD394604F0CBFD0146404604F027
:10F03000CFFE40F2DC53A0462746554663651023B9
:10F04000A4F852301823A061A4F850304FF0974133
:10F05000D8F8100004F0BCFE0021824605F056F8F6
:10F0600028B150464FF07C5104F0A8FD04E0504612
:10F070004FF07C5104F0A4FD05F0D2F8C7E90E0171
:10F080004FF09741D8F8040004F0A2FE0021824618
:10F0900005F03CF828B150464FF07C5104F08EFD4D
:10F0A00004E050464FF07C5104F08AFD05F0B8F8BA
:10F0B0000135032DC7E9080108F1040807F1080725
:10F0C000C4D1A6F2DC531B042367E3676367C4F86B
:10F0D0008030A367C4F884300123A4F80290237021
:10F0E000D4F85490B4F95280C9EB0606636A06FA64
:10F0F00008F67343276A4FEAE67B206F07FB0B3362
:10F100002667A7FB0667E26F1F44636CD4F840C014
:10F1100053434FEAE27B0CFB0B3ED4F88010C4F85B
:10F120008020ACFB02237344B61A67EB0307E36A43
:10F13000A26A43434FEAE07B02FB0B3EA2FB0023A3
:10F140007344B6185F41E36C656F4B436067A06C16
:10F150004FEAE17B00FB0B33C4F88410A0FB0101F4
:10F160001944636B361A05FB03F3206B4FEAE57B0A
:10F1700000FB0B3367EB0107A0FB05018019194465
:10F180007941B4F95020A56704F006FD08F1FF327B
:10F1900001239340E067C01841EBE371424604F05D
:10F1A000FBFC484403B0BDE8F08F00BF6F12833A08
:10F1B000DB0F4940F404B53F2DE9F8430024254B0B
:10F1C000E0B293F80061B0420DD203EB8003224A13
:10F1D000D3F8D03032F810101BB10B2801D8DB68FF
:10F1E00098470134EBE71D4B1B685B032FD50024C8
:10F1F0002346E2B2B2422AD2DFF858904FEA84089E
:10F2000009F1D00757F8242055689D4217D02846A9
:10F21000FBF726FDEFF31283502282F31288282198
:10F22000AA8C01FB009092B20132C0F82821AA8A70
:10F23000DBB292B242F00102AA8283F3118857F83E
:10F24000083000221B6801341A802B46D1E7BDE844
:10F25000F88300BF5C290020600F0020242F0020CD
:10F2600008B50E4B1B6813F4805F0D4B14BFD3F829
:10F27000A421D3F8A82193F8001192880023D8B2D2
:10F28000884204D2074820F813200133F7E7FFF73C
:10F2900093FFBDE8084032207DE500BF242F002009
:10F2A0005C290020600F00200A4B30B51A680A4B19
:10F2B00002F48052D3F8A441D3F8A85100230AB134
:10F2C000A18800E0A988054820F8131001330C2B11
:10F2D000F5D130BD242F00205C290020DE2E002037
:10F2E00070B5124D0024214605F2AD10702285F84C
:10F2F000AC4108F0ACFA2146D5F820320B4A0B4459
:10F3000093F9020088B11E6802F2AD140E5108197B
:10F310009C88073184809B797029837192F8AC3185
:10F3200003F1010382F8AC31E6D170BD5C29002005
:10F33000094B1A680E2303FB0020437AFF2B07D0EA
:10F34000064A12789A4203D9054A32F8130000E0BF
:10F35000808800B2704700BF58290020201F00207D
:10F36000602F00202DE9F041254C0646D4F82402F8
:10F37000D4F82882014604F02BFD4146074640465A
:10F3800004F026FD0146384604F01AFCD4F82C524D
:10F3900007462946284604F01BFD0146384604F07E
:10F3A0000FFC08F0C5FE0146284604F0C5FD1549CE
:10F3B000054604F0B5FEF8B9284608F0DDFCD4F89F
:10F3C000301204F005FD08F04FFCB0F5617FA8BFD6
:10F3D0004FF4617004F0A8FC0B4904F0ADFDF8F7A0
:10F3E000E0FE0446304604F09FFC214604F0F0FCA9
:10F3F00008F03AFC80B200E0002000B2BDE8F081E5
:10F400005C2900208FC2753CEFB6B0442DE9F84F5F
:10F410002F4E0446D6F834723846F8F735FF0546C5
:10F420003846F8F7BEFED6F8386280463046F8F720
:10F430002BFF83463046F8F7B4FED4F80490064616
:10F440002946484604F0C4FCA7688246414638462F
:10F4500004F0BEFC0146504604F0B0FB2168824631
:10F46000584604F0B5FC41460446484604F0B0FC5A
:10F47000314604F0ADFC0146204604F0A1FB3146C4
:10F480000446384604F0A4FC294604F0A1FC0146D9
:10F49000204604F095FB0146504608F0BDFC0D499E
:10F4A00004F096FC0C4904F047FD0C4B196804F07D
:10F4B00087FB0B4904F040FD08F0D6FB83B21A0429
:10F4C00044BF00F5B47083B218B2BDE8F88F00BF36
:10F4D0005C2900200000E144DB0F4940E41F0020CC
:10F4E0000000204101380A4B042804D8DFE800F06E
:10F4F0000507090B0D00074A08E0074A06E0074A1E
:10F5000004E0074A02E0074A00E0074A1A60704731
:10F510005C00002011C3000851E8000815370108FD
:10F52000D7BF000845BC000899B60008084BDA6848
:10F53000D10709D4DA68520708D4DB6813F0100F3A
:10F5400014BF032004207047012070470220704739
:10F550000020024003788B4286BF024B33F8110033
:10F5600000207047982B002070B50546FFF7ECFB94
:10F57000324CA369A061C31AB3F5FA5FE36182BF9D
:10F58000002384F8203084F8213094F820302BB9FF
:10F59000A12D02BF294A012182F8211094F82110DF
:10F5A000264A31B1D118EDB2013381F8225082F8E8
:10F5B000203094F8205094F84330AB423CD11F4B9C
:10F5C00093F84430052B02D0062B03D02FE0002007
:10F5D00003F0BCFF94F823301E2B28D100200246F4
:10F5E000C1B26B1E99421ADA214491F822300821E7
:10F5F000DBB283EA0206F60744BF83F01803C3F3C5
:10F60000460301F1FF3154BF5B0843F0800311F062
:10F61000FF01C2F34702ECD101301A46E0E7234470
:10F6200093F822309A4202D1032003F08FFF002387
:10F6300084F8213084F8203070BD00BF982B002062
:10F64000174AF0B5164692F84530D2F848E0042B38
:10F6500010D85C1C0EEBC3039D1CE4B208D09A8842
:10F66000D10705D5104203D008E00131052907D1A3
:10F670002346ECE786F845300020F0BD9F78002156
:10F680000C2202FB01F3064D05F14C0C1CF8032083
:10F690009742EAD12B4485F84540186DF0BD00BF74
:10F6A000982B00208A6810B50C6A036814430A6915
:10F6B00023F4FF4314434A6923F0700314438A6917
:10F6C0001443CA6914434A6A14438A6A224313439F
:10F6D0000360CB6843600B6883604B68C36010BDF8
:10F6E0004FF6FE730268134003600023036043601B
:10F6F0008360C360284B984201D1284A27E0284BF9
:10F70000984201D1254A2AE0264B984201D1234A4A
:10F710002DE0254B984201D1204A30E0234B9842FE
:10F7200001D11E4A33E0224B984204D11B4A536850
:10F7300043F470032EE01F4B984204D1174A5368DC
:10F7400043F0706326E01C4B984204D11B4A536877
:10F7500043F00F031EE01A4B984204D1174A536836
:10F7600043F0F00316E0174B984204D1134A536854
:10F7700043F470630EE0144B984204D10F4A53686F
:10F7800043F4704306E0114B984204D10B4A53688E
:10F7900043F47023536070470800024000000240A9
:10F7A0001C00024030000240440002405800024069
:10F7B0006C00024080000240080402400004024045
:10F7C0001C04024030040240440402405804024039
:10F7D0001F4A10B5536803F00C03042B03D0082B09
:10F7E00004D01C4B14E01C4B1B6811E0536851689B
:10F7F000C3F38343C90303F1020301D4174906E0AD
:10F80000516811F4003F1449096818BF49084B4377
:10F81000036053681249C3F30313CC5C0368E340ED
:10F8200043605468C4F302240C5D23FA04F484603A
:10F830005468C4F3C2240C5DE340C3605268C2F351
:10F8400081320A44127CB3FBF2F3036110BD00BFA6
:10F850000010024000127A004400002000093D0020
:10F860008AB1010810B50446FFF760FE012806D1F1
:10F870001CB1FFF75BFE013CF8E7052010BD002C32
:10F8800008BF052010BD0A88F0B54B888E88B1F8F6
:10F8900008E0CC88002A3AD1028C43F0010322F020
:10F8A00001021204120C0284058B078CADB225F004
:10F8B000F30545EA0E1189B241EA06027A49BFB260
:10F8C000884212D001F5006188420ED0B0F1804F1D
:10F8D0000BD0A1F59831884207D001F580618842AC
:10F8E00003D001F58061884202D127F0020701E0D0
:10F8F00027F00A071F4302830784038B23F00C03BE
:10F900001B041B0C0383038B9BB21C4344E0042A9F
:10F9100044D1028C22F010021204120C0284018BDA
:10F92000058C21F440721205120D42EA0E325E4936
:10F9300092B242EA06228842ADB292B212D001F5EA
:10F94000006188420ED0B0F1804F0BD0A1F5983104
:10F95000884207D001F58061884203D001F58061BB
:10F96000884207D125F0200141EA03139BB243F0FE
:10F97000100304E025F0A00143F010030B430283C1
:10F980000384038B23F440631B041B0C0383038B4E
:10F990009BB243EA0424A4B20483F0BD082A028C7B
:10F9A0003ED122F480721204120C0284828B3E4DEE
:10F9B00092B222F0F307018C47EA0E1292B2A842EB
:10F9C00089B242EA060212D005F50065A8420ED0BF
:10F9D000B0F1804F0BD0A5F59835A84207D005F5BA
:10F9E0008065A84203D005F58065A84207D121F4BF
:10F9F000007141EA03239BB243F4807304E021F4D5
:10FA0000206143F480730B4382830384838B23F050
:10FA10000C031B041B0C8383838B9BB21C4341E0B0
:10FA200022F480521204120C0284858B018C25F47E
:10FA300040752D052D0D45EA062545EA0E321A4D75
:10FA400089B2A84292B212D005F50065A8420ED044
:10FA5000B0F1804F0BD0A5F59835A84207D005F539
:10FA60008065A84203D005F58065A84207D121F43E
:10FA7000005141EA03339BB243F4805305E047F65B
:10FA8000FF5543F480530D402B4382830384838BC3
:10FA900023F440631B041B0C8383838B9BB243EAD8
:10FAA0000424A4B28483F0BD002C0140016830B569
:10FAB000CD43154B1C682C401C605A682A405A6084
:10FAC000027902F1804202F582321468214311600A
:10FAD00002689C68D5432C409C60D9682940D96055
:10FAE0004179102909BF996801F180431143996058
:10FAF00015BF03F58233D96819680A4316BF0A4354
:10FB0000DA601A6030BD00BF00040140054B1A687E
:10FB10005B69034004D0104214BF012000207047ED
:10FB20001846704700040140CA78F0B5D40648BFB3
:10FB30008C780D8802F00F0348BF234315F0FF0FA8
:10FB40001DD0016800240126A64006EA0507B74239
:10FB500011D14FEA840E0F2606FA0EF621EA0601AD
:10FB6000282A03FA0EF641EA060101D1476102E0B4
:10FB7000482A08BF07610134082CE4D10160FF2D39
:10FB80001FD94168002404F108070126BE4006EA97
:10FB90000507B74211D14FEA840E0F2606FA0EF67A
:10FBA00021EA0601282A03FA0EF641EA060101D1EC
:10FBB000476102E0482A08BF07610134082CE2D1FE
:10FBC0004160F0BD0F4B1A6842F001021A6059689B
:10FBD0000D4A0A405A601A6822F0847222F4803278
:10FBE0001A601A6822F480221A605A6822F4FE020F
:10FBF0005A604FF41F029A60044B4FF000629A6003
:10FC0000704700BF001002400000FFF800ED00E068
:10FC10002DE9F8435B4C0368013AC4F888308388C7
:10FC20000D46A4F88C30072A42D8DFE802F0040A17
:10FC3000101822292F35B4F888300B80B4F88A3098
:10FC400013E0B4F88A300B80B4F8883005E0B4F8DB
:10FC500088305B420B80B4F88A305B4205E0B4F830
:10FC60008A305B420B80B4F888306B80B4F88C30FB
:10FC70001DE0B4F888305B420B80B4F88A3012E0A3
:10FC8000B4F88A300B80B4F888300CE0B4F88830CF
:10FC90000B80B4F88A3005E0B4F88A305B420B8000
:10FCA000B4F888305B426B80B4F88C305B42AB8038
:10FCB000354B1B79002B62D1B5F9000004F034F804
:10FCC0008046B5F9020004F02FF80746B5F90400A4
:10FCD00004F02AF8D4F890100646404604F078F86C
:10FCE000D4F89C108146384604F072F80146484624
:10FCF00003F066FFD4F8A8108146304604F068F897
:10FD00000146484603F05CFF07F0AEFFD4F89410BC
:10FD10002880404604F05CF8D4F8A01081463846AC
:10FD200004F056F80146484603F04AFFD4F8AC10F8
:10FD30008146304604F04CF80146484603F040FF47
:10FD400007F092FFD4F898106880404604F040F81D
:10FD5000D4F8A4108046384604F03AF801464046EC
:10FD600003F02EFFD4F8B0100746304604F030F808
:10FD70000146384603F024FF07F076FFA880BDE86F
:10FD8000F88300BF982B002044000020F8B5494BB1
:10FD9000494C1B68D4F8B4209A1A002AC0F2888013
:10FDA00003F5C333A033C4F8B430444B04F1B800B6
:10FDB0005B689847424B04F1B8001A780146FFF798
:10FDC00027FF404B04F1B80519781A4611F0040FCB
:10FDD00014D0D4F8B430C4F8C03000233A48002618
:10FDE0001844A0F87661EE5A38481E5206301E526A
:10FDF0000233062BF2D121F00401117094F8D020C7
:10FE00002D4BAAB13049B3F8B820B1F87601121AD7
:10FE1000A3F8B820B1F87801B3F8BA20B1F87A1194
:10FE2000121AA3F8BA20B3F8BC20521AA3F8BC20C7
:10FE3000D4F8C010204A00293AD0D2F8B43002F1E8
:10FE4000C4045B1A224902F1CA008B421BD8214A22
:10FE5000D36883F00803D360002335F8132034F906
:10FE6000137016B2B742C8BF184F4FEA4301C8BF5C
:10FE700027F81320475E0133B742BCBF164E8A53A2
:10FE8000032BEAD1F8BD00231449C2F8C03034F97D
:10FE9000135030F9132001332A44022592FBF5F266
:10FEA000032B21F8022FF2D1BDE8F840F8F78ABD04
:10FEB000F8BD00BF00340020982B0020DC1F00207C
:10FEC0001C340020281800202C1000205C2C00205E
:10FED0007FC3C901000C0140622C0020A01100204A
:10FEE00038B50F4B1B689C890E4B186880F31000C7
:10FEF000201A03F019FF0C4903F06AFF054620465B
:10FF000003F012FF0146284604F016F804F026F923
:10FF10006428A8BF642020EAE070C0B238BD00BFEA
:10FF200010180020201800200000C84244F6FB7181
:10FF3000084B1A68137803EB431300FB0313507844
:10FF4000C0EB0030B3FBF0F39078B3FBF0F080B27D
:10FF5000704700BF1018002008B50A480A2290F820
:10FF6000D23000EB4303B3F8E210F03089B220F84E
:10FF7000061CFEF7F9FF80B2FFF7D8FF024B18808E
:10FF800008BD00BF982B002014180020F8B53F4C86
:10FF90000646B4F87831322B11D1D4F87C311A8866
:10FFA000A4F880215A889B88A4F88221A4F884317F
:10FFB0000388A4F886314388A4F8883101E0002B37
:10FFC00040D0D4F87C710023B4F878212F4D322A28
:10FFD0002F4A04BF002142F823104FEA830E05F593
:10FFE000CC7030F913C052F80E10614442F80E1074
:10FFF000002220F8132027F813200133032B114689
:020000040801F1
:10000000E2D1B5F87831012B17D10C2085F89E216B
:1000100085F89F31FEF7FCFED5F87C31B5F88021DC
:100020001A80B5F882215A80B5F884219A80B5F8F3
:1000300086313380B5F888317380B4F87831013B6C
:10004000A4F8783194F8A031104AEBB1D2F88C3191
:10005000322493FBF4F3D2F87C01002182F8A01142
:100060000380D2F8903193FBF4F34380D2F89431BB
:10007000084A93FBF4F312889B1A838031807180C5
:10008000BDE8F840F8F79EBCF8BD00BF982B0020F3
:10009000242D00202800002010B54B88DC0641BF2D
:1000A0002F4B14791B6853F8244044BF2D4B43F861
:1000B00020404B889B0641BF294B54791B6853F85D
:1000C000244044BF274B43F820404B881C070ED5E3
:1000D000254B0C781B78B3EB141FA1BF204BD478B1
:1000E0001B6853F82440A4BF1E4B43F820404B88A4
:1000F0009B070ED51D4B0C781B78B3EB141FDFBF8D
:10010000174B54781B6853F82440DCBF154B43F859
:1001100020404B88DC070FD5154C0B78247803F072
:100120000F03A342DFBF0E4B14781B6853F8244023
:10013000DCBF0C4B43F820404B885B070FD50B7896
:100140000C4903F00F0309788B42A1BF044B92784E
:100150001B6853F82220A4BF024B43F8202010BD97
:1001600054290020E2070020FB260020F926002069
:10017000F8260020FA260020254A0023F0B515684D
:100180001C461A462348244903700B702E197688A2
:100190004EB92F5D3FB9037000230A704B7007788A
:1001A0001C461A460CE0360548BF013204F104042F
:1001B00003F1010348BFD2B2802CDBB2E6D1EAE7FB
:1001C000E0B2B8420CD215F82400013406099E4270
:1001D00000F00F00A8BF731C9042A8BF421CEFE7BD
:1001E0008A704B70C2F3470102F001020A444C1EB0
:1001F0000A490B480A70C3F3470203F00103134492
:1002000004700849501E084A08701370F0BD00BF02
:10021000F0180020F0260020402D0020FA260020B3
:10022000F8260020FB260020F9260020924B2DE91D
:10023000F04FDA68914D1A612A6891B0DA60904AFD
:100240000295136843F0200313608E4B1A78012A3D
:100250000CBF002201221A708B4B1A78910740F1D3
:100260004D838A490978042940F2488388490978EE
:1002700001F0040101F0FF0011B922F001021A702F
:100280001B78DB0702D408B1FCF7BCFD8149CA78B2
:10029000531C052293FBF2F202EB82029A1A7E4B68
:1002A000CA701F7892000023DFF81082DFF81092E6
:1002B00058F82310794C91FBF9FE04F1080040F83E
:1002C00023E0774844F8231000FB0E1142F210702F
:1002D00091FBF0F004F1100680B226F813004FF005
:1002E000140C04F114060CFB036C04F13C0A5AF8DC
:1002F00023605CF802504CF80210761B314405264E
:100300004AF8231091FBF6F109FB0E114434012F3A
:1003100044F823104FEA830B444605D10238B0F568
:10032000797F98BF4BF808100BB90123BCE7594EF1
:10033000029BB2461868336DC01A03F0F1FC5949AC
:1003400003F0FAFD029B4FF07E511B6807463365B0
:1003500003F0DCFE08B94FF07E574B4BCAF85470DF
:100360001B78514E13F00103504D12D00DAA00928C
:100370004F4B0EAA01920CCB94E80300FCF758FCFB
:100380000D9A6421B2FBF1F20E9B328093FBF1F3E4
:1003900000E033802B809AF858303E4D002B35D04A
:1003A000696D4FF07E5003F0C7FD0746EB6D206886
:1003B000C01A03F0B9FC394603F00AFD03F0CEFE83
:1003C0002B6E86B2606836B2C01A03F0ADFC394BB2
:1003D000196803F0FDFC394603F0FAFC03F0BEFE99
:1003E000B5F9662000B28118B5F964200220B3186F
:1003F00091FBF0F193FBF0F389B29BB2A5F86A1080
:10040000A5F86830A5F86610A5F8643001238AF8CD
:100410005830294B61681B88206803F030031D4E5B
:10042000264DCAF86010CAF85C00002B00F0668206
:1004300006F17403009306F178030193F26E336FB3
:10044000FCF7F6FB6B68306FC01A03F06DFC194BBC
:10045000196803F0BDFC03F081FEF36E2A68C6F84C
:1004600080009B1AF3670C4B1B78012B2AD0022BC0
:1004700000F0E68042E200BF40010020482F00204B
:10048000241800208A0F0020281800202E18002091
:1004900019340020402D0020540E0020442D00204F
:1004A000806967FF00007A44A2180020A418002089
:1004B0008C0F00204C000020EC1800203018002089
:1004C00080969800D6F88430D6F8A0400293D6F8EB
:1004D000943004F100400393D6F89830776D05937B
:1004E00003F03CFE8146204603F038FED6F89C30EF
:1004F000BB4C0493BB4B06901B684FF0000B07935B
:10050000B94E4FEA4B0356F82B80A6F11402404631
:1005100032F81B50089303F007FC029903F058FCD3
:1005200003F01CFE401B1FFA80FA283626F81BA099
:100530000FFA8AFA504603F0F7FB039903F048FCE0
:1005400003F00CFE86B20AEB080003F0EDFB059900
:1005500003F03EFC394603F03BFC216803F030FB1E
:1005600003F0FCFD484504DB069B9842A8BF1846F3
:1005700000E0484603F0D8FB206003F0EFFD079B46
:10058000304486B2987803F0CBFB984903F020FC06
:1005900001464FF07E5003F0CFFC394603F010FBCC
:1005A0000146384603F0C8FC09906068D4F808A0FA
:1005B000C0EB080003F0B8FB394603F0BDFC514620
:1005C00003F0FCFA099A0146104603F001FC0146CB
:1005D000504603F0F5FA3135ADB2622D0146206187
:1005E000C4F80480A0600ED9049803F0F1FB03F076
:1005F000B5FD7F4AB0F5FA6FA8BF4FF4FA6090429C
:10060000B8BF104600E0002040F6B832064436B2CB
:100610009642A8BF1646774A089B9642B8BF164630
:10062000754A54F8140B9E52142202FB0BF27349C4
:100630005050BBF1000F40F061814FF0010B5FE7BC
:10064000684BB6F8A8401F68736F3D8902935B083A
:100650009D4228BF1D4623B29D4202DC1FFA85F948
:100660000AE06749706D03F0B3FB03F077FD2044A7
:100670001FFA80F9A6F8A890DAF87860DAF8AC40AA
:10068000341B2046FCF716FB41F293130028D8BF19
:1006900040429842CCBF0020012078B3204603F0AE
:1006A00043FB584903F094FBF7F77BFD044602989F
:1006B00003F036FB0146204603F08AFB03F04EFDB3
:1006C00040F6B83380B2AAF8B00000B29842A8BF92
:1006D0001846484B9842ACBF3018F01848F6A04373
:1006E000984203DDA0F50C40A03804E00028BCBF10
:1006F00000F50C40A030CAF8B40001E0CAF8B460BC
:10070000DAF8B4300026C3F50C502830039303F018
:100710000BFB3C4903F05CFB0446F7F7B5FD0F907B
:100720002046F7F73EFDDAF8B830DAF8C440059312
:10073000DAF8BC300E9004F10040089303F00EFD8F
:100740000490204603F00AFDDAF8C030DAF854804D
:100750002A4C09900793730048460A9303F0E4FA81
:100760000EAB53F8261003F033FBDFF8A0A00546CC
:100770003AF9160003F0D8FA0146284603F01EFAAB
:1007800003F0ECFC05B2204BB5F57A7FA8BF4FF41F
:100790007A759D42B8BF1D460AF13C0AA8B22AF8F4
:1007A000160000B203F0C0FA0599824603F010FB70
:1007B00003F0D4FC089983B25046069303F008FB7B
:1007C000414603F005FB216803F0FAF903F0C6FC8B
:1007D000049B98421CDB099B9842A8BF184618E06E
:1007E000900E0020580E0020BC2D0020DB0FC940C9
:1007F00030F8FFFF48F4FFFF620E0020B80E002023
:100800000000C842D302373918FCFFFFA82D002092
:10081000049803F089FA20608346B87803F080FAE0
:10082000384903F0D5FA01464FF07E5003F084FBBF
:10083000414603F0C5F90146404603F07DFB0B90AD
:100840006068D4F808A0281A03F06EFA414603F055
:1008500073FB514603F0B2F9DDF82CC00146604647
:1008600003F0B6FA0146504603F0AAF96560014666
:100870002061A060079803F0ABFA03F06FFC069BC1
:100880001434034458469A4603F068FC40F6B832E4
:10089000504400B29042A8BF10461B4A0A9B9042A7
:1008A000B8BF1046194A1A4998521422724342F8A6
:1008B00001B00EB901264EE73B792BB1039A6423B0
:1008C00092FBF3F3134A13803B88029A124C9A422C
:1008D0000DD9D4F8AC30A06FC01AFCF7EBF942F296
:1008E000107380EAE072A2EBE0729A4206DD0B4BD5
:1008F00001221A70B4F8C820064B1A8011B0BDE866
:10090000F08F00BFDB0FC94048F4FFFF620E0020EC
:10091000900E0020500E0020402D0020540E00208C
:100920000846F8F707B910B50D4C2068FEF77AF9BC
:1009300020680022047A02FB02F3193B634303F6AA
:10094000C4135343192193FBF1F3064921F81230E4
:100950000132072AEFD1BDE810400349FEF71AB96A
:10096000840F0020E00E0020701100200E4B1A783A
:10097000692A16D140F2E4725988914211D11A794C
:10098000BE2A0ED193F8E1270020EF2A0BD113F8ED
:10099000012B5040054A9342F9D1B0FA80F040094A
:1009A000704700207047704700F80108E4FF010815
:1009B0002DE9F74FEA4C002140F2E472204606F0A0
:1009C00046FFE84B04F53C721A60E74B00221A70B0
:1009D000E64B04F2BA711960692323700323637133
:1009E0004FF48173A3604FF41673A4F86631FA23B1
:1009F000A4F86831BC23A4F864314FF4FA73A4F866
:100A00006E31012384F8623184F87E3184F88631B6
:100A1000052384F82F3240F2DC53A4F8983140F2D9
:100A20004C43A4F89A3140F26C73A4F89C3140F224
:100A30007533A4F89E3140F64303A4F8A031234651
:100A4000202184F86A116E2184F87C110A2184F82F
:100A50007D112B2184F87F11212184F8801123211D
:100A600084F881114FF4C871A4F88211032ACCBF15
:100A70000121002102F1010283F8A21114BF1E21FD
:100A80007521122A83F8A31103F10203EED140F27B
:100A90007E41A4F8441140F23A71A4F8461140F2A4
:100AA0007E51A4F84C1140F2EA5140F2DC50A4F817
:100AB0004E1140F2B4514FF4FA63A4F8C831A4F8CF
:100AC000CC31A4F8D031A4F8D431052384F8E23134
:100AD000C82301264FF47A774FF0320BA4F8E631A1
:100AE000DFF880924FF4C8734FF01E0A1922A4F861
:100AF000EA31A4F84A01A4F85011A4F8C671A4F888
:100B0000CA71A4F8CE71A4F8D27184F8E46184F8B3
:100B1000E56184F8E861A4F84871A4F852B184F85A
:100B200095A184F8E32100920190A4F8543184F84F
:100B3000E16184F8EE61A4F856B184F8F161F9F747
:100B4000DDF9D9F80030009A00254FF00F0E267419
:100B5000E673A573A58183F805E0DA714FF0220EE4
:100B60002122172183F806E05A744FF00E0E53220B
:100B70005975997583F810E0DA7655210A224FF0FD
:100B8000350E4FF02808D97083F81AE02D214FF068
:100B90005A0E9A7400924FF0780C642283F80BA0DE
:100BA00083F80CA0597383F808E01A771D7083F856
:100BB000018083F80280DD7583F804B09D731D7693
:100BC000DD735D7683F8098083F80AC019754FF4E8
:100BD000FA71A3F84E103C2183F85110112183F8CB
:100BE00050106349DFF8A8C19963D9636149C3F81C
:100BF0002CC099626049C3F830C0DFF898C15963CE
:100C00004FF07F5A5D490198C3F820A0C3F824A093
:100C1000C3F848C04FF0000A4FF04B0C59649E7760
:100C200083F85250C3F840A083F84CC084F8BAE768
:100C3000A4F8C4074FF0410E042084F8BBE784F801
:100C4000BCB784F8BD5784F8C15784F8C25784F8FC
:100C5000BE5784F8BF5784F8C05783F85C00A3F8E8
:100C60005850A3F85A50A3F856501966152183F826
:100C7000681043494348D966434983F8648019673B
:100C8000424983F86580596783F87860F9F762F91B
:100C9000D9F80030009A18464FF4487183F8115182
:100CA00083F8125183F8138183F8146183F8185183
:100CB000A3F8161184F8D821C82284F8D921642217
:100CC000A4F8DA7184F8DC51A4F8DE210E2202FBCC
:100CD00005326FF0170482F81941032482F81A4193
:100CE0006FF02F0482F81B41072482F81C416FF03B
:100CF000230482F81D41052482F81E4101355A243F
:100D000080F8204180F821416422FF24082D80F8DA
:100D10001F2180F822414FF0000100F10E00D5D1D3
:100D2000C820A3F88A01142083F88C01A3F890212D
:100D30001E204FF4967283F88D01A3F892210120B2
:100D4000282283F8891183F88E01A3F894210B4699
:100D5000034D5A191033C02BC2F814A01CE000BF79
:100D60002C1000205C0F0020DC2E0020840F0020BF
:100D70008FC2F53C000060406666663F0000A04000
:100D80009A99193FB7D10108F6287C3F3D0A773F71
:100D9000CDCCCC3E00004040DAD105F52C700021CE
:100DA000402206F054FD0023264EEA1899590433D8
:100DB0000868382B244CC2F8B002F5D104F50C7049
:100DC0000021802206F043FD06F13801702204F56F
:100DD0000C7006F031FDFFF7CFF9D9F80060002361
:100DE0000125314604F591604FF4CC7284F8E03768
:100DF00084F8DE5784F8DF5706F01EFD04F5C46062
:100E000031464FF4CC7206F017FD104B1B681A6880
:100E1000C4F8C6275A68C4F8CA279A68C4F8CE2707
:100E20001A68C4F8D2275A68C4F8D6279A680223E9
:100E3000C4F8DA2784F8DC5484F8743603B0BDE8CB
:100E4000F08F00BFA0B101082C100020840F0020FB
:100E5000074B93F8E037012B08D1064A064BD068C0
:100E60001B68834234BF0020012070470020704778
:100E70002C10002018000020500D002038B5094B20
:100E800093F8E05765B9084C2068F6F733FE074B36
:100E900025601B78022B03D1BDE83840F8F7EFBF7F
:100EA00038BD00BF2C100020703000206D300020B5
:100EB000064B93F8E0371BB1012B05D1FCF720B9A5
:100EC000034B1868FEF741B8002070472C10002033
:100ED00070300020F8B5011F06460023083051F895
:100EE000042F02F120043F2C3BD802F108040F2C00
:100EF00006D80232032A04D9002B08BF012300E0E0
:100F000002238142EBD1012B30680ED0022B1AD084
:100F1000736800F0030003F003039B0043EA001032
:100F2000B36803F00303184317E000F00F0040F02C
:100F30004000F7F7FFFDB068736800F00F0040EA6B
:100F40000310C0B209E000F03F0040F08000F7F766
:100F5000F1FD3079F7F7EEFD307ABDE8F840F7F7AC
:100F6000E9BD06F10C0734463A46002552F8043D27
:100F7000AD0003F18001FF2910D903F50041B1F55F
:100F8000803F02D245F0010508E003F50003B3F10C
:100F9000807F34BF45F0020545F00305B242E5D13C
:100FA00065F03F00C0B2F7F7C5FD05F00303022B63
:100FB000207807D0032B0CD0012B13D1F7F7BAFD03
:100FC00060780FE0F7F7B6FD6078F7F7B3FDA0782B
:100FD00008E0F7F7AFFD6078F7F7ACFDA078F7F71A
:100FE000A9FDE0780434F7F7A5FDBC424FEAA5055A
:100FF000DBD1F8BD10B50446C0B2F7F79BFDC4F3D2
:101000000720BDE81040F7F795BD10B504467F2CCA
:1010100006D964F07F00C0B2F7F78CFDE409F6E76B
:10102000E0B2BDE81040F7F785BD430083EAE07009
:10103000EBE72DE9F047314B86B093F8E0370746F0
:10104000012B01D004464AE006F045FC0546064661
:1010500003A96846FBF762FF039B049A02971344B7
:101060002B443F2B059519D90023684603A9032279
:10107000FBF780FF039B3BB9049B2BB9204A1370FD
:101080005370059BABB301E0FBF730FF039B049A61
:10109000059E134433447F2B2BD8029FDFF86090CA
:1010A0003946CA461AF8024BC4F18008B04528BF39
:1010B000B0460AEB04004444E4B2424606F0BCFBEE
:1010C000802C89F8004014D1C8EB0606504607EB87
:1010D0000801324606F0B0FB89F8006009E02546B9
:1010E00014F8011B21B1074B1868FDF73AFFF6E72A
:1010F000ED1B284606B0BDE8F08700BF2C1000208D
:101100000C2E0020703000200FB407B504AB53F84C
:10111000042B054900200193F6F714FF03B05DF896
:1011200004EB04B0704700BF21090108054A08B567
:10113000138801339BB21380034B1878FCF722FC11
:10114000002008BD220F00200C2900209148F0B596
:101150000368914A9C8AA4B2E1B211F0010F2ED02B
:10116000198821F400610904090C1980198889B2D1
:1011700041F48061198000211170517899B1917802
:1011800011B9D178FF290ED101219170117902296D
:1011900001BF198889B241F400611980517941F089
:1011A00001011982E1E0517901F0FE011982D37841
:1011B000FF2B00F0DA80784BFF211970D5E08E0705
:1011C0003AD5BFF35F8F1479E4B2012C13D1517873
:1011D00089B1917879B1198821F480610904090CE9
:1011E0001980BFF35F8F198B1988947189B241F40C
:1011F000007119801BE0198BBFF35F8F147966496A
:10120000022C0AD14C7844B1897831B1198821F483
:1012100080610904090C1980A1E014795E49032C4E
:1012200005D14C781CB18978002940F098809988C4
:1012300089B241F4806197E04D0756D50121917143
:101240005178002937D09178002934D011791C8841
:10125000022911781DD924F480642404240C1C80F4
:101260001E8A9568CCB2F6B249B26E54198889B21A
:1012700041F4007119800168A31C13700B8A0134BA
:10128000DBB264B22B558B889BB243F480638B80B6
:1012900026E0A4B244F400741C801D8A9668CCB287
:1012A000EDB249B275541B8A611C49B2DBB20334FA
:1012B0007354147014E09178374C09B9217B41B113
:1012C000198889B241F400711980137801331370C1
:1012D00006E0198889B241F4807119800123A37056
:1012E00001680B88DB05FCD43FE001F0400101F010
:1012F000FF05E1B114781F8A9668E5B2691C64B2F3
:10130000FFB23755C9B21679117049B2CC1CA6424A
:1013100001BF9C8824F480642404240C08BF9C80B2
:1013200013798B4221D11C4B02351D701DE027061D
:101330001BD511784CB2661C0AD0156901312C5DA1
:10134000C9B21C821479117049B28C420DD106E0E9
:10135000D17815701982517809B9117929B999880C
:1013600021F480610904090C9980137992F90040F5
:1013700001339C4208490CD100238B708B7933B127
:1013800001688B8823F440731B041B0C8B800023A3
:101390001375F0BD08290020902E002010B5224CB6
:1013A0002368998A89B211F4706F1EBF1F4A012009
:1013B000507511F4E06F2BD01A8B9A88890522F4AE
:1013C00080624FEA02424FEA12429A8020D41A8881
:1013D00092051DD41A88D0050FD51A88D105FCD4E2
:1013E0001A8892B242F400721A801A889205FCD4CC
:1013F0000F4B1878FCF7C6FA0AE01A8892B242F44A
:1014000000721A809A8822F440721204120C9A8098
:101410002268938A23F470631B041B0C9382034B92
:1014200000221A7510BD00BF08290020902E002050
:101430000C29002010B51D4C4000C0B2A3602361F0
:101440001B4B6071E17001200021217360702271DB
:1014500020751868617538B383889B0515D4038897
:10146000D9050DD447F230530288920502D5013BCD
:10147000FAD112E08BB103889BB243F480730380EE
:1014800083889BB243F44073838047F23053227DBC
:1014900012B1013BFBD100E013B9BDE8104045E6B5
:1014A000024B587D80F0010010BD00BF902E00203F
:1014B0000829002013B51F4B400002ACC0B2587180
:1014C00004F8012DD970012200211A7359701A7184
:1014D0001A75194A1C6110689C60597538B3828866
:1014E000920515D40288D4050DD447F230520188F4
:1014F000890502D5013AFAD112E08AB1028892B286
:1015000042F480720280828892B242F440728280F9
:1015100047F23052197D11B1013AFBD100E012B906
:10152000FFF704FE03E0034B587D80F0010002B09A
:1015300010BD00BF902E00200829002008B50848E3
:1015400006F0C9F9C0B209280246054B04DC013097
:101550002021C0B29954F6E700221A5408BD00BFFA
:10156000A82E0020642928BF6421F8B501FB00F5EE
:10157000642495FBF4F40646E4B20027FBB2A342D0
:1015800004D29F20FCF745F90137F7E7B4420BD2AC
:10159000142195FBF1F5C4EB8410663DC4EB80008B
:1015A0002844C0B2FCF735F90134E4B2B44201D2A8
:1015B0009A20F7E7F8BD2DE9F743FDF7C5FB924CFC
:1015C000A369C31A002BC0F2608300F5433303F50F
:1015D000A073A3618D4B1E78237FC6F38006F31A98
:1015E00018BF012326774EB1002B00F04E83884BA5
:1015F0005A789A7001225A701A702BE0844A2BB1E3
:10160000D37843F00203D37093785370D57805F004
:10161000020101F0FF0339B97D498968411A0029A7
:1016200003DB05F0010300E0012303F00107784923
:1016300017707BB1EA070DD50A7905230132D2B2C2
:10164000B2FBF3F303EB8303D31A724ADBB20B71E1
:10165000D35C4B706E4DDFF804822B787BB3EB7854
:1016600023F00203EB706C4B0344AE20AB60FCF73D
:10167000F4F808B1FCF7F6F888F80000002800F04C
:101680000483B020FCF7E9F84020FCF7E6F80020DE
:10169000FCF7E3F81020FCF7E0F84FF48067013F17
:1016A0000020BFB2FCF7B0F8002FF8D13846FCF7A5
:1016B00048F96A78594B53F82200FCF7C5F898F8B6
:1016C0000030002B00F0E1826B78062B00F2AA823A
:1016D000DFE813F00700A8021800780061017E011E
:1016E000E4014F494F4A504B4748F6F716FD012099
:1016F000FCF727F94448FCF7A7F80220FCF721F98A
:101700004A48A3E14A4F3B689B0735D5DFF8508133
:101710000A23B8F80010DFF84C91B1FBF3F203FB99
:10172000121399F8001092B29BB2009136484149C9
:10173000F6F7F3FCF9F7E6FC0120FCF702F9324872
:10174000FCF782F83C4B99F800201868B8F8003094
:10175000057902FB153164234B43C17802204D1BF0
:101760005543B3FBF5F5EDB2FCF7EBF82946152030
:10177000FFF7F8FE032500E001253B681F0540F157
:1017800051822E4B2E491F68642397FBF3F20968A0
:1017900003FB127300911C482A49F6F7BEFCF9F7C7
:1017A000B1FC2846FCF7CDF81748FCF74DF8FEF7DA
:1017B00097FB0746681CFCF7C4F815203946FFF76D
:1017C000D1FE2FE20120204FFCF7BBF81F48FCF7A9
:1017D0003BF83B68980747D51D4A0B48B2F9021001
:1017E000B2F900300091B2F904201A4901921A4A64
:1017F000F6F793FCF9F786FC0220FCF7A2F8024802
:10180000FCF722F8032530E0A82E00201934002030
:1018100014290020C0D10108404B4C0078B20108C7
:10182000C5D10108CED10108A5C10108D5D1010853
:10183000242F0020DAD10108101800201C180020E5
:1018400020180020F2D101082418002007D2010836
:101850000E1000201DD201082CD20108DD09002045
:10186000141800205400002002253B68D9071AD51F
:10187000784A7948B2F90210B2F900300091B2F911
:10188000042076490192764AF6F747FC05F10108F3
:10189000F9F738FC2846FCF754F85FFA88F86E48E8
:1018A000FBF7D2FF45463B681A0718D56D4A6A48D0
:1018B000B2F90210B2F900300091B2F90420674980
:1018C0000192694AF6F729FC6F1CF9F71BFC2846C0
:1018D000FCF737F8FFB26048FBF7B6FF3D46634AB6
:1018E0005E49B2F90030B2F902205B480092604ACA
:1018F000604FB2F9002005F1010801925E4AF6F747
:101900000CFCF9F7FFFB2846FCF71BF85248FBF7E5
:101910009BFF51493868F6F79BFA4F4805F0DBFF0B
:101920005FFA88F8C1B2092908D84B1CDBB2202223
:1019300062540021E21851701946F4E72144786896
:10194000F6F786FAF9F7DEFB4046FBF7FAFF424866
:10195000FBF77AFFB8684049F6F77AFA3E4805F097
:10196000BAFF0235EDB2C7B2092F08D87B1CDBB233
:101970002022E2550021E21851701F46F4E73F4B48
:10198000B3F9000002F0D0F9E119F6F761FAF9F7BE
:10199000B9FB284657E00025394F3B78AB4240F26F
:1019A00041810E2D00F03E8168080130FBF7C9FF30
:1019B000284600F0F7FF3B78AB4206D92020FBF722
:1019C00028FF681CC0B200F0EDFF0235EDB2E3E77E
:1019D0002C4D2D4995F8B8271F48F6F79EFB01209E
:1019E000FBF7AFFF1C48FBF72FFF284B28491F7858
:1019F00019483A46F6F791FB0220FBF7A2FF16487A
:101A0000FBF722FF0C2303FB0755224995F8BB2760
:101A100095F8BA371048F6F780FBF9F773FB032007
:101A2000FBF78FFF0C48FBF70FFF95F8C01795F8F1
:101A3000BE2795F8BF37084800911749F6F76DFBA8
:101A4000F9F760FB0420FBF77CFF0348FBF7FCFE83
:101A5000E8E000BF440F0020A82E00201DD201089E
:101A600030D20108502C00202ADF01081C2F002052
:101A70001C100020802B002034D20108E00100203F
:101A8000201F00202C10002038D20108DC2E00205E
:101A900044D2010855D2010866D201087C4B1B686C
:101AA0001B0640F1BB80236A616A7A4A8B421CBFE5
:101AB000536292F828304FF001011CBF013303F04C
:101AC00003034FF0000018BF82F82830FBF745FFF2
:101AD00094F82830704A0025D05CFBF79AFE02206B
:101AE0000121FBF73AFF6D4B3620EB5C0135C3EB70
:101AF000C30393FBF0F0C0B2062828BF062060386D
:101B0000C0B2FBF786FE102DEDD1654B65491B7801
:101B1000604813F0020F644B1A7814BF59234E2308
:101B2000F6F7FBFAF9F7EEFA0220FBF70AFF59483D
:101B3000FBF78AFE5D495E4B4D680A68554892FB8B
:101B4000F3F25C4995FBF3F3F6F7E7FAF9F7DAFA03
:101B50000320FBF7F6FE4F48FBF776FE564B57493E
:101B60001A884C48F6F7D9FAFFF7E8FC0420FBF78F
:101B7000E8FE4848FBF768FE514B52491A88454831
:101B8000F6F7CBFAFFF7DAFC04210A20FBF7E5FEB3
:101B90004048FBF759FE4C49E26A3E48F6F7BDFA69
:101BA0004A4DFFF7CBFC0520FBF7CBFE3948FBF78E
:101BB0004BFE6A68AB6846493648F6F7AEFAFFF75F
:101BC000BDFC05210A20FBF7C8FE3248FBF73CFEAE
:101BD0002B69EA683F49D21A2E48F6F79EFAFFF7BA
:101BE000ADFC0620FBF7ADFE2A48FBF72DFEAA68E8
:101BF00039492848F6F791FAFFF7A0FC06210A2098
